:020000040000FA
:040000006FD00400B9
:101000006F00107D00000000000000009020002014
:10101000AA220020A9BDF9F56C23002000000000E1
:10102000000000006C230020902000200000000041
:101030000000000090200020000000009020002010
:101040000000000090200020902000209020002030
:101050009020002090200020402F00207A240020A3
:101060000000000090200020902000200424002098
:1010700090200020D22300209020002090200020EB
:101080009020002090200020902000209020002020
:101090009020002001A04111B7170040985F3AC688
:1010A000945F3247E39CE6FE3245410182800111A4
:1010B00013078008F337078093F787083EC20100C3
:1010C0000100B7170040930570052380B70413068D
:1010D00080FA2380C7040100010083C6B70493F699
:1010E000F60DA385D704238007049246F3A6068055
:1010F0000100010093760502D5CEF336078093F602
:10110000860836C4010001002380B7042380C70489
:1011100001000100B70614007D89558D88C70100C4
:1011200001000100010023800704A246F3A6068007
:101130000100010073370780137787083AC6010062
:1011400001002380B7042380C704010001000100CF
:1011500001003727004093061005A303D7802380A2
:101160000704B247F3A70780010001009307800836
:10117000F3B7078093F787083ECE01000100B71749
:101180000040130770052380E704130780FA2380CB
:10119000E7040100010003C7B70413670708A3852C
:1011A000E70423800704F247F3A70780010001004A
:1011B0000561828093760504BDC6F336078093F6F9
:1011C000860836C8010001002380B7042380C704C5
:1011D00001000100B7061400938606047D89558D31
:1011E00088C7010001000100010023800704C246F6
:1011F000F3A6068001000100733707801377870884
:101200003ACA010001002380B7042380C70401000B
:1012100001003727004093062005A303D7802380D1
:101220000704D24781B773370780137787083ACC12
:10123000010001002380B7042380C70401000100DE
:1012400098471367070C98C723800704E24719BF24
:101250000111814601468145114506CE97000000E7
:10126000E780C05693078008F3B7078093F7870895
:101270003EC601000100B717004013077005238028
:10128000E704130780FA2380E7040100010003C785
:101290006704136717002383E70423800704B2471A
:1012A000F3A7078001000100F2400561828041112F
:1012B000814601468145114597000000E7800051B5
:1012C00013078008F337078093F787083EC40100AF
:1012D0000100B7170040130670052380C70493066A
:1012E00080FA2380D70401000100FD552396B70240
:1012F00023800704A245F3A5058001000100733790
:101300000780137787083AC6010001002380C704CD
:101310002380D7040100010003C767041367170087
:101320002383E70423800704B247F3A70780010063
:10133000010001A0B1473305F50201007D1575FDDF
:101340008280411122C426C206C6AA8401446317C2
:101350009400B24022449244410182800504130566
:10136000803E420497000000E78000FD4180C5B741
:101370009305000273A04580824573901534924016
:101380002242B2424243D2436244F2440255925551
:101390002256B2564257D2576258F25806499649D9
:1013A000264AB64A464BD64B664CF64C065D965DD1
:1013B000265EB65E465FD65F09617300203041113C
:1013C000B7170040985F3AC6945F3247E39CE6FE49
:1013D000324541018280B71700401307000323887C
:1013E000E702854717170000232EF74473002030CB
:1013F000411122C406C637040020976000E0E78050
:10140000E0241C408297D5BF373700408347470010
:101410009146BD8B639ED702B73600401306F00F8E
:10142000973500009385051F9737000083D7872ED7
:1014300003C7A6001377F70F1DE3B7E70400BC4FFF
:101440000946894517150000034585F7829731A0A5
:1014500099466394D700834757007300203003C731
:1014600086001377F70FE365F6FC13851700AE9738
:10147000173800002310A82A2380E70075B7B78724
:10148000004003C76700098B6309071003C7770093
:101490009306000313770703630DD708173800007E
:1014A0000348D87417360000130686730547B30641
:1014B00006012380E60083C5770017370000130775
:1014C000A772429793F5F50F2300B70003C5870075
:1014D0009735000093850571C2951375F50F23802C
:1014E000A5000347070089451377F703630CB70C82
:1014F00063E7E50A6306071A8545630CB712973759
:10150000000083C7B76E3307F60003470700137761
:10151000F70F19CB850793F7F70F0D476363F71A9A
:1015200017370000A304F76CB787004009472383EF
:10153000E700B787004083C77700E207E18763DEF3
:1015400007049737000083C7776A1737000013072F
:1015500027693E9785462300D700173700001307F9
:10156000A7683E97930600032300D70017370000B3
:10157000130747673E97A14685072300D70093F7D7
:10158000F70F0D476364F71417370000A300F766E1
:10159000B787004009472383E70073002030930694
:1015A00010026300D70E930620026305D706930648
:1015B0000002E316D7F403C727021377C70F136798
:1015C0002700D5A803C767001377070465CB03C7B7
:1015D000A70217380000130828421735000013052A
:1015E0006539134707082385E70203C7A702137766
:1015F000370F136787002385E7028147130700042D
:10160000B305F5008C41B306F80091078CC2E3994D
:10161000E7FEF5B503C7A702134707042385E702D2
:1016200003C7A7021377C70F136727002385E702B5
:10163000F9B503C767001377070449C303C76702F7
:10164000173800001308082F17350000130545262A
:10165000134707082383E70203C767021377370F8F
:10166000136787002383E702814713070004B3054C
:10167000F5008C41B306F80091078CC2E399E7FEB0
:10168000BDBD03C76702134707042383E70203C7EF
:1016900067021377C70F136727002383E70285B517
:1016A00003C767001377070411CB03C7270213771B
:1016B000370F136787002381E70291B52380060067
:1016C0003DBD97370000A3830752B9BD973700008F
:1016D000A38E075075BD2303048015472303E480C0
:1016E00001002302A480828083076480E3CE07FE8A
:1016F00023030480828083076480E3CE07FE0345D2
:101700004480828083076480E3CE07FE2302A480A6
:101710008280411126C44AC24EC006C61377F50B1B
:10172000AD47AA892E899544630CF70019459700A7
:101730000000E78080FA97000000E78020FB8D44DE
:101740004E8597000000E78040F9FD59FD1463982D
:101750003401B240A24412498249410182801355AA
:1017600009011375F50F97000000E780E0F92209E1
:10177000F1BF011126CC06CEB70408009700000087
:10178000E780C0F6154597000000E78000F5970058
:101790000000E78080F697000000E78000F62AC688
:1017A00097000000E78080F432459377150089EBBD
:1017B000136515001375F50FF240E2440561828050
:1017C000FD14E9F00145CDBF397126DC4ADA4ED867
:1017D00052D656D45AD25ED006DE62CE66CCB7E779
:1017E00000E07D5783AA070022C603AA470023A072
:1017F000E71823A2E718B7170040130770052380E6
:10180000E704130780FA2380E70483C74704930B98
:1018100075FFB684E20793FBFB0F8546AA892E8BE2
:10182000328937240040E187015763FA7601630863
:10183000D5008946130700026313D5000157D98FDD
:1018400093F7F70FB71C00402382FC0411472303D2
:10185000E4801305F00F97000000E78000E8094CD2
:1018600097000000E78080E863657C15B7050700F6
:10187000DA9537870700795563FEE504B38795004D
:10188000636AF704370B0800A94733EB65016395DA
:10189000F90881E8814497000000E78020E526856B
:1018A00015A8DA85094597000000E780C0E605091C
:1018B0000345F9FFFD14050B97000000E780C0E425
:1018C00081C49377FB0FE5F797000000E780A0EA5B
:1018D00069F17D55B7170040130770052380E704B1
:1018E000130780FA2380E70403C74704418B238250
:1018F000E704F250B7E700E023A0571123A24711F5
:10190000E25432445259C259325AA25A125B825B93
:10191000724CE24C21618280A547639BF906856980
:101920001309F00FB3069900B3742B01B694134951
:10193000F9FFB3749900856B33796901416B938723
:10194000F9FFB3F7270199E363FC340193D9490008
:10195000C147E3E637FF3DBF0569C1697D19D9B7C6
:101960001305800D63886901130500026384790102
:1019700013051008CA8597000000E780C0D99700BA
:101980000000E78040DF31D54E99B38434416DBF0C
:10199000DA852D4597000000E780E0D7CA94E30B75
:1019A00099EE050997000000E78020D5A30FA9FE56
:1019B000FDB79387F9FF93F7F70F636DFC0C83C7AF
:1019C0001C04130730086315F70637070800636126
:1019D000EB06B3079B00B706100063FBD704334B3D
:1019E000EB0089476399F9068980D549E38404EAC5
:1019F000DA85094597000000E780E0D11109032747
:101A0000C9FF91472320E48003076480E34E07FE6B
:101A100023033481FD17EDFBFD14110B81C4937773
:101A2000FB0FE9FF97000000E780E0D461F155B5B6
:101A3000B717004003C75704B7070800137707021A
:101A400019E3B78707007955E376FBE833079B0076
:101A5000E3F9E7F841B58547E380F9F0DA852D45EC
:101A600097000000E78020CB9389F4FFE38404E231
:101A700097000000E78060C893F7390091EB832658
:101A800004800327090093074900E396E6E03E89B6
:101A9000CE84D9BFB5476399F9001305900B970021
:101AA0000000E78080C3FDB3B1471305B00AE388A7
:101AB000F9FE99476397F904B7050800B365BB00C1
:101AC0002D4597000000E78000C581448D4BA1495A
:101AD00097000000E78060C263967401832704804A
:101AE0002320F9008504E39534FF8327048013172E
:101AF0002B01635507002312F90069BB2322F9006B
:101B000051BB9D47639FF90281451305B0049700BF
:101B10000000E78040C0BD442320090023220900C3
:101B2000FD5997000000E78040BD93F77400CA9705
:101B300003C70700FD14398D2380A700E39334FF0A
:101B400091BBA1476397F90697000000E780A0C208
:101B50008144630D0B008D479304C0036308FB00B1
:101B60009304000563048B01930440041375C507B7
:101B7000E30295D2194597000000E78000B6970070
:101B80000000E780A0B6054597000000E780E0B4BC
:101B9000268597000000E78020B7094597000000E0
:101BA000E78080B697000000E780E0BCE31405CE34
:101BB0000DB39147639FF90013056006970000007D
:101BC000E780A0B197000000E78040B213059009BC
:101BD000F9B5E38109CCF1547DB9BD6601471736EB
:101BE00000001306E61D938606A68545834706007A
:101BF00093F7F70F91C382800507E3F9E6FE973765
:101C00000000238FB71ADDB77D1662066186931731
:101C10008601E18763D4070001458280931726007F
:101C20003307F500AE9718439C4363E7E7007D1642
:101C3000E37FF7FC7D55828005458280FD15E20536
:101C4000E18513978501618793F7F50F63480700D6
:101C5000FD15139725002A97584365D7138517005C
:101C60006205618582803308B5021C4283A80600A4
:101C7000B335B502C29733B50701AE98469585488E
:101C80006367B5006394A50063E3070181480C43D3
:101C9000C6950CC388C21CC28280814713978701F6
:101CA00061876343B7008280139727002A97232018
:101CB00007008507E5B78147014793968701E186CD
:101CC00063C5B60013351700828093962700AA9645
:101CD00094428507558FD5B793D755408A07AA9761
:101CE0009C4305453315B5007D8D828017F3FFDFDA
:101CF000E702A33D2A8497000000E78060F405C551
:101D0000931725003E940327C4FF814711EB7D15EF
:101D100016053E954205418517F3FFDF6700233D19
:101D200005838507E5B70145C5BF8147139787013F
:101D300061876343C700828013972700B386E5005D
:101D400094422A97850714C3D5B77D16620661862B
:101D5000014793178601E18763D507001335170004
:101D6000828093172600B306F500AE9794429C43F9
:101D70007D16B58F5D8FF1BF8A05AA950147636314
:101D8000B500828083A6C5FFF11593D71600D98FC1
:101D90009CC11397F601E5B72A8301480147014525
:101DA0006343D7008280B387050183A80700B30788
:101DB00006019C43C697AA976384F80033B51701C0
:101DC0000507B3080301620723A0F8006187110823
:101DD000C1BF2A8301478147014563C3D700828081
:101DE0003388E50083280800330EE600032E0E003A
:101DF0003388A8403308C8416384080133B508011B
:101E00008507B308E300E20723A00801E187110773
:101E1000E9B717F3FFDFE702432B0111B286B28463
:101E20002E86AA850A8597000000E780C0FA2A84DA
:101E3000A6850A8597000000E78020E833348000FB
:101E4000060413351500018D056117F3FFDF6700E8
:101E5000032A17F3FFDFE702C3244111AA89AE8AE0
:101E6000328BB68402C202C402C60144131C840130
:101E7000135C8C4163499C02939B1400FD1B054934
:101E8000138CF4FFF15C33048901620461846340C4
:101E9000740792478E04CE9423AEF4FE410117F3EB
:101EA000FFDF6700832313192400B30B2B01014AC2
:101EB00093172A00D69783A50B0088437800340037
:101EC000500097000000E78040DA050A93178A0166
:101ED000E187F11BE35EFCFC92474E990504232049
:101EE000F900A2473EC2B24702C63EC441B7131A28
:101EF0008901135A8A41131D240093178A01E1872F
:101F000063CF970092470A044E941CC0A24705096C
:101F10001379F90F3EC2B24702C63EC4ADB7B3074C
:101F20009A0313152A005695084178003400500092
:101F3000050AEA97DA978C4397000000E780E0D221
:101F40006DBF0000197106C212C416C61AC81ECA97
:101F500022CC26CE2AD02ED232D436D63AD83EDA69
:101F600042DC46DECAC0CEC2D2C4D6C6DAC8DECA99
:101F7000E2CCE6CEEAD0EED2F2D4F6D6FAD8FEDA49
:101F8000971500009385858B8841E70005009240F6
:101F90002242B2424243D2436244F2440255925535
:101FA0002256B2564257D2576258F25806499649BD
:101FB000264AB64A464BD64B664CF64C065D965DB5
:101FC000265EB65E465FD65F096173002030000072
:101FD0009721002093810103175100201301818272
:101FE00017F5FFFF1305450297050020938585012E
:101FF000171600201306C6FD63FAC50083220500EC
:1020000023A0550011059105E3EAC5FE170502005E
:102010001305C520971500209385C5FB17160020D2
:102020001306466563FAC5008322050023A0550008
:1020300011059105E3EAC5FE171500201305856318
:1020400097450020938585236377B50023200500FD
:102050001105E36DB5FEFD42739002BC8D42739095
:102060004280B722000093828288739002309702E8
:102070000020938222F993E23200739052309752FB
:1020800000009382A29D739012346FB07477730036
:102090002030397101436EC619A0397141536AC8A5
:1020A00066CA62CC5ECE19A0397101535AD056D29D
:1020B00052D44ED64AD826DA22DC06DE33016140FD
:1020C000828241114AC026C222C406C68282B24D13
:1020D0004101024D924C224CB24B4101024B924ABB
:1020E000224AB2494101024992442244B24041018C
:1020F00082803D432A876373C3029377F700BDEF65
:10210000ADE5937606FF3D8ABA960CC34CC30CC767
:102110004CC74107E36BD7FE11E28280B306C34090
:102120008A069702000096966780A6002307B700EC
:10213000A306B7002306B700A305B7002305B70021
:10214000A304B7002304B700A303B7002303B70019
:10215000A302B7002302B700A301B7002301B70011
:10216000A300B7002300B700828093F5F50F939684
:102170008500D58D93960501D58D61B7939627007F
:102180009702000096968682E78086FA9680C117AD
:102190001D8F3E96E374C3F8A5B73367B500FD53B2
:1021A0000D8B79E7B7877F7F9387F7F710419441CD
:1021B000B372F6003363F600BE92B3E26200639737
:1021C000720C6318D6065041D441B372F6003363E3
:1021D000F600BE92B3E262006398720A631BD604F3
:1021E00010459445B372F6003363F600BE92B3E235
:1021F00062006391720A631ED6025045D445B372E1
:10220000F6003363F600BE92B3E26200639A72088E
:102210006311D60210499449B372F6003363F60095
:10222000BE92B3E26200639372085105D105E30FD9
:10223000D6F61317060193970601631CF700135790
:10224000060193D706013305F7409375F50F91E921
:1022500082804183C1833305F7409375F50F91E187
:1022600082801377F70F93F7F70F3305F7408280DB
:102270000346050083C60500050585056313D600E2
:1022800065FA3305D640828011059105E312D6FE2A
:10229000014582802105A105E31CD6FC0145828011
:1022A0003105B105E316D6FC014582804105C10523
:1022B000E310D6FC01458280B717004003C77705BD
:1022C0001377E70FA38BE704130700F8A38DE70448
:1022D0003D47238CE70413075003A38CE70403C78F
:1022E000A7051377D70F238DE7048280B717004027
:1022F00003C7E7020D8941111377C70F498F930672
:102300008008F3B6068093F6860836C60100010001
:10231000930670052380D704930680FA2380D704A0
:10232000010001002387E70223800704B247F3A7D7
:102330000780010001004101828041112A83014E82
:10234000930E407E130F0019930F400663E56E1243
:102350009308001913034006B3781503854E0D4FFB
:10236000A14F337365020D891335150063EFBE125B
:102370001308F6FF7946729842081358080133078C
:10238000C70213D61700BE0732976146B3F6C602DE
:1023900013068070B386C6023697A166F58F420792
:1023A0005D8FB716004083C7F60293F70708A303B3
:1023B000F1000346710083C7F60293F70708E39420
:1023C000C7FE83477100B716004093F7F70F638885
:1023D000071293078008F3B7078093F787083EC476
:1023E00001000100B7170040930670052380D70451
:1023F000930680FA2380D7040100010023AA070373
:1024000083C6170393E60608A388D7022380070430
:10241000A247F3A70780010001001166B71700402B
:102420007D16D45BC85F93854703A98EF18EF5FABC
:1024300093068008F3B6068093F6860836C6010038
:102440000100930670052380D704930680FA238049
:10245000D7040100010098C103C7170313670704DD
:10246000A388E70223800704B247F3A7078001008F
:102470000100410182807D133368E3039308E01675
:10248000630E08003368F3039308D016630808004E
:102490009378330093B818009388D81633081E0138
:1024A000131E0801135E0E0155B56393E50305483D
:1024B000638608000148630303002A887108729844
:1024C000FD15131E0801C205135E0E01C18179BD01
:1024D00013F8150063F4BF007908D5B71338180056
:1024E000E5BF83C7F60293F70708A303F10003468D
:1024F000710083C7F60293F70708E394C7FE83478A
:10250000710093F7F70FF1DFE9B531714AD966CB66
:1025100006DF22DD26DB4ED752D556D35AD15ECF09
:1025200062CD6AC96EC7AA8C02D897100000E780F6
:1025300020B12A8993078008F3B7078093F78708AB
:102540003EDA01000100B717004013077005238031
:10255000E704130780FA2380E7040100010003C7A2
:10256000F7021377770FA387E70203C7F702136712
:102570008700A387E70223800704D257F3A70780C9
:1025800001000100054597000000E78060D61307B1
:1025900080C13347E902116A93070AE893065002A3
:1025A000BD69930BA004814A014B13048008930476
:1025B00070057D1AB347F9023307D7023EC0FD8785
:1025C0003ECC938709A69309803E3347F7023AC26F
:1025D0007D873AC4334739038549B399990193D923
:1025E0003940B306D702B30B7703B3C6F602B3CBB9
:1025F000FB0236C6FD8636C893D6FB4136CEB746BB
:102600000F00938606243349D9028566938606FA1D
:10261000B3969601B389E902130760553309D902CD
:1026200093060010B389E9023349D902B3C9F9020C
:102630009316390036CA37190040FD8636D0930DFF
:10264000090493D7F9413ED2F336048093F6860805
:1026500036DC01000100930770052380FD0093061E
:1026600080FA2380DD00010001008346390593F6DE
:10267000860FA309D9048346390593E61600A309FA
:10268000D90423800D00E256F3A606800100010064
:10269000130C80FA116DF336048093F6860836DE4B
:1026A00001000100930770052380FD0023808D0148
:1026B0000100010083463905216693E60602A3095D
:1026C000D90483560905B3E6A6012318D904835615
:1026D0000905D18E2318D90423800D00F256F3A6E4
:1026E0000680010001008346390593F606026381E6
:1026F000061A03463905218A6DDE08189710000076
:10270000E78000987336048013768608B2C2010011
:10271000010023809D0023808D0101000100B71777
:10272000004003C637051376F60DA389C70403C618
:10273000370513660602A389C70483560905216677
:10274000B3E6A6012318D90483560905D18E2318B0
:10275000D90423800D009646F3A6068001000100EF
:102760008346390593F60602638B061483463905C2
:10277000A18AEDFE97000020E780E091AA8636D47A
:1027800097000020E7802091A256E30AD5FE8356E9
:1027900009054255B3E6A6012318D9049710000095
:1027A000E780C08F83463905A18AEDDE035609050F
:1027B0008346290582473376CA00B306DA0293D5E9
:1027C000F641B296B388F640E24733B8C6002E9879
:1027D0003308F840A247B3B616013308D84063C7A0
:1027E0000701631DF800924763FA1701C247634F60
:1027F000F80E63950701B24763EAF80E894663E96C
:10280000660FF2469315180013D3F8015E861395F0
:102810001800B365B30042D646D497C00100E780E4
:1028200020BD3258050B137BFB0F63470001631A71
:102830000838A2586387083813081500B336A80073
:10284000B69513D6F5013298B336C800AE96135834
:102850001800FE06B3E60601733604801376860878
:10286000B2C60100010023809D0023808D0101007C
:1028700001000356C902B296C206C1822316D902CC
:1028800023800D00B646F3A606800100010021B5A5
:10289000F336048093F68608B6C001000100238059
:1028A0009D0023808D01010001008346390593E6D8
:1028B0000602A309D90423800D0086460DB5F33620
:1028C000048093F68608B6C40100010023809D00B1
:1028D00023808D01010001008346390593E606023D
:1028E000A309D90423800D00A646BDB5E30B0BF068
:1028F000F336048093F68608B6C8010001009306FB
:1029000080FA23809D002380DD00010001008346C2
:10291000390593F5FC0F93F6860FA309D904834676
:102920003905CD8EA309D90423800D00C646F3A630
:10293000068001000100130580FA0346390593065D
:1029400039051D8A631C9629733604801376860820
:10295000B2CC01000100130680FA23809D00238081
:10296000CD000100010003C606001376F60D23809A
:10297000C60003C60600136606022380C6008356FF
:1029800009051166D18E2318D904835609052166DD
:10299000D18E2318D90423800D00E646F3A60680C5
:1029A00001000100130680FA8346390593F60602FA
:1029B0006380062683463905130C3905A18AFDDAA2
:1029C000081897000000E780A06BF336048093F6A8
:1029D0008608B6D001000100930680FA23809D008E
:1029E0002380DD000100010083460C00116693F690
:1029F000F60D2300DC0083460C0093E6060223005C
:102A0000DC0083560905D18E2318D90483560905A5
:102A10002166D18E2318D90423800D008656F3A693
:102A2000068001000100130680FA8346390593F6FB
:102A30000602638A062083463905A18AEDFE97F0D7
:102A4000FF1FE78040652A8C97F0FF1FE780A06496
:102A5000E30C85FF8356090511664255D18E231874
:102A6000D90497000000E7806063834639051306A8
:102A70003905A18AFDDAF336048093F68608B6D4C8
:102A800001000100930680FA23809D002380DD0071
:102A9000010001008346060093F6F60D2300D600E0
:102AA00023800D00A656F3A6068001000100835680
:102AB000090503462905D247B376DA003306CA0270
:102AC0001305800C9355F6413696330DF640825728
:102AD000333CD6002E9C3336A601330CFC40330C1D
:102AE000CC403308850392564E86B335A503330593
:102AF000A503C29597C00100E780808F63468001DF
:102B0000631E0C16630C0D16130615003335A60054
:102B10002E959356F5013696B335D600AA95939621
:102B2000F50105828585D18E6346B000639D051A47
:102B3000638B061A0356C90215823305D600333655
:102B4000C500B2956348B000639105241306F00FE9
:102B5000637DA622894663F3561593078008F3B771
:102B6000078093F78708BED60100010037170040A1
:102B7000930770052300F704930780FA2300F704F6
:102B8000010001008356C70289678117D58FC207EC
:102B9000C1832316F70223000704B657F3A7078063
:102BA00001000100FA506A54DA544A59BA592A5AB3
:102BB0009A5A0A5BFA4B6A4CDA4C4A4DBA4D296173
:102BC00082801308F5FF3335A800FD152E951356A6
:102BD000F5013298B336C800AA9695B9F336048049
:102BE00093F68608B6CA0100010023809D00238069
:102BF000AD000100010083463905CD8EA309D9043B
:102C000023800D00D646F3A606800100010035B3EF
:102C1000F336048093F68608B6CE010001002380C7
:102C20009D002380CD00010001008346390593E615
:102C30000602A309D90423800D00F646F3A60680F8
:102C40000100010095B3F336048093F68608B6D2EE
:102C50000100010023809D002380CD0001000100C0
:102C60008346390593E60602A309D90423800D00A3
:102C70009656F3A606800100010045BB9306F5FFBA
:102C800033B5A600FD152E959355F501AE96B3B557
:102C9000B600AA951396F501858269B5F3360480CE
:102CA00093F68608B6D801000100930680FA2380C7
:102CB0009D002380DD00010001008356C9020566E6
:102CC000011693F6F60FD18EC206C1822316D902E1
:102CD00023800D00C656F3A6068001000100850A78
:102CE00093FAFA0F95B233E6B60045C20356C9020D
:102CF0003305D0403338A000B305B040B38505415B
:102D000015826345B000D1E16371A608894663F07E
:102D1000560593078008F3B7078093F78708BEDA54
:102D200001000100B7170040130770052380E70476
:102D3000130780FA2380E7040100010003D7C702CC
:102D40007D8B2396E70223800704D65781BDF33697
:102D5000048093F68608B6DC01000100930680FA31
:102D600023809D002380DD00010001008356C902FD
:102D70000566011693F6F60FD18EC206C1822316A0
:102D8000D90223800D00E656B9B793078008F3B740
:102D9000078093F78708BEDE010001003717004067
:102DA000930770052300F704930780FA2300F704C4
:102DB000010001000356C70293975600B297C2075D
:102DC000C1832316F70223000704F657C1BB9147BE
:102DD00063EEB70217D701001307074D8A05BA95AE
:102DE0009C41BA978287B717004003A7470B13454A
:102DF000F5FF698F23AAE70A03A7070B698F23A8AA
:102E0000E70A03A7070A798D23A0A70A8280B717CC
:102E1000004083A6470B1347F5FFF98E23AAD70A74
:102E200083A6070B558D23A8A70A83A6070A758FCB
:102E300023A0E70A8280B717004003A7470B498FFA
:102E400023AAE70A03A7070B1345F5FF45BFB717EA
:102E5000004083A6470B1347F5FF758F23AAE70AA7
:102E600003A7070A598D4DB7B717004003A7470BB3
:102E7000498FEDB7914763EEB70217D701001307EB
:102E8000E7438A05BA959C41BA978287B7170040F5
:102E900003A7470D1345F5FF698F23AAE70C03A786
:102EA000070D698F23A8E70C03A7070C798D23A0D2
:102EB000A70C8280B717004083A6470D1347F5FF84
:102EC000F98E23AAD70C83A6070D558D23A8A70C2E
:102ED00083A6070C758F23A0E70C8280B7170040EC
:102EE00003A7470D498F23AAE70C03A7070D134536
:102EF000F5FF45BFB717004083A6470D1347F5FF01
:102F0000758F23AAE70C03A7070C598D4DB7B71788
:102F1000004003A7470D498FEDB7797122D43714CC
:102F2000004026D24AD0035924028354040206D614
:102F30004209C2044ECE52CC56CA13590901C1806F
:102F40002DE11379F9F793F4F49F4209C204135960
:102F50000901C18093078008F3B7078093F78708BA
:102F60003EC401000100930770052300F404930799
:102F700080FA2300F404010001002311240323102C
:102F8000940223000404A247F3A707800100010074
:102F9000B250225492540259F249624AD24A4561CF
:102FA0008280B7F5070081463000B10519459700CA
:102FB0000020E7806081A24713972701E34A07FCBE
:102FC0001369090893E4044093098008F3B7098062
:102FD00093F787083EC001000100930A70052300A3
:102FE0005405130A80FA230044050100010023114F
:102FF000240323109402230004048247F3A70780CC
:1030000001000100294597F0FF1FE780A032F3B9C6
:10301000098093F989084EC201000100230054057C
:1030200023004405010001008357040293E70720B1
:103030002310F402230004049247B9B7B7170040E5
:103040008847420541819377050491EB9377F50119
:103050003755E801130505803345F50282809377E3
:10306000050C130700046397E7009377F5013745D4
:103070009C1CCDB72165130505D0828037E700E0A1
:103080001C435443A183E206D58F1CC1FD57232066
:10309000F7182322F718828013178500B7E700E09E
:1030A00023A0E710618123A2A7108280B7F700E078
:1030B0008847CC478280814737370040A14663C4A8
:1030C000C700328582800345B740E38EA6FE338574
:1030D000F5000345050085072304A740CDB79707F2
:1030E0000020938727EF9C43173700201307071909
:1030F0003E95636EE500173700201307A7506368FD
:10310000A700170700202327A7EC3E858280FD57E4
:10311000EDBF8280411122C406C62A8497000000B8
:10312000E78000F22947B307E502B2408D83B3D7A9
:10313000870222449507B3D7E70237370040C2071A
:10314000C1832316F70041018280411137150E001B
:1031500006C697000000E78020FCB7370040130741
:1031600070F82381E7000D47A381E70013070004EF
:10317000A380E70005472387E700B2404101828032
:1031800037370040834727001A0593F7F703C98FA5
:1031900093F7F70F2301F7008280B737004003C78A
:1031A000170019C9D98DA380B70003C7070013679B
:1031B00087002380E700828093C5F5FFF98DA38007
:1031C000B7008280AE872A87B7360040214637385D
:1031D000004089E7170300006700E3F383C8B600E7
:1031E000E30916FF05078348F7FFFD17C20723040D
:1031F0001801C183F9BF411122C406C62A84970071
:103200000000E780E0E32947B307E502B2408D8381
:10321000B3D7870222449507B3D7E7023737004078
:10322000C207C1832316F7404101828071654111B5
:103230001305052006C697000000E78000FCB7379D
:103240000040130770F82381E7400D47A381E74052
:1032500013070004A380E74005472387E740B240F7
:1032600041018280CC41411106C6328503C615005A
:1032700083C5050022064D8E42068D654186138862
:1032800075A2630C0611634BC804138845A2630042
:10329000060D634AC800938535A26301B6082390E2
:1032A000060029464DA0138855A26305060D938597
:1032B00065A2E316B6FE8D451D4663E6E508114698
:1032C000198E63F3C7003E86B7E704002390C6005B
:1032D000FC4797D501009385A5009DA0138895A272
:1032E00063030611634E060D1388A5A2630006133F
:1032F000938505A5E315B6FA99451D4663E5E504F2
:10330000198E63F3C7003E86B7E704002390C6001A
:10331000FC4797050020938525D61DA09D451D4699
:1033200063E3E5022146198E63F3C7003E86B7E7E3
:103330000400FC472390C6009705002093850534C0
:10334000BA9582970146B240328541018280AD45EF
:103350001D46E3EAE5FE3146198E63F3C7003E865B
:10336000B7E704002390C600FC4797D5010093857A
:10337000A5F9F9B7B1451D46E3E7E5FC3546198ED9
:1033800063F3C7003E86B7E704002390C600FC47FE
:1033900097D50100938545F865B78D451D46E3E453
:1033A000E5FA1146198E63F3C7003E86B7E70400BD
:1033B0002390C600FC4797D50100938525F349B7B4
:1033C0008D451D46E3E1E5F81146198E63F3C7000C
:1033D0003E86B7E704002390C600FC4797D501005E
:1033E000938545F5B1BFA5451D46E3EEE5F42946B5
:1033F000198E63F3C7003E86B7E704002390C6002A
:10340000FC4797D50100938525EF1DBFB5451D46A7
:10341000E3EBE5F23946198E63F3C7003E86B7E762
:1034200004002390C600FC4797D50100938545EA28
:1034300001BFB7E7040003A3071397060020938694
:10344000A6C24146A545170500201305E5B802832D
:103450002D455DE703C505000947631FE50803A87F
:103460004500411106C6034718003285034608008F
:1034700022074168518F930828FE6307170563E907
:10348000E80005186303070323900600294591A867
:10349000130648FE630AC7041518E31707FF15460D
:1034A0003E87637BF600154701A8130600023E879E
:1034B0006374F60013070002B7E704002390E600E8
:1034C000FC471316070111A83E8691C30546B7E7CE
:1034D0000400FC472390C6004206CC4541828297F7
:1034E0000145B24041018280130600083E87E37522
:1034F000F6FC13070008C9B7239006000545828033
:103500008280416779176304E504411122C406C62D
:1035100085472A84639FF500B7E70400228522448B
:10352000B24003A38713970500209385652F4101BF
:10353000028389476399F500B7E7040083A7070B67
:103540008545829771D9B2402244410182808280B0
:10355000797122D452CC2E842A8A97D50100938582
:1035600065DF17D50100130565E106D63AC626D2F8
:103570004AD0B68432894ECE97B00100E7808032BF
:10358000A68517D50100130565E097B00100E78017
:103590006031294597B00100E780A035834784005A
:1035A00093F70702E1E7834904008947054532475D
:1035B0006396F908544083C7160083C60600A20725
:1035C000D58FC166138616FE638CC7028D16638F76
:1035D000D7068D669386269029456391D706B7E76F
:1035E0000400A285225403A34714B250F249A686D0
:1035F0004A86925402595285624A85474561028340
:103600002D450DEF93070002354563E99702B7E7B3
:103610000400FC47484413060002CA85829781498A
:1036200097070020938787209C43014581CB9C43CB
:1036300091C74E852686CA8582970145B25022548D
:1036400092540259F249624A456182802D457DF7C4
:103650009307700F3545E3E397FEB7E70400FC4797
:1036600048441306700FCA8582975DBF2145F9B79C
:10367000411122C437E404008327841326C2AA849C
:10368000416506C697050020938585197D158297AB
:103690008327C40A170500001305E5E6858882978D
:1036A00095C0032304132244B2409244970600209D
:1036B000938606AE4146C545170500201305459C77
:1036C00041010283B240224492440145410182807B
:1036D00019C59707002023ABA714014582804545F3
:1036E00082801147636AA70A97D60100938646C570
:1036F0000A0536951841411106C63697AE87B28540
:103700000287130700026145639DE700B7E70400E5
:10371000FC4713060002170500201305A5F6829743
:103720000145B2404101828005476145E39BE7FEC8
:10373000B7E70400FC47054617050020130585F68A
:10374000F9BF1307700F6145E39DE7FCB7E704007D
:10375000FC471306700F170500201305E5F4C1B7E9
:10376000130700086145E39EE7FAB7E70400FC474A
:103770001306000817050020130585024DB71547ED
:103780006145E390E7FAB7E70400FC4715461705E3
:1037900000201305250961B709458280411126C221
:1037A000B7E4040083A7C41322C44AC006C62E840B
:1037B000970500209385C5062A898297058905C546
:1037C000970700209387C78B83D7A70BA28503A3F6
:1037D000440D2310F4002244B24092444A85024929
:1037E000014641010283B2402244924402494945C4
:1037F0004101828097070020238C07029707002051
:1038000023AA0702B717004003A7070CB706C0FF9B
:10381000FD16758F23A0E70C03A7070DB706400020
:10382000558F23A8E70C03A7070C3D9B23A0E70CAB
:1038300003A7070D1367070123A8E70C8280B717BA
:10384000004003A5470C83A7470C59811345150079
:10385000C18B058999E3136525009707002083C76D
:1038600027FD6380A702970700202383A7FC11C9C7
:1038700097070020938707FC03A307006303030057
:1038800002838280114517F3FFFF670043C841118F
:1038900093962500AA852D4506C697F0FF1FE78061
:1038A000A0F2B240014541018280011122CC06CE36
:1038B0003714004026CA4AC84EC652C48344740511
:1038C000034AB405834984050349940597F0FFFF33
:1038D000E780C09E8347A40593F4F40F137AFA0F90
:1038E00093E71700230DF40493F9F90F1379F90FF7
:1038F000B717004003C7A705058B6DFF03D5C705A4
:10390000A38D4705238C3705A38C2705A38B97042C
:10391000F2406244D2444249B249224A056182805F
:1039200041119397050122C406C626C2C1872E8481
:1039300063DC0700B7E40400FC54829719C1BC544F
:1039400082972165218D15A893F7150013C51500E1
:103950008DE793F725009DC797000000E78060EE94
:10396000B7E70400BC4F1306000A8945170500207D
:103970000345C5EC829713452400B240224492448B
:10398000410182809397250163D80702B7E40400C0
:1039900083A7C41E829797000000E780E0EEBC4C2E
:1039A00037560700130606308965170500200345C2
:1039B000E5E88297096579B7939715010145E3DE3C
:1039C00007FA17D50100130565A497B00100E78039
:1039D0004005B7E70400BC4F130600649165170566
:1039E00000200345A5E582971165A9BF2D71232A03
:1039F0009110FD74E98C232C81102328211123269A
:103A000031112A84AE893289930600100A86A68570
:103A10002D45232E111097F0FF1FE780E0DA1315D4
:103A20004401B7E70400FC4751810A0513962900B9
:103A3000CA850A958297A68585660146254597F031
:103A4000FF1FE78060D80A86A685930600102945E7
:103A500097F0FF1FE78040D78320C1110324811115
:103A600083244111032901118329C110156182802A
:103A7000B7F7070003C70701411106C622C426C2D3
:103A80004AC0A547631DF70097000000E78040F695
:103A9000B24022449244024901454101828013947C
:103AA0002500AA843289A286AA850146254597F079
:103AB000FF1FE78060D1A2864A86A685294597F038
:103AC000FF1FE78060D0E9B71D71A2CC37E4040086
:103AD0005C5C485886CE494697D501009385858E13
:103AE000829711E917D501001305058F97B00100E2
:103AF000E78020F301A0B7F600E0795798CAFD5798
:103B0000DCCA0567B7E700E023A0E7101306F00260
:103B100090C223A0E71801000100370700201847D2
:103B20001306000481459706002023A7E6D04157DD
:103B3000A38AE7403C4408088297970700209387B0
:103B4000E76C3EC8856713870740231AE1001D67AD
:103B50003ACC37070105130707103ACE938757D1A0
:103B60001307B00F2310E1022312F102054797F764
:103B7000FFFF9387E7532301E1023ED817070000B8
:103B8000130727D197070000938767D2B7F507007F
:103B9000BAC23EDC170700001307C7ED9707000005
:103BA000938787CE81463000E1051945BAC43EDED1
:103BB00097F0FF1FE78040C1180881479946300001
:103BC0003E960346060085070507A30BC700E3984A
:103BD000D7FEC24791C70357410185676373F7005A
:103BE00001A0B7E7040083A7470A08088297AA85BF
:103BF00011C917C501001305657F97B00100E78063
:103C000060CA01A0F640664425618280411126C247
:103C1000B7E4040083A7040806C622C41705000001
:103C2000130545D0829717040020130424C12300F4
:103C3000A40097000000E780800297000000E78062
:103C4000A0BB03450400224403A38405B240924470
:103C500013060032896541010283797106D622D4A8
:103C600013078008F337078093F787083EC20100E7
:103C70000100B7170040930570052380B7041306B1
:103C800080FA2380C7040100010083C6F70293F67F
:103C9000A60FA387D702238007049246F3A60680C7
:103CA0000100010073370780137787083AC40100C9
:103CB00001002380B7042380C7040100010003C76B
:103CC000F70213672700A387E70223800704A247B0
:103CD000F3A7078001000100054597E0FFFFE7809B
:103CE000206197000000E78020BA014781468147A4
:103CF000054685451305407E97E0FFFFE780206479
:103D000037E404003C446800514681458297B70778
:103D1000C0A83EC8B787E803938707D03ECA97E795
:103D2000FF1F9387C7693EC67C5868008297B250D0
:103D3000225445618280411197D50100938545D376
:103D400017C501001305856306C697B00100E7801B
:103D500060B517D50100130565EA97B00100E7804B
:103D600060B4B2402945410117B30100670063B850
:103D7000411197D501009385E5D017C501001305C2
:103D8000E55F06C697B00100E780C0B117D5010016
:103D9000130585E597B00100E780C0B0B240294522
:103DA000410117B301006700C3B4411122C406C624
:103DB000834705002A849DC797D50100938545D286
:103DC00017C501001305855B97B00100E78080AD42
:103DD0004C4017D501001305A5F097B00100E7800E
:103DE00060AC3DA058410DEF97D50100938545CFBC
:103DF00017C501001305855897B00100E78080AA18
:103E000017D50100130545EF97B00100E78080A9A1
:103E10002244B2402945410117B30100670063AD58
:103E2000A1679386D7036313D70297D501009385C3
:103E300025CB17C501001305655497B00100E78035
:103E400060A617D50100130525EC7DBFED0797D5BA
:103E500001009385E5C817C5010013052552631BB2
:103E6000F70097B00100E780E0A317D50100130524
:103E7000E5EA59BF97B00100E780C0A24C4017D5D2
:103E800001001305A5EB91BF411197D50100938562
:103E9000A5C017C501001305654E06C697B0010001
:103EA000E78040A0B2402945410117B301006700F7
:103EB00043A4797122D426D24AD02E842A898145FE
:103EC000B2844800714606D697E0FFFFE780A02243
:103ED00097F7FF1F9387874CDC4783D7070023148E
:103EE00021012313F10097500000E780E0C39547BC
:103EF000A305F1009307401F3EC6FD572305A1000F
:103F0000230AF10097500000E78040D62686A2855C
:103F1000480097500000E78000C4B25022549254E9
:103F2000025945618280971700202394077E9717D6
:103F30000020238D076CB7E70400BC47411106C67B
:103F400041468145170500201305851A8297972061
:103F50000000E780C05F97200000E780C040014577
:103F600097500000E780E068170700200347471AD2
:103F70009307F00A6315F7029307F0F889451705D0
:103F800000201305E518170700202303F7189707EB
:103F90000020A38F071697600000E78020909760AD
:103FA0000000E780E09C814537050400970700206A
:103FB00023AE0712970700202398071297070020C7
:103FC00023850712970700202396070A97070020EA
:103FD00023940708970700202397071097070020CE
:103FE0002390071297300000E780800C014597600E
:103FF0000000E780A09397D50100938565AC17C5B5
:1040000001001305A53797B00100E780A08917D5F7
:1040100001001305E5D897B00100E780A088B24001
:104020002945410117B301006700A38C411122C447
:1040300006C626C293F715002E84638F07108146AB
:1040400017F6FF1F1306C6328545170500200355D6
:10405000650097C00000E780A0F615C997D501005C
:104060009385C5A617C501001305453197B001001A
:10407000E780408317C501001305054897B001008C
:10408000E7804082294597B00100E780808697D578
:1040900001009385A5A317C501001305252E97B030
:1040A0000100E780208017C501001305254697A071
:1040B0000100E780207F294597B00100E7806083F9
:1040C00017F5FF1F1305852D5C4505472390E70075
:1040D00097400100E78020A797D501009385059FB1
:1040E00017C501001305852997A00100E780807B93
:1040F00017C501001305C54297A00100E780807A2B
:10410000294597A00100E780C07E930710F81707A4
:104110000020230FF7FE9707002083D767F31707C8
:104120000020A307F7FE17050020130565FEA183F5
:10413000914517070020230EF7FC97070020A38A5C
:1041400007FC97500000E780607513451400B240EB
:10415000224492444101828093F72500E1C317076E
:104160000020035767F845CB97060020938606F892
:10417000944297D701009387A7C4170600200346EF
:10418000C6F6814517050020130585F697700000D7
:10419000E7806002AA8441C197D501009385C59943
:1041A00017C501001305851D97A00100E780806FEA
:1041B000A68517C501001305253897A00100E780E3
:1041C000606E294597A00100E780A0729707002044
:1041D000239C07F0930710F817070020230AF7F233
:1041E0009707002083D7C7E617070020A302F7F23E
:1041F000A18317070020230EF7F091458D4717057F
:1042000000201305E5F017070020A304F7F09750EE
:104210000000E780A0681345240015BF93F7450010
:10422000D1C397D501009385259117C501001305CA
:10423000E51497A00100E780E06617C501001305AB
:10424000653197A00100E780E065294597A001004E
:10425000E780206A930720F817070020230AF7EA6F
:104260009707002083D707E117070020A302F7EA8A
:10427000A18317070020230EF7E8854717070020C2
:10428000A309F7E897500000E780409E170500203B
:10429000130505E8914597500000E780206013451D
:1042A000440075B593F78500A9C797D5010093859C
:1042B000A58817C501001305650C97A00100E780CC
:1042C000605E17C501001305252A97A00100E7804D
:1042D000605D294597A00100E780A0619707002055
:1042E000239407E097700000E780C0FC134584002A
:1042F000B9BD93F70501D1C38545170500200355C6
:1043000065D797600100E780E0AE97D501009385FF
:10431000A58217C501001305650697A00100E78077
:10432000605817C501001305652597A00100E780B7
:104330006057294597A00100E780A05B930730F8FC
:10434000170700202306F7DC9707002083D787D2C2
:1043500017070020A30EF7DA17050020130545DB29
:10436000A1838D45170700202305F7DA9750000039
:10437000E780C05213450401D9BB93F70502D1C7AA
:1043800097C501009385457B17C50100130505FFFF
:1043900097A00100E780005117C5010013054520D3
:1043A00097A00100E7800050294597A00100E78011
:1043B0004054930740F817070020230BF7D49707C2
:1043C000002083D767C917070020A303F7D4A18370
:1043D00017070020230FF7D2854717070020A30AED
:1043E000F7D297070020239907C697500000E7806F
:1043F000E087170500201305A5D1914597500000CF
:10440000E780C0491345040299B393F70504FDC33F
:1044100097C501009385457217C50100130505F680
:1044200097A00100E780004817C501001305C518D3
:1044300097A00100E7800047294597A00100E78089
:10444000404B9707002083C7A7CC1307700A6386E9
:10445000E7061307800A638CE7081307600A639373
:10446000E704930760F8170700202303F7CA9707AC
:10447000002083D747C717070020A30BF7C8A183E5
:10448000170700202307F7C8854717070020A30652
:10449000F7C8B14517050020130585C797500000E0
:1044A000E780C03F97400000E780407C134504044C
:1044B00097070020239907C259B9930770F8170787
:1044C00000202307F7C49707002083D7C7C1170729
:1044D0000020A30FF7C2A18317070020230BF7C208
:1044E000854717070020A307F7C2994565B79307CB
:1044F00080F8F1B793F705080145E38A07C497C52B
:1045000001009385656317C50100130525E797A092
:104510000100E780203917C501001305650B97A03E
:104520000100E7802038294597A00100E780603C22
:104530009307A0F817070020230CF7BC970700206B
:1045400083D707BC17070020A304F7BCA183170774
:1045500000202300F7BC854717070020A30BF7BAFC
:1045600097070020239E07B897400000E78000705F
:10457000170500201305C5B9914597500000E78045
:10458000E03113450408E1B6411122C497C501008A
:10459000938545562A8417C50100130525DE06C6F6
:1045A00097A00100E78000304C4017C501001305BB
:1045B000A57097A00100E780E02E294597A0010093
:1045C000E7802033034704009307F00F631FF702CF
:1045D00097C501009385055217C50100130505DA3B
:1045E00097A00100E780002C4C4017C5010013057F
:1045F000A56D97A00100E780E02A2244B24029453A
:10460000410117A301006700C32EB24022444101BB
:104610008280B1C1411122C417C50100130505D61E
:104620002E8497C501009385E54706C697A0010033
:10463000E7804027A28517C501001305257497A0C0
:104640000100E78020262244B2402945410117A3FA
:1046500001006700032A8280411122C426C22E84F1
:10466000AA8497C501009385A54417C501001305C9
:10467000E5D006C697A00100E780C02217C501005B
:104680001305857097A00100E780C021294597A0F8
:104690000100E780002697C50100938565419707D3
:1046A00000202399979A17C50100130525CD85444D
:1046B00097070020239E879897070020239B9798B1
:1046C000971700202397870497A00100E780801D9B
:1046D0009715002083D5E50317C501001305456B29
:1046E00097A00100E780001C294597A00100E78002
:1046F000402097170020238B97F097200000E78039
:1047000080C6228597500000E780A0EE05459750AF
:104710000000E780A02197F7FF1F938727C8DC4799
:1047200003D70700C167FD176312F7022244B7E7FA
:104730000400B240924403A3870517F5FF1F034509
:1047400065101306000A854541010283B2402244E8
:10475000924441018280011122CC37E404005C5C68
:1047600006CE354697C501009385854A17D50100C9
:1047700013058510829711E917C501001305C5C5FA
:1047800097A00100E780E02901A097F7FF1F93871A
:10479000270C3EC4B7F507008567938707808146DD
:1047A00017F6FF1F1306460AE10519453EC697E0B6
:1047B000FF1FE78060017C44194697F5FF1F938532
:1047C000A508170500201305258B8297340017F6DE
:1047D000FF1F1306660797D501009385A59417D58B
:1047E00001001305A59597600000E780C0712A8439
:1047F0001DCD97C501009385253317C5010013050D
:10480000E5B797A00100E780E009A28517C5010080
:104810001305054197A00100E780C008294597A02E
:104820000100E780000DF24062440561828097E05C
:104830000000E78020D417C50100130565359750A7
:104840000000E780006697A00000E780602897607E
:104850000100E780E08C17F5FF1F1305A5B0975006
:104860000100E780807517C5010013056533976067
:104870000100E780608D2A8497600000E78040CCCB
:1048800097000100E780C06497800100E780E0FDA9
:1048900097700000E780802497600000E780404226
:1048A00097300100E780202697C501009385C52732
:1048B00017C50100130585AC19C897A00100E78052
:1048C00060FEA28517C501001305C537A1B797A0E3
:1048D0000100E78020FD17C501001305E53897A00A
:1048E0000100E78020FC294597A00100E7806000D7
:1048F00097300100E780000297F00000E780C020B9
:1049000055C985453705040097200000E780407AA7
:1049100097C501009385452117C50100130505A61C
:1049200097A00100E78000F817C501001305453581
:1049300097A00100E78000F7294597A00100E780D4
:1049400040FB97F7FF1F9387279583D7070017171B
:1049500000202310F7DC8547171700202308F7CA2B
:1049600097200000E78020B997200000E780A09FF3
:10497000171500200355E5D997500000E78060C760
:10498000054597500000E78060FA97C501009385C0
:10499000A51917C501001305659E97A00100E780C2
:1049A00060F017C501001305E52F97A00100E7800F
:1049B00060EFADB597C501009385051717C50100D8
:1049C0001305C59B97A00100E780C0ED17C5010046
:1049D0001305053D97A00100E780C0EC294597A08D
:1049E0000100E78000F1014569BF411122C437E4AD
:1049F00004008327041A06C6829797500000E780B8
:104A000000C38327040817F5FFFF1305656282972B
:104A100097F7FF1F2388A7E217F5FF1F13050598D7
:104A200097400000E78020572244B240410117031D
:104A30000000670083D2B7E70400FC471171A2DDD4
:104A4000CAD986DFA6DBCED72E8432892E86AA85E8
:104A500017F5FF1F1305C56B829717F7FF1F130785
:104A6000276B83470700930680029387E70793F736
:104A7000F70FE3ECF610BA898A0717C7010013078E
:104A80002799BA979C43BA9782878D4797C50100AB
:104A90009385C50B17C501001305458E630FF40000
:104AA00097A00100E78000E017C501001305C5C805
:104AB00097A00100E78000DFBDA497A00100E78078
:104AC00060DE17C501001305A5C897A00100E780A7
:104AD00060DD294597A00100E780A0E1930720F859
:104AE000114697F5FF1F9385A5624A8517F7FF1FAB
:104AF0002300F76297F7FF1FA38D076097F0FFFF72
:104B0000E780603B2A841DC997C501009385050491
:104B100017C501001305858697A00100E78080D89E
:104B2000A28517C50100130565C697A00100E7809F
:104B300060D7294597A00100E780A0DB97C5010059
:104B40009385C50017C501001305458397A0010093
:104B5000E78040D517C50100130585C497A0010063
:104B6000E78040D4294597A00100E78080D84165BF
:104B7000930730FA054697F5FF1F938565597D1514
:104B800017F7FF1F2306F75897F0FFFFE780A032C3
:104B90002A841DC997C50100938545FB17B50100FF
:104BA0001305C57D97A00100E780C0CFA28517C57A
:104BB00001001305A5BD97A00100E780A0CE2945FF
:104BC00097A00100E780E0D2B7E70400BC4F05667C
:104BD000130606C8A14517F5FF1F0345A5C6829712
:104BE000FE506E54DE544E59BE5911618280914779
:104BF0006303F40297C50100938545F517B50100DD
:104C00001305C57797A00100E780C0C917C501004B
:104C1000130545BC71BDB7E70400FC4F914517F57E
:104C2000FF1F034525C2829797C50100938505F2B2
:104C300017B501001305857497A00100E78080C6B1
:104C400017C501001305C5BA97A00100E78080C50C
:104C5000294597A00100E780C0C997400000E78080
:104C6000E000914535A485476303F40297C5010030
:104C70009385C5ED17B501001305457097A0010098
:104C8000E78040C217C50100130505B815B597F7B1
:104C9000FF1F2391273FB7E704000566BC4F1306AB
:104CA00006C8C1450DBF8D476303F40297C50100D7
:104CB0009385C5E917B501001305456C97A0010060
:104CC000E78040BE17C501001305C5B5D5B39307EE
:104CD00040F8114697F5FF1F938585434A8517F7DE
:104CE000FF1F2307F74297F7FF1FA384074297F0A0
:104CF000FFFFE780401C2A84E30405EE97C501000E
:104D00009385C5E417B501001305456797A0010019
:104D1000E78040B9A28517C50100130525A797A014
:104D20000100E78020B8294597A00100E78060BC1A
:104D300045BD9147E31CF4F6B7E70400FC4F93052B
:104D4000000217F5FF1F0345E5AF829797C50100E5
:104D50009385C5DF17B501001305456297A00100D3
:104D6000E78040B417C50100130545ADF1BD894783
:104D700063E3870297C50100938545DD17B5010000
:104D80001305C55F97A00100E780C0B117C50100FA
:104D9000130505AC31BB97F4FF1F83C4843797F725
:104DA000FF1F83C7F73697C50100938525DAA20454
:104DB00017B501001305855CDD8C97A00100E78025
:104DC00060AEA28517C501001305C5A997A0010013
:104DD000E78040ADC204294597A00100E78060B19B
:104DE000C1849305D4FF93960401C1824A8693F54A
:104DF000F50F17F5FF1F1305D53197200000E78049
:104E0000E02EE35F90DC930750F817F7FF1F2301B4
:104E1000F73083C73900228697F5FF1F9385452F0A
:104E200085074A8517F7FF1FA305F72E97F0FFFFA9
:104E3000E78060082A84E30505DA97C501009385B9
:104E4000E5D017B501001305655397A00100E78071
:104E500060A5A28517C50100130545F1C9B58947AD
:104E600063E3870297C50100938545CE17B501001E
:104E70001305C55097A00100E780C0A217C5010027
:104E8000130505A035B197400000E78020DEA2851C
:104E900017F5FF1F1305C52797500000E78000A0F6
:104EA00081B38D476303F40297C50100938505CA5A
:104EB00017B501001305854C97A00100E780809E7F
:104EC00017C501001305859DE5B6B76602000146CA
:104ED000B7750200054597E0FF1FE780E08E930756
:104EE00060F817F7FF1F2305F72297F7FF1FA3822C
:104EF00007229307000617F7FF1F230DF7208947A6
:104F000017F7FF1FA308F72097F7FF1F2385072038
:104F100097F7FF1FA3810720C14717F7FF1F230D36
:104F2000F71E930720F917F7FF1FA307F71E314657
:104F300097F7FF1FA383A71E97F5FF1F9385451DB6
:104F40004A8597F7FF1F238A071C97F0FFFFE7802A
:104F500080F62A84E30605C897C50100938505BF3E
:104F600017B501001305854197A00100E7808093E4
:104F7000A28517C501001305E59355B3B147630337
:104F8000F40297C50100938565BC17B501001305B0
:104F9000E53E97A00100E780E09017C501001305EA
:104FA000259339B6B7E70400FC4F9305000417F5C5
:104FB000FF1F03452589829797400000E78000CBBB
:104FC000B145F9B5914763E3870297C50100938521
:104FD000E5B717B501001305653A97A00100E78012
:104FE000608C17C5010013056590D9B497F4FF1FB5
:104FF00083C4441297F7FF1F83C7B711A204DD8C47
:105000008E04B77702006D14BE942286A68517C55C
:1050100001001305E58E97A00100E780A088B7E79F
:105020000400FC47228697F5FF1F9385B50E2800E4
:10503000829793160401C1823000A685094597D056
:10504000FF1FE78060782A8409C917C5010013058E
:10505000E58C97A00100E780C09C930770F8194683
:1050600097F5FF1F9385C50A4A8517F7FF1F230190
:10507000F70A97F7FF1FA38F870897F0FFFFE780D6
:1050800080E32A84E30E05B497C50100938505AC3F
:1050900017B501001305852E97A00100E7808080D9
:1050A000A28517C501001305658895B99947630B5B
:1050B000F41297C50100938565A917B50100130582
:1050C000E52B97900100E780E07D17C501001305EF
:1050D0006587F9BA914763E3870297C50100938515
:1050E000E5A617B501001305652997900100E78033
:1050F000607B17C50100130565865DBA97F4FF1F35
:1051000083C4440197F7FF1F83C7B700A204DD8C57
:105110008E04B77702006D14BE942286A68517C54B
:1051200001001305E58497900100E780A077B7E7B9
:105130000400FC47228697F5FF1F9385B5FD2800E4
:10514000829793160401C1823000A6850D4597D041
:10515000FF1FE78060672A8409C917C5010013058E
:10516000E58297A00100E780C08B930780F819467D
:1051700097F5FF1F9385C5F94A8517F7FF1F230988
:10518000F7F897F7FF1FA38787F897F0FFFFE780EF
:1051900080D22A84E30605A497C501009385059B68
:1051A00017B501001305851D97900100E780806FFA
:1051B000A28517B501001305A57E95B6994763032F
:1051C000F40297C501009385659817B50100130592
:1051D000E51A97900100E780E06C17B50100130510
:1051E000A57DF9B0B7E70400FC4F9305000417E56F
:1051F000FF1F03452565829797400000E78000A7C1
:10520000994579B18D476303F40297C501009385F1
:10521000E59317B501001305651697900100E78027
:10522000606817B501001305A57A59B017B50100DC
:105230001305057B97900100E780A07E1305C0123F
:1052400097D0FF1FE780E00F014597E0FFFFE78061
:1052500020E30D4597100000E780009F294597D077
:10526000FF1FE780000E97D0FF1FE78060FE8DBA1A
:1052700099476303F40297C501009385258D17B5FF
:1052800001001305A50F97900100E780A06117B5F5
:1052900001001305A57529B817F7FF1F034797E706
:1052A00097F7FF1F83C707E722075D8F9166BA96BE
:1052B000C2061166C1821306F6EF8D476365D602FA
:1052C00097E7FF1F9387870D9C4B17F6FF1F034639
:1052D00056E49386C7002DC203D6070069CA890722
:1052E000E39CD7FE89471307A0F8114697F5FF1FE7
:1052F000938505E24A8597F6FF1F238BE6E017F7B3
:10530000FF1FA308F7E097F0FFFFE780C0BA2A84E9
:10531000E308058C97C501009385458317B5010007
:105320001305C50597900100E780C057A28517B502
:1053300001001305E56CE5B203D60700630EE60A2B
:105340008907E39BF6FE8D4779BF91476304F4021A
:1053500097B501009385857F17B5010013050502F8
:1053600097900100E780005417B501001305C56A46
:105370006FF00FF4B7E70400FC4F9305000817E542
:10538000FF1F0345254C8297C9B897B50100938547
:10539000E57B17B50100130565FE97900100E780D6
:1053A000605017B501001305A5686FF06FF02390EA
:1053B000E70017E5FF1F130565FE97200100E78052
:1053C000E07A97B501009385657817B5010013055C
:1053D000E5FA97900100E780E04C17B5010013054E
:1053E000256697900100E780E04B294597900100E2
:1053F000E78020508147C5BD2390070017E5FF1FB8
:105400001305C5F997200100E780407697B50100A4
:105410009385C57317B50100130545F697900100F4
:10542000E780404817B50100130505635DBF4111D2
:1054300022C406C6834705002A849DC797B501008C
:105440009385856C17B50100130545F3979001000E
:10545000E78040454C4017C50100130565979790BC
:105460000100E7802044E1A05841B707CF009387AF
:10547000777D631DF70697B501009385E56817B53D
:1054800001001305A5EF97900100E780A0411C449F
:105490008356E4008355C40003C6070017C5010006
:1054A0001305859497900100E780C03F29459790A8
:1054B0000100E78000440357E4009707002083D7EA
:1054C00047256309F7008355C400084497E0FFFFB0
:1054D000E78080CF0356E4008355C400084422448B
:1054E000B240410117F3FFFF67002355B707CC0017
:1054F0009387777D6315F70497B501009385C560A1
:1055000017B50100130585E797900100E780803902
:105510001C448356E4008355C40003C6070017C526
:1055200001001305658C97900100E780A0372244A5
:10553000B24029454101179301006700833BB7073B
:10554000CE009387777D6304F70297B501009385BA
:10555000A55B17B50100130565E297900100E78090
:1055600060344C4017B501001305457DCDBDB240F8
:10557000224441018280B7E70400FC4741112E8696
:1055800006C622C426C24AC02E842A89AA8517F5D7
:10559000FF1F1305E5B7829797B501009385C55C9A
:1055A00017B50100130585DD97900100E780802F76
:1055B00097F5FF1F83C5C5B517B501001305C502D3
:1055C00097900100E780002E294597900100E78021
:1055D000403297F4FF1F9384A4B383C7040041476C
:1055E0009387070693F7F70F636AF75C17B7010015
:1055F000130747EC8A07BA979C43BA9782879D475F
:105600006307F40297B501009385055617B50100AD
:105610001305C5D697900100E780C02817B5010093
:10562000130505FD97900100E780C027ADAC97F703
:10563000FF1F83C7F7ADDDCB17F7FF1F034777AD1C
:1056400097F7FF1F83C7E7AC22075D8F97F7FF1F10
:1056500083C747ACC2075D8F97F7FF1F83C797AB20
:10566000E207D98F17F7FF1F2322F7A883C764002B
:1056700097B501009385454F17B50100130505D077
:1056800017F7FF1F2303F7A697900100E7808021FB
:1056900097F7FF1F938787A58C4317F6FF1F0346D5
:1056A000C6A417B50100130565F697900100E780C1
:1056B000601F294597900100E780A02397F7FF1FFF
:1056C000A38807A42244B24092440249930700F8F9
:1056D00017F7FF1F230EF7A29D4517F5FF1F1305B0
:1056E00025A34101174300006700431B976000009A
:1056F000E780C0CB97F7FF1F238DA7A093578500A6
:1057000017F7FF1FA307F7A0935705012A8417F780
:10571000FF1F2301F7A093578501014517F7FF1FCE
:10572000A30AF79E97600000E78000C997F7FF1F64
:105730002383A79E97B501009385054317B5010004
:105740001305C5C397900100E780C01517F6FF1F2A
:105750000346669CA28517B501001305A5ECB1B7F9
:10576000CD476303F40297B501009385E53F17B574
:1057700001001305A5C097900100E780A01217B59E
:1057800001001305A5EB79BD37E404007C444146D4
:1057900097F5FF1F9385D59717F5FF1F13054595BF
:1057A000829717F5FF1F1305A59497100000E78057
:1057B000A0CD97100000E78000BB97F7FF1F83C7BD
:1057C000479617F7FF1F0347B795A20703238405E2
:1057D000D98F17F7FF1F2319F7901306000A894581
:1057E0002244B2409244024917E5FF1F0345850554
:1057F000410102838D476303F40297B5010093854D
:10580000A53617B50100130565B797900100E7802D
:10581000600917B50100130525F229B517F4FF1F1C
:105820000344248F97F7FF1F83C7978E97B5010016
:1058300093858533220417B50100130525B45D8CCB
:1058400097900100E7800006A28517B501001305B7
:1058500065E097900100E780E004294597900100FA
:10586000E78020090D4697F5FF1F9385658A2285FD
:1058700097E0FFFFE7802064AA8421C197B501006B
:105880009385852E17B50100130545AF979001004C
:10589000E7804001A68517B501001305E5DC979068
:1058A0000100E78020002244B24092440249294589
:1058B0004101179301006700C30397E7FF1F239B74
:1058C000877AB7E70400116603A38705130606E885
:1058D000914539B78D476303F40297B5010093856D
:1058E000A52817B50100130565A997900100E78069
:1058F00060FB17B501001305E5F22DB317F4FF1F88
:105900000344248197F7FF1F83C7978097B5010051
:1059100093858525220417B50100130525A65D8C06
:1059200097900100E78000F8A28517B501001305E4
:10593000E5D497900100E780E0F6294597900100B3
:10594000E78020FB0D4697E5FF1F9385657C228548
:1059500097E0FFFFE7802056AA841DC197B501009C
:105960009385852017B50100130545A19790010087
:10597000E78040F3A68517B50100130565D105B78B
:1059800097E7FF1F239A876CB7E70400116603A30C
:105990008705130606E89305000299B5894763E376
:1059A000870297B501009385251C17B501001305E3
:1059B000E59C97900100E780E0EE17B50100130524
:1059C00025E98DB197E4FF1F83C4A47497E7FF1FF7
:1059D00083C7177497B5010093850519A20417B5FD
:1059E00001001305A599DD8C97900100E78080EBFD
:1059F000A68517B50100130525CB97900100E78018
:105A000060EA294597900100E780A0EE228697E59D
:105A1000FF1F9385E56F268597E0FFFFE780A0498C
:105A20002A84630E051A97B501009385E51317B50F
:105A300001001305A59497900100E780A0E6A285D8
:105A400017B50100130585C799BD854763F9871808
:105A5000834519002244B24092440249B335B00054
:105A600097E7FF1F2382B76217B50100130545C6EC
:105A70004101179301006700E3E2A2852244B2408E
:105A800092444A850249410117030000670003223E
:105A900099476303F40297B501009385E50C17B5A8
:105AA00001001305A58D97900100E780A0DF17B5D1
:105AB00001001305A5F3BDB617E4FF1F0344646599
:105AC00097E7FF1F83C7D76497B501009385C50982
:105AD000220417B501001305658A5D8C97900100BB
:105AE000E78040DCA28517B501001305E5BF97905C
:105AF0000100E78020DB294597900100E78060DF07
:105B0000194697E5FF1F9385A560228597E0FFFF63
:105B1000E780603AAA841DC197B501009385C5044A
:105B200017B501001305858597900100E78080D7A0
:105B3000A68517B50100130525BC95B397E7FF1F90
:105B40002390875CB7E70400116603A3870513065B
:105B500006E89305000869B1854797B5010093856C
:105B6000A50017B5010013056581630BF40097903C
:105B70000100E78020D317B50100130525B95DB4F6
:105B800097900100E78000D217B50100130585B991
:105B900097900100E78000D1294597900100E780A8
:105BA00040D52244B2409244024997E7FF1F239D0B
:105BB00007524101175300006700C36F97B50100FA
:105BC000938585FA17A501001305457B9790010081
:105BD000E78040CD17B50100130585E5A1B4B240BB
:105BE00022449244024941018280411106C622C4E6
:105BF00097E0FFFFE780202C9377F50FA1C32A845D
:105C000097B501009385C5F717A501001305057722
:105C100097900100E78000C99375F40F17B5010054
:105C20001305C51497900100E780C0C72244B24015
:105C300029454101179301006700A3CBB2402244DC
:105C400041018280411122C491462A8417E6FF1F38
:105C50001306465A9D652D4506C697D0FF1FE7805F
:105C6000A0B6B7F7070003C70701A5476313F700FE
:105C700001A09306001001469D65254597D0FF1FA2
:105C8000E78080B497E7FF1F238687562244B240FF
:105C9000914617E6FF1F1306E6559D65294541010C
:105CA00017D3FF1F670043B21171CED7B7E90400C5
:105CB00083A7C904CAD917E9FF1F13096945A2DDE3
:105CC0002E8686DFA6DB2E84AA854A85829797E7F3
:105CD000FF1F83C7E7431307700A6385E710636DEF
:105CE000F7001307600A6385E704FE506E54DE5424
:105CF0004E59BE59116182801307800A6385E716E9
:105D00001307900AE393E7FE8D476306F41C97B5EB
:105D100001009385E51817A50100130525669790E6
:105D20000100E78020B817B501001305A51425A0D0
:105D30008D47630CF40297B501009385651617A58E
:105D400001001305A56397900100E780A0B517B582
:105D500001001305650B97900100E780A0B4294569
:105D600097900100E780E0B849B7854717B5010073
:105D70001305450B17E7FF1F2308F7309790010025
:105D8000E78020CAB7750200B766020001460545E4
:105D900097D0FF1FE78040A3930760F817E7FF1F26
:105DA0002308F73697E7FF1FA385073693070026DA
:105DB00017E7FF1F2320F736E5779387072117E7BB
:105DC000FF1F231BF734B14597E7FF1F23870734D5
:105DD00097E7FF1FA383A7344A8597000000E78059
:105DE000E01621B7914763E3870297B501009385D9
:105DF000250B17A501001305655897900100E78052
:105E000060AA17B501001305E503B1B797E4FF1FBA
:105E100083C4443097E7FF1F83C7B72FA204DD8CEC
:105E200083A7C9046D14228697E5FF1F9385952EDD
:105E3000280082978E0493160401B7750200C18270
:105E40003000A695094597D0FF1FE780E09793079C
:105E500070F817E7FF1F230DF72A994597E7FF1FF3
:105E6000A38AA72A95BF914763E3870297B50100EC
:105E70009385050317A50100130545509790010070
:105E8000E78040A217B50100130545FDE9B597E489
:105E9000FF1F83C4242897E7FF1F83C79727A20407
:105EA000DD8C83A7C9046D14228697E5FF1F9385B7
:105EB0007526280082978E0493160401B775020098
:105EC000C1823000A6950D4597D0FF1FE780C08F97
:105ED000930780F8BDBF17B501001305E5FA979049
:105EE0000100E78000B4930790F82304F100834792
:105EF00019008D452800A304F100834729002305DC
:105F0000F10097000000E78060041305C01297C0FD
:105F1000FF1FE7800043014597D0FFFFE780401651
:105F20000D4597000000E78020D2294597C0FF1F4C
:105F3000E780204197C0FF1FE78080317DB397E75E
:105F4000FF1F23A1A72C828097E7FF1F9387872B32
:105F500003A30700630303000283174300006700E5
:105F6000E39341114AC097F6FF1F83D6867A3289A0
:105F700017D6FF1F0356A64422C426C206C62A848B
:105F8000AE8497000000E780606435C12DC099475A
:105F900063FF97048347140003470400A207D98FC7
:105FA00013978700A183D98FC2073167C183130775
:105FB000C755639EE70297D7FF1F83D74740A301CA
:105FC000F400A1832302F40097F7FF1F83D76774BF
:105FD00091C7A302F400A1832303F400A68517B59B
:105FE00001001305E5EF97900100E780A08B97F77C
:105FF000FF1F83C7A761B9CF97D5FF1F83D5253C66
:1060000017B50100130585EF97900100E78080899F
:106010002686A28517D5FF1F0355653A9700000015
:10602000E780E0BC6301090497E7FF1F83C7C71D32
:106030009DCB95C897E7FF1F83C707058DE722858E
:106040002244B2400249A685924441011743000010
:106050006700C38417B50100130545EB9790010055
:10606000E780209CC1B7B2402244924402494101DA
:106070008280834755008345450017B5010013050D
:10608000E5E4A207DD8D179301006700A38117B532
:1060900001001305A5E217930100670083988D475F
:1060A00063FBB70A011126CA06CE22CC0344350091
:1060B00097E4FF1F83C4541597B501009385C5E588
:1060C000B337800017E7FF1FA300F71409C497B583
:1060D0000100938525E517B50100130525E5978097
:1060E0000100E780207C97E7FF1F83C7F7116386D5
:1060F000970097000000E780202B97E7FF1F83C7DA
:10610000B7108DC785472306F100B7E7040083A7C2
:1061100047177000854513055030829717B5010069
:106120001305C5E197900100E780A08F99679387D9
:1061300057EE2316F100680085479145A3078100BB
:106140002307F10097000000E78040E0F24062443E
:10615000D244056182808280894763F7B7080111C4
:1061600022CC06CE26CA8344250085472A84639D17
:10617000F404914763F5B7040345450083473400B1
:1061800022055D8D97D7FF1F239BA7229700000054
:10619000E780A04C9967938767EE2314F10083474B
:1061A000340023059100A305F10083474400954581
:1061B00028002306F10097000000E78020D9F24074
:1061C0006244D24405618280FDF89967938767EE47
:1061D0002314F10097D7FF1F83D7671EA305F10093
:1061E00023050100A183E1B782800111996722CCC8
:1061F000D51717F4FF1F130464412314F1008347DC
:10620000040026CA97F4FF1F9384A4502305F100CD
:1062100083D7040028009545A305F100A18306CE8D
:106220002306F10097000000E78040D203D6040067
:106230008345040017B501001305C5D197800100FF
:10624000E7804066F2406244D244056182809D67E7
:106250007971D9172316F10097F7FF1F83C7073B02
:1062600006D62307F100A9C3B7E70400FC4741465F
:1062700097E5FF1F9385C5E71305F1008297680036
:10628000CD4597000000E78060CC97F5FF1F83C5E0
:10629000E53717B501001305E5CE97800100E780CB
:1062A0006060B25045618280B7E70400BC47414658
:1062B00081451305F1008297D9B75DC1411106C62A
:1062C00022C4930750FA2300F5009307A005A3000A
:1062D000F50089472301F5009147A301F500F54733
:1062E000A302F50097F7FF1F9387473283C7070084
:1062F000230205002A842303F50097E7FF1F9387F5
:10630000B7F083C70700414697E5FF1F938545DE39
:10631000A303F50097F7FF1F83D7A73F2304F500DA
:10632000A183A304F50097D7FF1F83D7470923054F
:10633000F500A183A305F500B7E70400FC4731058C
:1063400082972285F14597000000E7802024230EE4
:10635000A4002181A30EA400B24022444101828006
:1063600082805D710A8586C6A2C497000000E7801E
:1063700000F537E404007C448A850810794682974A
:106380003C441305E10309468145829710109305AB
:106390000002014597D0FFFFE780E034B640264475
:1063A00061618280B7C7A55A01119387C7333EC484
:1063B00097E7FF1F83C757E53EC6B7F7070003C738
:1063C000070106CE22CCA5476313F70001A0116494
:1063D000930504F0930600100146254597C0FF1F62
:1063E000E780803E3000930504F0A146294597C020
:1063F000FF1FE780603D97E5FF1F83C5F5E017B5F8
:1064000001001305E5C897800100E780A049F2402C
:1064100062440561828001119165A1463000938537
:1064200005F02D4506CE97C0FF1FE780E0392247D3
:10643000B7C7A55A9387C7336314F702B24517B598
:106440000100130525B8B335B00097E7FF1FA38DF2
:10645000B7DA97800100E780E044F240056182806E
:10646000814517B50100130525B897E7FF1FA38DD8
:1064700007D897800100E780E04297000000E7809E
:10648000A0F2E1BFB7C7A55A79719387F7353EC629
:10649000B7E70400FC47AA8506D622D4414608087F
:1064A0008297B7F7070003C70701A5476313F700F3
:1064B00001A01164930504E89306001001462545E8
:1064C00097C0FF1FE78040307000930504E8D14675
:1064D000294597C0FF1FE780202F17B5010013053E
:1064E000E5BE97800100E780C053B2502254456159
:1064F000828079719165D1467000938505E82D45BC
:1065000006D697C0FF1FE780202C3247B7C7A55A91
:106510009387F73517B50100130505B56310F7022A
:10652000B7E70400FC4717E5FF1F130565BC4146AC
:106530000C08829717B50100130505B1978001007B
:10654000E780204EB25045618280B7F7070003C74D
:106550000701A5476313F70001A091654111930658
:1065600000100146938505E8254506C697C0FF1F24
:10657000E7808025B24017B501001305E5A241016F
:10658000178301006700E349C16769768146FD17FB
:1065900005061397060141836364B7003E85828038
:1065A0003307D50003470700B98F214713F81700B9
:1065B000858363050800B18FC207C1837D171377F8
:1065C000F70F6DF78506F1B741C5A547054763F29B
:1065D000B70883471500034705003168A207D98F24
:1065E00013978700A183D98FC207C1831308C855A9
:1065F000054763900707411106C622C426C203441B
:106600002500914763F087049307540063ECF5027B
:10661000A301C50021822302C5009304340091C662
:10662000A302D500A1822303D5002A84A685970062
:106630000000E780A0F526942300A4002181A30098
:10664000A4000147B240224492443A85410182802D
:1066500005473A858280B7C7A55A01119387E73469
:106660003EC42AC6B7F7070003C7070106CE22CCEF
:1066700026CAA5476313F70001A091642A84938575
:1066800004EE930600100146254597C0FF1FE780E2
:10669000A0133000A146938504EE294597C0FF1F43
:1066A000E7808012A28517B50100130565A09780C9
:1066B0000100E780201F97000000E780C0CAF24079
:1066C0006244D2440561828001119165A146300087
:1066D000938505EE2D4506CE97C0FF1FE780C00EBF
:1066E0002247B7C7A55A9387E7346318F702B24524
:1066F00017B501001305459197D7FF1F2391B7CC1C
:10670000C205C18197800100E780C0199700000091
:10671000E78060C5F24005618280D147D14517B559
:1067200001001305659017D7FF1F231AF7C897803C
:106730000100E780201717D5FF1F035545C89700B4
:106740000000E78080F1F9B721C1411126C206C6D9
:1067500022C4AE848DC52A8497000000E780A05D26
:1067600097E7FF1F83C747AA99CB22852244B240EF
:10677000A685924441011733000067002312B240FE
:106780002244924441018280828001114AC806CE8F
:1067900022CC26CA4EC693F715002E899DCBAD6735
:1067A000371700409387A7AA1CC3B7E70400BC4F64
:1067B00013060019854517D5FF1F034525C082978D
:1067C00013451900F2406244D2444249B24905617E
:1067D000828093F725006382071C17F7FF1F03577A
:1067E00027F3954763F9E70C014417F6FF1F1306DB
:1067F00026E293063005130550041308100493088D
:10680000B00413039005930764006374F7043A849B
:10681000FD5997F4FF1F83C4A4DF97F7FF1F83C7B9
:1068200037DFA204DD8CAD679387B7556383F4141B
:1068300063E3970AA9679387A7556386F414A28533
:1068400017F5FF1F1305C5DC97000000E78000F077
:10685000F5A8B307860083C50700639AD50483C5EE
:1068600017006396A50483C527006392050583C5B9
:106870003700639ED50283C54700639A150383C71B
:10688000570063966702A2890DE897F5FF1F83D52D
:1068900025E8B3853541C20517F5FF1F130545D718
:1068A000C1814E9597000000E78040EA65A8050485
:1068B0004204418089BF3A84FD598547E3EB87F460
:1068C00059CC854517F5FF1F130585D497000000A7
:1068D000E780C0E769A0B1679387C7556380F40478
:1068E000B5679387D755E39CF4F4A28517F5FF1F8E
:1068F000130505D297300000E78040FA8947630707
:10690000F4049305E4FFC205C18117F5FF1F1305C9
:1069100045D097000000E78000420DA897000000D6
:10692000E780C04011C9A28517F5FF1F130545CEAA
:1069300097000000E78020400546A28517F5FF1F5D
:10694000130505CD97F0FFFFE780E061A68517A549
:1069500001001305A57997800100E780A0F4FD5799
:10696000E395F9F297F7FF1F239407DA13452900FF
:1069700091BDA28517F5FF1F130585C997F0FFFF8D
:10698000E780606FE1B7A28517F5FF1F130545C8C3
:1069900097F0FFFFE780E06F55BF93F74500014593
:1069A000E38207E217A501001305857597800100B2
:1069B000E780200797300000E78040FD134549003D
:1069C00011B5411122C437E404005C5C06C63546AB
:1069D00097A501009385C52317B501001305C5E9E7
:1069E000829711E917A501001305457297800100F0
:1069F000E780200301A08327041C82972A84054591
:106A000097C00000E78060B697600100E780803B98
:106A100097600100E780801097B00000E780E0C732
:106A20002285B2402244410182801567B717004099
:106A30001307575598C3D8439D66558FD8C3D8437D
:106A4000FD76758FD8C3D8431367F70FD8C3356762
:106A50001307C7CC98C382804111054506C622C4DE
:106A600026C297C0FFFFE780804B1305A00497B0B4
:106A7000FF1FE780C063757585457D1597C0FFFFD3
:106A8000E78020357D7585451305F53697C0FFFFF6
:106A9000E780803E371400408327840A8D45130524
:106AA000002093E707202324F40A97C0FFFFE78024
:106AB0004032B7E4040097C0FFFFE7806077C85812
:106AC00097800100E780E0F517B501001305C5DAEE
:106AD00097800100E780E0F48327840C85454145D9
:106AE00093E707082324F40C97C0FFFFE780C03822
:106AF0008D451305000897C0FFFFE780E03797C07A
:106B0000FFFFE780C06437A507001305051297C093
:106B1000FFFFE7806060014597C0FFFFE780806668
:106B200095450545894717F7FF1F2305F7BE97C011
:106B3000FFFFE780C066B7E700E013070006238D7C
:106B4000E7403707000423A0E71097D0FFFFE78056
:106B5000E0F797D0FFFFE780A00B97000000E780E9
:106B600080E697000000E780408B97000000E780F8
:106B7000E0B597E0FFFFE78080E797000000E7803F
:106B8000C01C97000000E780600B83A7040817056E
:106B900000001305C5BF829797D7FF1F2380A782E8
:106BA000BC4C130600648545829797000000E7807F
:106BB00000E897C0FF1FE780A08301458280B7F7F8
:106BC000070003C70701A547AE866316F700939732
:106BD000450191C301A0AA850146254517C3FF1FA2
:106BE000670083BE4111B2862E86AA852D4506C652
:106BF00097C0FF1FE78040BDB24001454101828040
:106C00009307000463E8C7021D71A2CC2A84080818
:106C100086CE32C697800100E78060BDB24610087C
:106C2000A285294597C0FF1FE78000BAF640664459
:106C3000256182803955828041110D658D4506C6DA
:106C400097C0FFFFE780E018B71700408D6623A6C6
:106C5000D70A17F5FF1F130525AC1387C70A9387BB
:106C6000870A1CC15CC5856689675CC958C114C5A3
:106C700018C9B7E70400B24003A3871E410102838D
:106C80008145B307B5008387070089E71723000014
:106C9000670023A28505C205C181E5B7411126C25F
:106CA000E97797F4FF1F9384A4B722C49387A7556D
:106CB0002E842381B4002E86AA8517F5FF1F1305A5
:106CC00065B606C62390F400A381040097800100F6
:106CD000E780E0B193052400C205C18117F5FF1FCD
:106CE000130525B497000000E780408AB38784002D
:106CF0002382A7002181A382A70093056400224478
:106D0000B24026859244C205C1814101172300008B
:106D10006700239A09C99307800263E6B700170347
:106D200000006700E3F7828017F5FF1F034545A0C9
:106D3000828097F7FF1F83C767AE89E7172300009C
:106D400067002397828097F7FF1F83C747B099EFAB
:106D5000411106C697200000E780808DB24085472C
:106D600017F7FF1F2305F7AE410182808280630E73
:106D70000532638C05325D71CAC04EDE86C6A2C480
:106D8000A6C252DC56DA5AD85ED662D466D26AD02F
:106D9000B9472A89AE8963F9B706394697A5010034
:106DA0009385853D97800100E78000A231ED834700
:106DB000E900130710036394E702854717F7FF1FE5
:106DC000230EF7A417A501001305053C97F7FF1F35
:106DD000239507A497000000E780C0EA71A013077D
:106DE000000317A501001305253DE395E7FE97F77E
:106DF000FF1F238507A297F7FF1F239007A217A560
:106E000001001305E539F9B797F7FF1F83C707A1FD
:106E100063870722BD6AB96B938CFA55014A17FB49
:106E2000FF1F130B2B91138CEB65938AFA6605A851
:106E3000B307490183C6070097F7FF1F83D7E79D74
:106E4000B1E39307A005639BF600854717F7FF1F83
:106E50002315F79C97F7FF1F238ED78C050A9317EE
:106E60000A01C183E3E637FDB6402644964406494D
:106E7000F259625AD25A425BB25B225C925C025D6A
:106E800061618280054D639BA7039307500A639E4F
:106E9000F600894717F7FF1F2311F798930750FA59
:106EA00017F7FF1FA308F78855BF9307A005E387CF
:106EB000F6FA97F7FF1F239207964DB7138717002F
:106EC0004207DA9741832380D70017F6FF1F231666
:106ED000E6948D47E3F4E7F817F4FF1F0344B48505
:106EE00097F7FF1F83C7278522045D8C9307F4FF64
:106EF000C207C1839306F00DE3EDF6FA9307640031
:106F0000C207C183E31CF7F493052400C205C181C5
:106F100017F5FF1F1305258297F0FFFFE780006735
:106F200033078B008347570003474700A207D98FD9
:106F300017F7FF1F2313078E6318F50E8144630CA8
:106F4000A40197E4FF1F83C4247FA20497E7FF1FD7
:106F500083C7977EDD8C170500001305E5DB97F0EE
:106F6000FFFFE78000FE63878407636D9C029387C1
:106F7000EB556382F40497E7FF1F83C7E77B054760
:106F80006389E70681CB1387A7051377F70F8D4633
:106F900063F2E6081307F0072300E100A300F10005
:106FA00089459DA063829405E39754FD97F0FFFF08
:106FB000E780202A11A8A28517E5FF1F1305C577D2
:106FC00097F0FFFFE780E00D014597F0FFFFE780B6
:106FD00040F769B5A28517E5FF1F1305E57597F022
:106FE000FFFFE780A017CDB797F0FFFFE7802020D5
:106FF000E1BF930710F8130511002300F10097F08B
:10700000FFFFE780C02BFD450A8597000000E78061
:1070100020C95DBFA28517E5FF1F1305E57197F035
:10702000FFFFE780A0C84DB79307F00789450A85A1
:107030002310F10097000000E78080C605B5C14726
:1070400063FE3705414697A50100938525194A85BA
:1070500097700100E780407731E18347090113070A
:107060001003639CE700854717E7FF1F2302F76CB7
:1070700017A501001305C517B1BB1307000317A51A
:1070800001001305E519E397E7D497E7FF1F238174
:10709000076A17A50100130525172DBBCE854A8564
:1070A00097C0FFFFE7804012C1B38280411126C222
:1070B000AE848D4522C406C62A8497C0FFFFE780B0
:1070C000A0DBB717004099C803A5C70C418D23A6C4
:1070D000A70CB240224492444101828003A5870C50
:1070E000418D23A4A70CF5B783470500034715007E
:1070F000A207D98FC2076177C18713072720639A38
:10710000E7008345250037050400170300006700EA
:1071100023FA828017E6FF1F1306C6738147B286E3
:107120001303F00FA9483308F6000348080013F7CB
:10713000F70F6307A80C630668008507E39517FF40
:107140002947B387E6002380A70097E7FF1F9387AF
:1071500027715DA8411113D765001347170006C6B4
:1071600093F63500058B954791CA05469947638785
:10717000C60009469D476383C600A14713F6450034
:107180003336C00093F68503050685C2A145638B9F
:10719000B604E145638AB604930580026388B604A9
:1071A000930580036393B600914697F5FF1F238EE6
:1071B000F59097F5FF1F2389C59097F5FF1FA385CD
:1071C000D590BE8517A501001305850A97700100AB
:1071D000E780406DB240854717F7FF1FA307F78E82
:1071E000410182808546D1B78946C1B78D4675BFBA
:1071F00017A501001305450A177301006700836A8C
:1072000017E7FF1F1307C765BA972380B700E14749
:10721000E302F5F493077002E30CF5FC82802A8701
:1072200023800500814717E5FF1F1305A56213089A
:10723000F00F2946B306F50083C606006396E60202
:1072400097E6FF1F9386C661B69783C7070005457B
:107250002380F5009947636EF7029D4763FDE700C1
:10726000E147630DF7008280638506018507E3939C
:10727000C7FC0145C5B7238005008280B7370040B1
:1072800003C7370083C7050093F70704D98F23800E
:10729000F5008280797126D24AD097F4FF1F83C40B
:1072A000A49417F9FF1F1309699306D622D44ECE72
:1072B00052CC56CA5AC8B307990083C7070093F740
:1072C000F70FA5C79387140093F7F70F0D47636176
:1072D000F70C17F7FF1F2309F79097F7FF1F938706
:1072E0006790A69783C707001307100293F7F70369
:1072F0006389E7226363F70A054463808720E3829A
:10730000076809476389E71413070002E387E75218
:10731000B7E700E03707400023A0E71801000100AD
:10732000CA942380040023A0E710B787004003C756
:107330006700058BE308077297F6FF1F83C6E68A8E
:107340000547E393E67029472381E7020947238332
:10735000E7022385E70297E7FF1FA389077697F7E0
:10736000FF1FA3840788B7870040A381070017E7A2
:10737000FF1FA30F077405472383E700B250225471
:1073800092540259F249624AD24A424B4561828084
:1073900097F7FF1F238A078489B713073002638694
:1073A000E70A63E6E71413074002638AE708130756
:1073B0000003E39FE7F497F7FF1F93876782A69781
:1073C00003C70700A1471377F70FE313F71617EA70
:1073D000FF1F130AAA4983476A0097E6FF1F238D00
:1073E000F66C97E7FF1F83C7D74891C7FD5797E60D
:1073F000FF1F2383F66C97E5FF1F83C5354797E78B
:10740000FF1FA38BB76A97E7FF1F83C7274693F930
:1074100007089306000493F70706639DD74A93076E
:10742000A0096387F51463E4B7109307F00563843C
:10743000F548930750096382F52801440DABFD57C9
:1074400017E7FF1F2309F766E1B5FD5717E7FF1F91
:107450002302F76675BD17A50100130565F5977042
:107460000100E780005C97E7FF1F93876777A69787
:1074700003C40700814917EAFF1F130AAA571374B0
:10748000F40F97AA0100938A2AF363C78904294558
:1074900097700100E780E045854717E7FF1FA309C4
:1074A000F75417E7FF1F2306875417E7FF1F230F23
:1074B000F76037E700E0B70640002320D718010047
:1074C0000100378600408347A60293F7370F230554
:1074D000F6022320D7102DBDB3073A0183C507005C
:1074E0005685850997700100E780C03B79BF8547C5
:1074F00017E7FF1F230EF74E21BD17E7FF1F1307E6
:10750000276E26970347070097E6FF1FA380F642E2
:1075100097E6FF1F238DE64017E7FF1F2308F75A62
:10752000C5BB854717E7FF1F2302F740D5B3930775
:10753000400A638DF5349307200B6388F536930773
:10754000100AE39CF5EE83072A00014463D1074249
:1075500097E7FF1F83C7B73193F63700638E061A8C
:107560000546638EC62209466399C61A1D4775A251
:1075700017E5FF1F0345A52FC94717EAFF1F034A59
:107580001A2F97E5FF1F83C5A52E17E4FF1F03449D
:10759000342E6319F510CD476316FA10930770085F
:1075A000639CF5021307300FB7170E006308E40061
:1075B0001307900DB7B704006314E40817E7FF1F23
:1075C0002322F750BE8517A50100130565DF9770CC
:1075D0000100E780202D95B593078008639DF50095
:1075E00033048040B77746001374F40F938787CD38
:1075F000B3D78702E1B793079008639AF500330485
:10760000804091671374F40F9387C766D5B79307CB
:10761000A008639BF50033048040B7173D00137446
:10762000F40F93870790E9B79307B008639AF500C2
:107630003304804091671374F40F938797D04DBF44
:1076400093F5F5078D47639BF50033048040B797AA
:107650005B001374F40F938707D859BF8947639B66
:10766000F50033048040B7770B001374F40F938751
:10767000071BBDBF8547639AF50033048040DD6773
:107680001374F40F938767E3A5B789E93304804047
:107690008D671374F40F938777DC99BFF167938735
:1076A000072029BF97000000E78000A7A285528528
:1076B00097000000E78040A649B39305610017E5F5
:1076C000FF1F0345C51A17E4FF1F0344541A970010
:1076D0000000E78000B59305710022859700000047
:1076E000E78020B43C0017E7FF1F2327F74E8347AE
:1076F00061002304F10083477100A304F10089476E
:1077000017E7FF1F230AF73A8357810017E7FF1F88
:10771000231EF7140944A1AC154793F64700B3366E
:10772000D00093F78703850685C32146638BC70680
:107730006146638AC706130680026388C70613067C
:1077400080036393C700914717E6FF1F230ED636C9
:1077500097E6FF1FA38AF63697E7FF1F2387E736D2
:1077600017E7FF1F0347C7109376070497E7FF1F2C
:1077700083C717108DEE1377770C93067008630C90
:10778000D7021377F7078D46631ED70AB307F04079
:10779000B7955B0093F7F70F938505D881A8194734
:1077A000ADBF854755B7894745B78D4771BF93062C
:1077B00070086311D7021307300FB7150E006389E5
:1077C000E7021307900DB7B504006383E7021307C0
:1077D000700845BF9306800C6311D702B307F040D1
:1077E000B775460093F7F70F938585CDB3D5F502AE
:1077F00097E7FF1F23A8B72CF9B39306900C631AE1
:10780000D700B307F040916593F7F70F9385C566EE
:10781000F1BF9306A00C631BD700B307F040B71568
:107820003D0093F7F70F93850590C9B79306B00C09
:10783000E319D7F4B307F040916593F7F70F9385F9
:1078400095D06DB78946631BD700B307F040B77575
:107850000B0093F7F70F9385051B49BF8546631A05
:10786000D700B307F040DD6593F7F70F938565E325
:10787000B5BF09EBB307F0408D6593F7F70F93851C
:1078800075DCADB7F165938505209DB783472A0068
:10789000C18B99C7854717E7FF1F2302F72271BEE7
:1078A00097E7FF1F238D072049BE854717E7FF1F76
:1078B000A30DF72059B63C0017E7FF1F232EF73022
:1078C0000947930700032314F10097E6FF1F238560
:1078D000E61E2DBD63990758A94763EBB74417A768
:1078E0000100130727968A05BA959C41BA978287AB
:1078F00017E4FF1F0344B4F7094A630C440F636C99
:107900008A0885476309F40A9307F00F17E7FF1FFA
:107910000347871A63F6E70017E7FF1F230EF718E0
:1079200017EAFF1F034A4A19930700041374FA0F5A
:1079300063F447011304000497E7FF1F9387C729E7
:1079400083AA0700228617E5FF1F130525F2D685B7
:10795000330A8A40A29A97700100E78040E997E7CE
:10796000FF1F238B471597E7FF1F23A7572797E78D
:10797000FF1F83C7771415476399E762B7E700E0F5
:107980003707400023A0E71801000100B786004038
:107990002380860285A58D47630CF40A9947E31579
:1079A000F4F697A701009387679017E7FF1F232539
:1079B000F722A947A1BF17E7FF1F0347072397E750
:1079C000FF1F93876711494697A501009385059787
:1079D0006306870097A50100938545923E859770C1
:1079E0000100E780C0E017E7FF1F2327A71EC94754
:1079F00031BF97E6FF1F83C6461F054797E7FF1F66
:107A00009387870D6394E6023E851306700297A55F
:107A100001009385259097700100E78040DD17E70E
:107A2000FF1F232BA71A93077002CDB53E851306BF
:107A3000300497A501009385258897700100E780A1
:107A400000DB17E7FF1F2329A718930730047DBD2C
:107A500097E5FF1F83C5A5E117A5010013058597CD
:107A600097700100E78000E4854A17EBFF1F034B86
:107A7000CB1797E5FF1F83C585DF17A50100130509
:107A8000659563185B0B97700100E780A0E197E7AD
:107A9000FF1F83C7C7DDB5CBE368F4E617A4010079
:107AA0001304048E638C670117A401001304C48DB2
:107AB0006386470117A401001304848E2285977002
:107AC0000100E780C0FE1375F50F930715008607C8
:107AD00017E7FF1F2302F7008D4717E7FF1FA30DCE
:107AE000F7FE97E7FF1F938727FF0147BE861376B0
:107AF000F70F89076365A60297E7FF1F23AED70C30
:107B000097E7FF1F83C747FD11B597A7010093872C
:107B1000278017E7FF1F2321F70C9147C5BB3306CA
:107B2000E40003460600A380070005072380C70082
:107B30007DBF97700100E780E0D697E7FF1F83C7FE
:107B400007D3E1D7E362F4DC17A4010013044480F7
:107B5000638C570117A40100130404806386470156
:107B600017A401001304C480228597700100E780E8
:107B700000F41375F50F93071500860717E7FF1F2D
:107B8000230CF7F48D4717E7FF1FA307F7F497E7D8
:107B9000FF1F938767F40147BE861376F70F8907A7
:107BA000E37CA6F43306E40003460600A380070046
:107BB00005072380C700D5B797E5FF1F83C525CBF1
:107BC00017A501001305C58197700100E78080CDDE
:107BD00097E7FF1F83C717F093E7470017E7FF1FDB
:107BE000A30AF7EE83472A0017E7FF1FA302F7EE69
:107BF000A9B0179501001305E57F97700100E78094
:107C000040E297E7FF1F9387A7EC83C7070017E7BA
:107C1000FF1F230DF7C417E4FF1F0344E4E93334C7
:107C20008000B1B3179501001305057E9770010020
:107C3000E78020DF97E7FF1F83C7D7E993E70701B6
:107C400017E7FF1FA308F7E883472A0017E7FF1F7E
:107C50002300F7E86FF06FFE179501001305057C10
:107C600097700100E780E0DB03470A007D8B51EF4E
:107C7000B787004003C767021377C70B1367270056
:107C80002383E70203C7A7021377C70B13672700F5
:107C90002385E70203C7E7021377C70B13672700A3
:107CA0002387E70203C727031377C70B1367270050
:107CB0002389E702854717E7FF1F2309F7C617E760
:107CC000FF1F2307F7D217E7FF1F2305F7DE17E78C
:107CD000FF1F2302F7DE97E7FF1FA38907C497E77B
:107CE000FF1FA38707D097E7FF1FA38507DC97E750
:107CF000FF1FA38207DC97E7FF1FA38907DC97E735
:107D0000FF1FA38407EE6FF04FF389476312F7025A
:107D100097E7FF1F83C7C7B59146638CD70863E019
:107D2000F604638EE70C6369F70A05476380E70E84
:107D3000FD5717E7FF1FA301F7D837074000B7E744
:107D400000E023A0E71801000100B78600401306F9
:107D5000F0FC2381C60223A0E7106FF06FDB13074E
:107D600020086382E7086362F70213071008E391B3
:107D7000E7FC378700408347670293F7C70B93E719
:107D800027002303F7026FF04FEB130730086389D6
:107D9000E70213074008E39DE7F837870040834771
:107DA000270393F7C70B93E727002309F7026FF028
:107DB000CFE8378700408347270393F73707F5B7A6
:107DC000378700408347E70293F7C70B93E7270005
:107DD0002307F7026FF06FE6378700408347E7021B
:107DE00093F73707F5B7378700408347A70293F724
:107DF000C70B93E727002305F7026FF00FE43787DF
:107E000000408347A70293F73707F5B7378700404D
:107E10008347670293F73707ADB71795010013053E
:107E2000E56097700100E780C0BF97E7FF1F238FD1
:107E300007A2D5B31795010013054560977001009F
:107E4000E78020BE97E7FF1F239207A297E7FF1F57
:107E5000938787C603C40700894763F387000944F3
:107E60001374F40F29B613070002E393E7EC639948
:107E7000090A638FF500930720026381F5081795BF
:107E800001001305255F97700100E780A0A14DB5A3
:107E9000179501001305455B97700100E78060B8F6
:107EA0000144179B0100130B6B5BA14AB3078A00C7
:107EB00083C507005A85050497700100E780809EFE
:107EC000E31654FF17950100130505B297700100E2
:107ED000E78020B517E4FF1F0344849911E497E776
:107EE000FF1F2387079661B48947E313F4E48547AE
:107EF00017E7FF1F230EF7946FF02FD417E6FF1F2D
:107F00000346F69697E5FF1F83C565961795010012
:107F10001305455597700100E780C0986FF0EFD1C9
:107F2000638FF50493071002E39BF5F497E5FF1FB9
:107F300083C50594179501001305C554977001007A
:107F4000E780409697E7FF1F23A847C997E7FF1FE1
:107F5000938747B7944383D7470017E7FF1F03472B
:107F6000C7B617E6FF1F2323D6901D4497E6FF1FD1
:107F70002390F69097E7FF1F238DE78ECDBA97E504
:107F8000FF1F83C5E58E17950100130525519770D6
:107F90000100E780209197E7FF1F238B078A97E76F
:107FA000FF1F2395078C6FF0EFF62547E388E79CCA
:107FB00019476391E702B786004023808602B7E73E
:107FC00000E03707400023A0E71801000100130676
:107FD00000FC41B31307100A6391E702B786004023
:107FE00023808602B7E700E03707400023A0E718A8
:107FF00001000100130680FCA9BB1307A009E38F51
:10800000E7FC1307400AE38BE7FC13072002E38732
:10801000E7960547E384E796B7E700E037074000B7
:1080200023A0E718E392099601000100B7860040FB
:1080300023808602130620FC29BB17E7FF1F034796
:10804000B7A76308F71E63E7E7029547630EF70ECD
:1080500099476308F704B786004023800602B7E714
:1080600000E03707400023A0E718010001001306D5
:10807000A0FCC5B19307F005630AF7009307500908
:108080006306F70093071002E317F7FCB7E700E079
:108090003707400023A0E71801000100B786004021
:1080A00051BF97E9FF1F83C929A193070004CE8A16
:1080B00063F43701930A000497E7FF1F9387C7B162
:1080C00003AA070013F4FA0F2286D28517D5FF1FE3
:1080D0001305C57997600100E7806071B387894017
:1080E000529417E7FF1F2309F79C97E7FF1F23A56B
:1080F00087AE638E0902B787004023805703B7E637
:1081000000E03706400023A0C6180100010003C7A5
:108110002702134707042381E70203C727021377C7
:10812000C70F2381E70223A0C6106FF06F9EB786AA
:10813000004023800602B7E700E03707400023A095
:10814000E71801000100FDB537870040834737007D
:1081500097E6FF1F83C6D69793F70708D58FA3012D
:10816000F700B7064000B7E700E023A0D7180100EA
:1081700001001306A0FC2301C70223A0D7106FF053
:108180002F9997E7FF1F9387A7A5A69783C7070097
:1081900093F7F70FD9CF97E7FF1F83C707A5D1EB59
:1081A00017E7FF1F03475791930700026313F70870
:1081B00097D7FF1F9387876B03AB070097DAFF1FE3
:1081C00083CA0A6B17DAFF1F034A9A6A97D9FF1FFF
:1081D00083C9296AD2875687CE865A8697D5FF1FCC
:1081E00083C50567179501001305C52C976001002D
:1081F000E780406B97E7FF1F23A6678D97E7FF1F78
:108200002384578D97E7FF1FA380478D97E7FF1FB4
:10821000238D378B97D7FF1FA38B8762B7E700E0CB
:108220003707400023A0E71801000100B78600408F
:10823000D1B3B7E700E03707400023A0E7180100FB
:108240000100B786004025B529472381E702094789
:108250002383E7022385E7022387E7022389E702D6
:108260006FF06F8F03C76700118B6309079083C797
:108270005700918BB5CF17E7FF1F03470797854737
:108280006313F70697E7FF1FA381E78497D7FF1FC4
:10829000238E076897D7FF1F238C077497E7FF1F6C
:1082A000238A078097E7FF1F2387078097D7FF1F41
:1082B000A38E076697D7FF1FA38C077297D7FF1F60
:1082C000A38A077E97D7FF1FA387077E97D7FF1F35
:1082D000A38E077E97E7FF1FA3890790B78700400B
:1082E00011476FF06F8917D7FF1FA302F75679BFA9
:1082F000854717D7FF1F230BF76217D7FF1F2309E7
:10830000F76E17D7FF1F2307F77A17D7FF1F23042E
:10831000F77A69BF854717D7FF1F2309F76017D77B
:10832000FF1F2307F76C17D7FF1F2305F77817D711
:10833000FF1F2302F77817D7FF1FA309075E17D780
:10834000FF1FA307076A17D7FF1FA305077697D755
:10835000FF1FA38207768280411106C697000000A6
:10836000E78080FBB787004023800700130740FCAD
:108370002386E7001307C004A386E70017D7FF1F73
:108380001307C74E2398E70017D7FF1F130707529D
:10839000239AE70017D7FF1F1307875D239CE70089
:1083A00017D7FF1F13070769239EE700294723817B
:1083B000E70209472383E7022385E7022387E702D1
:1083C0002389E702A3810700930600F8A380D70062
:1083D000930690022380D700FD562383D700238184
:1083E000E700B706400037E700E02320D71003C7B7
:1083F000170013671700A380E700B24097D7FF1F4D
:108400002398076C41018280411106C69700000045
:10841000E78080F0B787004023800700130700FC47
:108420002386E7003147A386E70017D7FF1F13070E
:10843000E7432398E70017D7FF1F13072747239A1F
:10844000E70017D7FF1F1307A752239CE700294710
:108450002381E70209472383E7022385E702A381FB
:108460000700930600F8A380D700930690022380AC
:10847000D700FD562383D7002381E700B7064000CD
:1084800037E700E02320D71003C717001367170052
:10849000A380E700B24097D7FF1F239B07624101EB
:1084A0008280F1679387072017D7FF1F232CF7607F
:1084B000854717D7FF1F2319F760A14717D7FF1F5D
:1084C0002305F76097D7FF1FA381076097D7FF1F8A
:1084D000238E075E97D7FF1F238C073697D7FF1F82
:1084E000A3870736814717D5FF1F1305A536FD550E
:1084F00017D6FF1F1306C6362947B306F50023809B
:10850000B600B306F600238006008507E397E7FE72
:1085100097D7FF1F2384076C97D7FF1FA380076C93
:1085200097D7FF1F238D076A97D7FF1FA387075889
:1085300097D7FF1FA385075897D7FF1F238007589A
:1085400097D7FF1F238B075697D7FF1F238A0756FE
:1085500097D7FF1FA384075697D7FF1F238107567E
:1085600097D7FF1FA38D0766828017D7FF1F03478A
:10857000C76785476316F70017030000670003E924
:1085800017030000670083DD411122C406C617D718
:10859000FF1F0347876585472E8613F4F50FAA85CD
:1085A0006317F70417D5FF1F130585409760010077
:1085B000E780E02397D7FF1F238C0742B78700404F
:1085C00023848702B7E600E03706400023A0C618E0
:1085D0000100010003C7A7021377C70F2385E70235
:1085E000B240224423A0C61001454101828017D524
:1085F000FF1F1305A52F97600100E780401F97D745
:10860000FF1F23850732B787004023828702B7E622
:1086100000E03706400023A0C6180100010003C790
:1086200067021377C70F2383E7025DBF411106C6B8
:1086300097000000E78020E7B240410117030000E7
:108640006700E3F2411106C697F0FFFFE780C0C460
:1086500097D7FF1F83C7972DA1CB97D5FF1F83C542
:10866000052D89C917D5FF1F1305852C97E0FFFF3E
:10867000E780207097D7FF1FA38A072A97D7FF1F8D
:108680002386074437E700E0B70640002320D718C9
:1086900001000100378600408347660293F7370FD9
:1086A0002303F6022320D710B2404101828041C942
:1086B000D9C597D7FF1F83C7A741D1C3011122CCCA
:1086C0004AC84EC656C25AC006CE26CA52C42E89C1
:1086D000AA890144930A0004371B0300637724032B
:1086E000B3078940C207C183BE8463F4FA009304D0
:1086F0000004C204C180130A1BD497D7FF1F83C78D
:10870000E7229DE37D1A631C0A00F2406244D244D2
:108710004249B249224A924A024B0561828097F04F
:10872000FFFFE78060B7D1BF338589002694A68517
:10873000420497000000E78060E5418045B78280F1
:1087400097D7FF1F9387074E18429C4383D6450057
:108750000345070083C5C700035646006396A5007E
:1087600083D5E700638DD502011106CE2386A700CD
:108770002397D700B705CF00DC4B9385757D0507A0
:108780007D162EC2230001003AC42316C100231710
:10879000D10099C30A858297F24005618280828068
:1087A000DC4DDC4B81CFB7E70400904503A3870580
:1087B000914517D5FF1F03452547028382806D71C0
:1087C0003C083EC6B707E500232291103EC8AA84A4
:1087D0003C083285232611103ECA23248110232011
:1087E00021112E8997300000E78020562A84979522
:1087F00001009385A5CF17850100130525B8976063
:108800000100E780200AA28517950100130585DE87
:1088100097600100E7800009294597600100E78023
:10882000400DB705CB009385757D6800971000005B
:10883000E780405FA285680097300000E7804043F2
:10884000014781467000CA85268597200000E78091
:10885000C08205CD2A8497950100938525C9178587
:1088600001001305A5B197600100E780A003A28570
:10887000179501001305C5D897600100E7808002B5
:10888000294597600100E780C0068320C1100324BA
:10889000811083244110032901105161828097D7F0
:1088A000FF1F9387273818429C43797122D406D63C
:1088B0000348070083C807012A8483D6450003556F
:1088C00046006396080183D82701638DD802238868
:1088D000070105072399D7003708CC00DC4B1308A4
:1088E000787D3ACC1307F5FF42CA23080100231E06
:1088F000E100231FD10099C7080832C62EC4829711
:108900003246A245228597000000E78080EBB250F6
:108910002254456182806D713C083EC0B707E50076
:108920003EC23C083EC4232611102324811023227A
:108930009110231701002318010023190100231AA5
:108940000100231B010097B7FF1F83D7A7A999E355
:10895000C167FD172316F10097B7FF1F83D7A7A89C
:1089600091EB97D7FF1F9387E72B9C439C43DC47F2
:1089700083D7070017B4FF1F1304C4A6584C23174E
:10898000F10083574400484B2318F10031E19795DB
:1089900001009385A5BC178501001305259E9760EE
:1089A0000100E78020F017950100130565BC976072
:1089B0000100E78020EF294597600100E78060F320
:1089C0008320C110032481108324411051618280CF
:1089D00097B7FF1F83C777A189EBB7E70400BC57A0
:1089E00082975C4C23AA0700E1BFFD1797B6FF1FD3
:1089F000A38DF69E03560701834704014C470A8561
:108A0000230BF10097300000E780A02397D7FF1FCA
:108A1000938747219C430147814688430A866C001F
:108A200097100000E7806065AA8429C1979501002E
:108A30009385C5B217850100130545949760010021
:108A4000E78040E6A68517950100130525B39760DA
:108A50000100E78020E5294597600100E78060E993
:108A6000584CB7E70400BC57484B9DBF97B7FF1F52
:108A700083C7B797F5D7B7E70400BC4F10448545C7
:108A800017D5FF1F0345451A82971DBF5C4EDC4B6F
:108A9000B9CFB1CD411122C4178501001305058E50
:108AA0002E84979501009385A5A906C697600100BD
:108AB000E78040DFA285179501001305E5AE9760BA
:108AC0000100E78020DE294597600100E78060E231
:108AD000B7E704002244B24003A3870517D5FF1F60
:108AE00003458514130640069145410102838280A7
:108AF000411122C417B4FF1F1304848C1C4C06C6FA
:108B000089C7DC4399C34C488297584CB7E70400A7
:108B1000BC57484B82975C4CB240224423AA0700C2
:108B20004101828017B7FF1F1307878B8347070018
:108B30009306F00B850793F7F70F63E9F60097B6F6
:108B4000FF1F238FF688034507008280930700F8F4
:108B5000FDB7835745006386071001114AC817B94E
:108B6000FF1F1309298852C4032AC90106CE22CC4B
:108B700003274A0126CA4EC656C2F15735E31307EA
:108B8000D00DFD57636EC704B7E9040083A709073A
:108B90002A841305860042054181B284AE8A8297F9
:108BA000232AAA000325C9015C49A9E7979501007A
:108BB00093850597177501001305457C97600100A3
:108BC000E78040CE17950100130545A69760010088
:108BD000E78040CD294597600100E78080D1DD57CF
:108BE000F2406244D2444249B249224A924A3E8506
:108BF0000561828093874400B705CF002319F500F3
:108C00009385757D310597100000E780A02103252D
:108C1000C90183456400310597300000E7804005B5
:108C20000325C9012686D685310597300000E780E7
:108C300040017146A2854A8597600100E78020BB0C
:108C4000504419CA83A78905854517D5FF1F0345D9
:108C5000A5FD8297814769B797000000E780E0CBC8
:108C6000D5BFFD573E858280411126C297A4FF1FC4
:108C700093844477D84C22C437E404003C54484BD6
:108C800006C68297DC4C0323C4052244B2409244BA
:108C900023AA070017D5FF1F034505F985454101A4
:108CA0000283411126C297D4FF1F9384A4F79C40EE
:108CB00006C622C44AC0D5C3DC43C5C35CC1230079
:108CC000B5002A84979501009385C580177501002A
:108CD0001305C56A97600100E780C0BC294597600D
:108CE0000100E78000C19C4023A4070023A20700E5
:108CF00097A7FF1F9387C76CDC4FDC4B91C72955A3
:108D000097000000E78000DF97A7FF1F9387876D1C
:108D1000DC4FDC4B89C797000000E78020F537E97E
:108D200004008327C905894517D5FF1F0345C5EFF3
:108D300082978327C905914517D5FF1F0345C5EEC7
:108D400082979C4003A347016309030022852244C4
:108D5000B2409244024941010283B240224492440B
:108D60000249410182800111328506CE22CC26CAF9
:108D70002E8497300000E78040FDAA84978501008B
:108D800093858578177501001305455F976001008D
:108D9000E78040B103078400035664008355440014
:108DA000A686179501001305258297600100E780CC
:108DB00060AF294597600100E780A0B397A7FF1F28
:108DC00083C76760639D9700014597000000E780B7
:108DD00060D281450A8597000000E780C0ECF24030
:108DE0006244D244056182806D7123248110232660
:108DF00011102322911093F745002E8463870714E6
:108E00003C083EC0B707E5003EC23C083EC42317FD
:108E100001002318010023190100231A0100231B5C
:108E2000010097A7FF1F83D7A75999E3C167FD17D3
:108E30002316F10097A7FF1F83D7A75891EB97D769
:108E4000FF1F938727DE9C439C43DC4783D70700A3
:108E500017A7FF1F1307C7562317F100544F835757
:108E600047002318F100DC4AA1E7978501009385AC
:108E7000E56D177501001305655097600100E780E7
:108E800060A2178501001305A56E97600100E780B9
:108E900060A1294597600100E780A0A51345440023
:108EA0008320C110032481108324411051618280EA
:108EB00097A7FF1F83C737512555D9C3FD1717A69D
:108EC000FF1FA302F65003D6060183470701CC46D5
:108ED0000A85230BF10097300000E78080D697D7F2
:108EE000FF1F938727D49C4317A7FF1F1307474DE6
:108EF000978601009386C66A88430A866C0097109D
:108F00000000E7808017AA8451D9978501009385D6
:108F1000E563177501001305654697600100E7805A
:108F20006098A685178501001305456597600100C7
:108F3000E7804097294597600100E780809B268560
:108F400097000000E78000BB91BF93F725009DC705
:108F5000B7E70400BC47414681452808829725555C
:108F600097000000E78000B928089305F00F9700EC
:108F70000000E78040D3134524001DB793F7150088
:108F8000014599DF97000000E78020991345140000
:108F900001BF5C4D411106C688C317D7FF1F2323AD
:108FA000F7C8B7E7040083A70708170500001305F3
:108FB000E5E38297B24097D7FF1F2387A7C60145F5
:108FC0004101828001113335A000A307A100B7E75A
:108FD000040083A7471706CE1306F1008545130545
:108FE00050308297F240056182808280411122C414
:108FF00006C697D7FF1F83C7A7C4014489EF97B759
:10900000FF1F83C77720054499E717C4FF1F034458
:10901000E45F13441400228597000000E780C0FA43
:10902000178501001305456C09E417850100130538
:10903000A56C2244B240410117630100670083869A
:10904000797122D4A30F010037E404008327841729
:1090500026D24AD006D6AA842E891305503093050D
:10906000F10132C6829732468347F101931506011A
:10907000C18185CB01452EC697000000E780C0F472
:1090800083274417B2454A8626858297054597006F
:109090000000E78060F3B2502254925402594561B7
:1090A0008280832744174A8626858297EDB741112F
:1090B0009397050122C406C626C2C1872E8463D4B5
:1090C0000702B7E40400FC5417A5FF1F03458534CD
:1090D000829719C1BC5482972165218DB2402244E8
:1090E00092444101828093F715008DC7B7E70400D1
:1090F00083A7471A17A6FF1F1306C63097D5FF1F71
:10910000938545B317A5FF1F0345C53082971345C7
:109110001400E9B793F7250099CFB7E70400BC4FD7
:1091200013060064894517A5FF1F0345A52E8297E6
:109130001345240065B793F785009DC7B7E7040082
:1091400003A8871A1307401F97A7FF1F83C7872C01
:10915000814613064006994517D5FF1F035585AE76
:109160000298134584009DBF93F745000145BDD784
:10917000B7E4040083A7041817D5FF1F035585AC77
:109180008297BC4C13060064914517A5FF1F034549
:10919000652882971345440091B797D7FF1F83D75F
:1091A00067AA6398A70217D7FF1F231EB7A817D770
:1091B000FF1F231BC7A817D7FF1F2318D7A82E866A
:1091C0001785010013058558BE85175301006700F8
:1091D000636D178501001305E558176301006700EB
:1091E00043840357450097D7FF1F83D7A7A5631A6A
:1091F000F704C1674111F91722C417D7FF1F2323B2
:10920000F7A437E4040097D7FF1F23AF07A297D72F
:10921000FF1FA38707A27C4C06C6894517A5FF1F21
:109220000345451F82977C4C914517A5FF1F0345B9
:10923000651E82972244B240410117030000670077
:1092400023DB178501001305E55117530100670063
:10925000437D7D15954763E2A71C1787010013071F
:1092600067460A053A951C41011122CC06CEBA97F1
:109270002E848287178501001305454F9750010002
:10928000E780207AA1A203C7250099476311F7025E
:109290002E8597000000E78000F583456400178560
:1092A00001001305A54D97500100E780A05F97B717
:1092B000FF1F238B07F4178501001305E54D7DBFC4
:1092C00003C7250095476319F702C16717D7FF1F2A
:1092D00003574797F91703D5A5006309F702B7E7C6
:1092E000040083A7C7178297178501001305C54B94
:1092F00097500100E780E072854717B7FF1F2305ED
:10930000F7F0178501001305A54C8DBF97D7FF1FF8
:10931000239AA79283D7E50097D6FF1F2395F6924D
:1093200083D7050197D6FF1F2390F69283D7250197
:1093300097D6FF1F239BF69097D7FF1FA382079016
:10934000631BE502B7E70400BC4F096613060690ED
:10935000A14517A5FF1F0345E50B82970356E400BF
:109360008355A4001785010013054545975001005A
:10937000E780405351B79307700F2316F100B7E70A
:10938000040083A7870D17A6FF1F0346A6086C00DD
:1093900082974DF9854717D7FF1FA303F78A5DB75B
:1093A0001785010013058543D1BD83C5250091476D
:1093B0006392F502178501001305C543975001001C
:1093C000E780206697000000E78080C2F240624498
:1093D0000561828099476392F5022285970000001B
:1093E000E78060E0834564001785010013050539B7
:1093F00097500100E780004BD1BF9547639AF50075
:1094000083471400E1F3178501001305E540BDB55E
:10941000178501001305C540E1BF82806D712324CB
:1094200081102326111023229110328401CD894707
:10943000630AF5028320C1100324811083244110A4
:1094400051618280178501001305453EAE84975017
:109450000100E780005DA285268597C0FFFFE780B9
:10946000C011C9BFB7E70400FC47280082971785E1
:1094700001001305653C97500100E780805A83473F
:10948000810039C41307000B6380E7021387A70527
:109490001377F70F8D4663EDE602A285280097D07B
:1094A000FFFFE780A08079B78547E3F587F883451C
:1094B0009100177501001305A521B335B00097B7CA
:1094C000FF1F2383B7BC97500100E780A03D9DB7E5
:1094D00003479100A207D98F35671307D7556385D6
:1094E000E7086368F7022D671307B7556387E70638
:1094F00031671307C755638AE70429671307A75520
:109500006394E702A285280097D0FFFFE78060B848
:1095100015B739679306E765638DD70663E9F600EB
:109520001307E7556380E706A28528003DB73D672E
:109530009306F7556386D7061307F766E396E7FEAB
:1095400097D0FFFFE780E0D0F5B50146A28528005F
:1095500097D0FFFFE78020A1F1BDA285280097D01A
:10956000FFFFE78040B1F9B58947E3F587EC930544
:10957000E4FFC205C1811305A10097A0FFFFE780AA
:10958000A0C44DBDA285280097D0FFFFE78060B141
:1095900055B5A285280097D0FFFFE78020BC59BDB4
:1095A00097D0FFFFE780A0C471B5411122C417A472
:1095B000FF1F130464E7AA8617860100130606122C
:1095C0002285C14506C697500100E780C046035773
:1095D000440097A7FF1F938727E62393E7000357CD
:1095E00064002394E700B24022444101828041118B
:1095F00006C697000000E78080FBB7E7040083A75A
:10960000871417A6FF1F130626E2D545014582974A
:10961000B2404D4697A5FF1F938505E213057030B4
:109620004101170300006700E3A161712324811A3F
:1096300037E40400832704082326111A2322911AF1
:109640002320211B232E311917050000130565A6C1
:10965000829717A9FF1F1309E9DB99478544230067
:10966000A900231CF100978501009385250B930722
:10967000400617750100130565D0231CF108230867
:10968000910097C9FF1F9389C90897500100E7808F
:10969000602183D509001785010013052507975020
:1096A0000100E7802020294597500100E7806024D1
:1096B00003D50900896997000000E78040EF832700
:1096C00044171008854513055030829783274417A7
:1096D00017A6FF1F130646D6CD4513057030829797
:1096E0008327441717A6FF1F130606D3B545130596
:1096F000603082978327441730088945130510315D
:1097000082978327441730098945130520318297B2
:1097100083274415938509900D4582978327441527
:109720009385099011458297A30591002306910026
:109730002308910002CD230C0100832784163009F1
:109740009145130570408297832784161306B10054
:109750008545130500408297832784167000854550
:10976000130510408297832784163008854513051A
:1097700020408297832784161008854513055040A2
:109780008297832704157D558297832744137D553F
:1097900082977D5597A0FFFFE780C0ED8327440C9B
:1097A000829797A0FFFFE78000C98327841417A63C
:1097B000FF1F130666C7D5450145829789471306E3
:1097C000700F814528092306F1009790FFFFE7807D
:1097D00080928D471306000881452808230CF10864
:1097E0009790FFFFE78020919147230CF100977736
:1097F0000100938727AA984383C747003AC8230AE2
:10980000F10097D0FFFFE78000B670008545054561
:1098100097A0FFFFE78020ED30099305700F094501
:1098200097A0FFFFE78020EC3008930500080D4566
:1098300097A0FFFFE78020EB10089545114597A002
:10984000FFFFE78040EAC16717C7FF1F1307873F85
:10985000F9171CC32322070017A5FF1F130545BBDB
:1098600097A0FFFFE78000E78327C41D17C5FF1FF0
:109870001305C53B82973C480345090085458297FF
:109880008320C11A0324811A8324411A0329011A4F
:109890008329C1195D618280C16717C8FF1F035802
:1098A000683AF9176301F8083DCDB5CD011126CA14
:1098B000B7E4040083A7841222CC2E862315B100BE
:1098C00006CE2A8401478146ED45428582972AC605
:1098D00011ED17850100130565E597500100E7803C
:1098E0004014F2406244D24405618280FC44035635
:1098F000A100A28582972C0017C5FF1F0355853450
:1099000097A0FFFFE780C0E969DD17850100130517
:1099100025E397500100E780C01083A7C412ED45EE
:10992000280082977DBF8280411106C61DC98547E8
:1099300017A7FF1FA307F7AE354697A5FF1F93850F
:10994000A5AD1305603097A7FF1F238D07AC97F0D7
:10995000FFFFE780206FB240410117F3FFFF670070
:10996000236997A7FF1FA38E07AAF9B7C16717C579
:10997000FF1F0355252DF9176307F500B7E704000E
:1099800003A3C71702838280854717C7FF1F2309D8
:10999000F72A014517F3FFFF670003631783FFFFF3
:1099A000E702C3702A8408452E89B28919C900C10B
:1099B000971500009385A586610597300100E78023
:1099C000800181447D5A97100000E780E03963C729
:1099D000A404814497100000E780003A63C8A404FF
:1099E00097C7FF1F938787269C43DC47B307F9403F
:1099F00091872302F400638309048327C900B30716
:109A0000F4409587A302F4001C4C89C79C4799C376
:109A1000228582971783FFFF6700836C5C4413974E
:109A200014008504BA972390470171BF1C4813970F
:109A300014008504BA972390070069BF8327890023
:109A40000547B307F4409587A302F4008357040049
:109A5000638EE7028DC309476384E7040D47E395EE
:109A6000E7FA978701009387E72F1CCC97870100BF
:109A70009387473011A897870100938727F61CCC5E
:109A800097870100938787F65CC8BDBF9787010061
:109A90009387C7E11CCC97870100938727E2EDB736
:109AA000978701009387C7301CCC97870100938765
:109AB0002731D9BF95E51783FFFFE702C360004652
:109AC00018448347940075839D8B6317F7009710A4
:109AD0000000E78060B448C41783FFFF6700E360BD
:109AE00082801783FFFFE702635C13893500C1643E
:109AF00042094111AA890144F11413590901054A87
:109B00002EC697100000E7802026B2456348A400C7
:109B1000014541011783FFFF6700835C83A70900AC
:109B200013171400BA9783D707006388B7006394AC
:109B3000970063742A010504E1B70545D9BF17836F
:109B4000FFFFE702C355AA892E89328BB6843A8A71
:109B5000BE8A97A00000E78020FB71C92685972068
:109B60000000E78020098D4763E7A7007D55178334
:109B7000FFFF6700435683DB440097100000E78037
:109B8000A0242A8497100000E780402593077400E2
:109B900031443305850263CDA70297100000E780AA
:109BA000A02297100000E78020222A84971000004E
:109BB000E780C0229307740031443305850263C3F4
:109BC000A70497100000E78020209307450029A8EC
:109BD00097100000E7808020330585021307F017F7
:109BE0009307C017E35FA7FA2D55E3C277F9630423
:109BF0000B02D6865286A6854A8597200100E7800B
:109C000020BAB5B797100000E780401D33058502E4
:109C10009307C5FFD1BF832749001385C90083D5AA
:109C2000270097000000E78000EC61F581B76955D7
:109C30003DBF97C7FF1F239DA70097C7FF1F9387AF
:109C4000E700904381470C463307F5004207418304
:109C50006393B70082805446139847008507C296E5
:109C60002390E600D5B797C7FF1F938727FE9C4335
:109C700003C58700828017C5FF1F035565FD8280DD
:109C80001783FFFFE7022344C1671387D7FF630BE6
:109C9000E502636AA700F1176300F5020145178327
:109CA000FFFF670083441387E7FF6302E502FD17A8
:109CB0001D8D13351500E5B797500000E780C026CD
:109CC0007D15C5BF97500000E78040FBD5BF97507A
:109CD0000000E78060F9EDB71783FFFFE702A33EBE
:109CE0004111AA8401442EC697100000E780C008E5
:109CF000B2456348A400014541011783FFFF670097
:109D0000C33E9C48131514003E9583570500E38518
:109D1000B7FE0504C9BF03485500814693F7F60F07
:109D200063E5070181473E85828058459397560039
:109D3000BA9703D727006316B70003D70700E304D9
:109D4000C7FE8506E1BF8346450001479377F70FBD
:109D500063E4D700814711A81C4513165700050777
:109D6000B29703D60700E313B6FE3E8582801783C1
:109D7000FFFFE702A33393170501C18797CAFF1FAF
:109D8000938ACAEC635BF00883A70A00C0479C472C
:109D900003570400198D420541816368F5000144B1
:109DA00022851783FFFF6700A33312052A94CDBFD6
:109DB000DC4713944900014A3E94834744006341C1
:109DC000FA02014A834754006349FA028509C2092D
:109DD00093D9090183A70A009847E3EBE9FCC1B7CF
:109DE0001C4413195A00A6853E994A859700000025
:109DF000E780C0EE05E1050AC9B75C4413195A00B3
:109E0000A6853E994A8597000000E78020ED19E17C
:109E1000050A4DBFE30C09FA61B7AA8481495DBF09
:109E20001783FFFFE702232A1C452A8481E7930753
:109E3000C5001CC51C44231204001CC09307F00F6E
:109E400063EDB70093F5F50F228597200000E780BA
:109E500020E21783FFFF6700432993940501C16740
:109E6000C18063F9F500A685228597200000E78070
:109E700040E5C5B7C18193F5F50F22859720000015
:109E8000E78000DFA685228597200000E78040E07C
:109E9000C9B797C7FF1F938767DB884382801C453C
:109EA00099C797C7FF1F23A3A7DA014582807D5575
:109EB000828097C7FF1F938767D9984383474500E0
:109EC000484792073E9582801783FFFFE702A31F52
:109ED000617100451C183EC6B70780013EC81C18BA
:109EE0003ECA8357440002CE02D002CC231EF100AA
:109EF000834784002A8902D22301F1023C083ED420
:109F000002D697000000E78000FB83570500231668
:109F1000F10297500000E78060C42307A1025C4073
:109F200003556400F18313F717008347F1025205CC
:109F30005181F99BD98FA307F10297100100E780A7
:109F4000807539CDAA840355050097A00000E780ED
:109F500080BC83D704002AD26800231CF10083D779
:109F60002400231DF1001C4803D647008C43972092
:109F70000000E78000CD8347B400CA861786010041
:109F80001306468C8117A305F4006C004810972037
:109F90000100E780E0805D611783FFFF6700E31445
:109FA0002155D5BF1C45B1CF03C5A700894613571E
:109FB0006500630BD7028D46630ED70285466300AA
:109FC000D702130740063305E50203C7B700418BEC
:109FD00015CB83C7B700BD8B3355F5408280137511
:109FE000F5031307803EC5B709671375F50313071B
:109FF0000771D1BF372709001375F5031307077CD5
:10A00000D9B7014582801783FFFFE702C30B03A97D
:10A010008500630C09048347B900AE8493F7070EEB
:10A0200085C303459900930520030D810505B305FC
:10A03000B5028844610597300100E780E0A935A0AA
:10A040002E8597000000E78020F62A8419CD97001E
:10A050000000E780605C8325C900B307B54063FA60
:10A0600087002E94B305A440E9F51783FFFF67002E
:10A07000C30785457DBF1783FFFFE702C3042A841A
:10A0800003D50500011132C636C43AC22EC002CA39
:10A0900002CC02CE97A00000E780E0A782452ACA42
:10A0A00022852ECC97000000E780E0E003570500F2
:10A0B000231EE10097500000E78040AAA2463246E6
:10A0C0009247230FA10036874C08B28622850146AD
:10A0D00097000000E780E0A605611783FFFF670097
:10A0E000C3001783FFFFE70203FE61711C183EC621
:10A0F000B70780013EC81C183ECA3C0800453ED444
:10A10000AA8402CC02CE02D002D202D6970000006E
:10A11000E78060DA8357050035592316F10297501E
:10A120000000E780A0A32307A10209C483574400CD
:10A1300081EB21594A855D611783FFFF6700E3FAD0
:10A14000035564005205518197100100E780A05427
:10A150002A8965D18347B40093F7070E99C7130581
:10A16000840197300100E780609983574400231EE3
:10A17000F100834784002301F1025C40035509008C
:10A18000D98313F7070883471102231CA10093F713
:10A19000F707D98FA300F10283572900231DF1008F
:10A1A0005C40F18313F717008347F102F99BD98FC5
:10A1B000A307F10297A00000E780E0952AD235D9E5
:10A1C000834794006800139757008347B400FD8BC2
:10A1D000D98FA305F4001C4803D647008C43972071
:10A1E0000000E78000A6A6871777010013078765A0
:10A1F000740005464C10268597000000E7806094A7
:10A200002A890DD98347B400A685FD8BA305F400E8
:10A2100097000000E78060DF31BF1783FFFFE70290
:10A2200083EA832485FE2A84411126859700000055
:10A23000E78080D7834734FF93F7070E8DCB2AC67C
:10A24000268597000000E78060C809CD834734FF6A
:10A25000B245FD8BA309F4FE91C52285973001001C
:10A26000E780808741011783FFFF670003E87DD9FE
:10A270008327C4FF2685829775F5834734FF93F7BC
:10A28000070E91C7228597300100E78020870325BC
:10A2900084FE97000000E78000E5E9B71783FFFF21
:10A2A000E70263DF9C4141112A8903C70700894700
:10A2B0002E84935667006380F6040D466388C604B7
:10A2C0009307F0076304F7022E8597200000E780CC
:10A2D000C0A7AA848149C16B130C490097C7FF1F0F
:10A2E0009387C7969C43984763E4E9044101178329
:10A2F000FFFF670003DE03D745008547E3F8E7FE6D
:10A300002E8597200000E780A0A9E1B703D745007C
:10A31000E3FEE7FC2E8597200000E78000A3AA84D7
:10A32000228597200000E78060A4C204C98C5DB735
:10A33000DC470355A900139A49003E9A931705017B
:10A34000C187635DF00083570A006397A70263E744
:10A3500074038327CA00034D5A002DA0A16721670B
:10A36000A98F1307F7EFE374F7FE639709009700CF
:10A370000000E780209161FD85098DB783278A0061
:10A38000034D4A00835DA90003576900216A138BBE
:10A39000C7003AC6814A33CA4D01631E5D0197C7A3
:10A3A000FF1F9387278B9C43E1DBA2866286814552
:10A3B00026858297D1B7A1679387F7EF930C4BFF60
:10A3C00063F24703B2455A8597F0FFFFE780A0711B
:10A3D0000DC103278B00104709CE10436382C402CE
:10A3E0003107D5BFEE85668597000000E780008FB6
:10A3F00071F993861A0093FAF60F130B0B0271BFD3
:10A40000835644005C43E3E9F6F622853AC697108A
:10A410000000E780807DA1679387D7042A8A035DC7
:10A420004400324763E897008347D90093E707F871
:10A43000A306F9001C4766852286E2858297C167DC
:10A440000844FD17337AFA00529508C02312A4017C
:10A4500025B797B7FF1F9387677F9843814715C339
:10A460001447814763FFD500939745004C47BE953D
:10A4700019C903C7550081476375E600DC45160618
:10A48000B2973E85828003C745008147E37BE6FEA5
:10A4900016069C45F5B71783FFFFE70223C1AA897B
:10A4A0002E8A814497BAFF1F938A4A7A83A70A00AB
:10A4B000984763E6E4001783FFFF670063C2DC4749
:10A4C0001394440001493E9413BB14008347440095
:10A4D000634BF900014913BB140083475400634FD9
:10A4E000F9008504E1B70844931759005287DA86CA
:10A4F0000146A2853E9582990509C9BF4844931734
:10A5000059005287DA860546A2853E95829905094B
:10A51000E9B71783FFFFE70203BB814517F5FFFF8C
:10A520001305054897B7FF1F239407729700000093
:10A53000E780A0F61783FFFF670023BB97B7FF1FD5
:10A540009387C7709C4395C31783FFFFE702A3B7A8
:10A55000814517F5FFFF1305A54497000000E7802C
:10A56000C0F31783FFFF670043B882801783FFFFA4
:10A57000E702C3B337E40400832784124111231593
:10A58000E100AE893289368A3A8681460147ED4537
:10A59000AA8482972AC621C90356A100D285974072
:10A5A0000100E780C0248327C413CE8526858297C7
:10A5B000058905C98327440D2314210101462C0078
:10A5C000268582972A8401C9B7E7040083A7C712AA
:10A5D000ED4528008297228541011783FFFF670020
:10A5E00023B04944D5B76554FDB75C41FD175CC144
:10A5F00082801783FFFFE70203ADB7E70400FC5F2B
:10A60000829795473305F50281450D811783FFFF3A
:10A610006700A3AD1783FFFFE702E3AAB7E70400D3
:10A62000FC5F829795473305F5020D811783FFFF85
:10A630006700A3AB1783FFFFE702E3A8B7E70400B7
:10A6400083A7870B0355050082971783FFFF6700D9
:10A65000C3A91783FFFFE70203A70355050032874D
:10A66000AE861796FF1F035646E397B5FF1F9385E7
:10A67000A55E97000000E780A0EF1783FFFF67004B
:10A68000C3A61783FFFFE70203A4B7E7040083A76D
:10A69000C71782971783FFFF670023A51783FFFF64
:10A6A000E70263A2B7E7040083A7871397B5FF1FEC
:10A6B0009385855A829701451783FFFF6700E3A2C0
:10A6C0001783FFFFE70223A0B7E7040083A7C71F94
:10A6D00081451795FF1F035545D882971783FFFFC4
:10A6E0006700A3A01783FFFFE702E39DB7E704001D
:10A6F00083A7871397B5FF1F938505578297014559
:10A700001783FFFF6700639E1783FFFFE702A39B8A
:10A71000B7E7040083A7C71F81451795FF1F03559F
:10A72000C5D982971783FFFF6700239C1783FFFF1C
:10A73000E70263992E8597800000E780E0AF97805D
:10A740000000E780E0EC1783FFFF6700039A1783A0
:10A75000FFFFE702439797800000E780E0F617834A
:10A76000FFFF670083985C49E1175CC95CC58357AC
:10A770002501A1072319F50083570501A107231817
:10A78000F5008280F1473305F50297B7FF1F9387E5
:10A79000A74F9C433E9582808D476315F60803D7EB
:10A7A0004600854763F0E7081783FFFFE702A391A0
:10A7B000368536842E8997100000E780005929C914
:10A7C0008357440093140501C18063E397042285F5
:10A7D00097100000E7806057FD1423129400930740
:10A7E000A0026300F5029307B0026307F502930726
:10A7F0009002631FF500228597000100E780C08565
:10A8000001A80146CA85228597A00000E78060B0B4
:10A810001783FFFF6700638D228597100000E78094
:10A82000C003FDB7828097B6FF1F938626469C42E1
:10A83000014599CF9843D44217B6FF1F2328E64419
:10A840006396D70097B6FF1F23A4E6441385C7FE7F
:10A8500082801783FFFFE702038797000000E780ED
:10A86000A04B714433058502914597900000E78025
:10A8700020E911E565551783FFFF6700038797B748
:10A88000FF1F23A1A74097000000E780E0483305A1
:10A890008502914597900000E78080E661DD97B7DB
:10A8A000FF1F23A3A73E97000000E780E04697B76D
:10A8B000FF1F2393A73C97000000E780E04597B770
:10A8C000FF1F239CA73A977701009387E7FC17B7F0
:10A8D000FF1F2327F73A97070000938707E917B769
:10A8E000FF1F232DF738014579B71773FFFFE702E4
:10A8F000837DAA8517B5FF1F130505389710000043
:10A90000E780C05B1773FFFF6700237E1773FFFFAD
:10A91000E702637B97000000E78060FD971000006E
:10A92000E780405B97B7FF1F938747369C4391CFE3
:10A930001387C7FE19CB83D5C7FF17B5FF1F1305B4
:10A94000653597200100E78020191773FFFF670026
:10A95000C3791773FFFFE702037797000000E780D2
:10A96000C0EC09CD834785002A8493F7070499EB4F
:10A970000355E50097000000E78080F91773FFFF9B
:10A980006700A3768347C5009304450117B9FF1FED
:10A990001309C92F85E3832709005CC997B7FF1FF7
:10A9A00023A6972E83274900F1FB97B7FF1F23A10A
:10A9B000972EE9B7FD172306F50061059780000083
:10A9C000E780C0D68307840063CB070483478400F5
:10A9D00093E707F82304F400B7E704009C5F82972D
:10A9E0004205A94741813375F5028347840093F7F7
:10A9F00007FCC98F2304F4008347D4003E951C4014
:10AA00002318A40089CF984319CB8347C400504032
:10AA1000814585073305F502420541810297832769
:10AA200009005CC897B7FF1F23A297268327490018
:10AA300089E797B7FF1F23AD97248347C4009DDFA5
:10AA40008355040117B5FF1F1305C5249720010086
:10AA5000E780800825B71773FFFFE702C36697B743
:10AA6000FF1F938767489C4701448583858B85E357
:10AA7000AE84B2853A8697100000E780804B2A8426
:10AA800019C597100000E780C041829408CC228548
:10AA90001773FFFF670063651773FFFFE70203612A
:10AAA00041112E8932C6AA8997000000E780C03183
:10AAB000324713060502CA86970500009385C5CC68
:10AAC00017B5FF1F1305451B97000000E780E0F84E
:10AAD0002A8425C99304C50097000000E780E0415F
:10AAE0001946AA85268597100000E78080158545C0
:10AAF000268597100000E780601117750100130587
:10AB000065D74E9583450500268597100000E780A0
:10AB100020165C4831468145A1075CC85CC4835758
:10AB20002401E1172319F40083570401E1172318C6
:10AB3000F4001C4C3E859770FFFFE780C05BA304C8
:10AB40002501228541011773FFFF670063591773C1
:10AB5000FFFFE70243574111AA842EC632C4971063
:10AB60000000E7806036004DB245224683478400EE
:10AB70000CC050C093F7F70393E707042304F400D5
:10AB800023180400268597100000E7808031834752
:10AB90009400A9462317A40013D7370005073307ED
:10ABA000D7029D8B85072306F400A306E40083C724
:10ABB0000401D8488507230FF7FE17B7FF1F1307B7
:10ABC000E70C5843232A04009307440129E317B7ED
:10ABD000FF1F232FF70A17B7FF1F2329F70A17B400
:10ABE000FF1F1304240B228597200100E78000E15A
:10ABF0001C44858B5D8D19E58145228597200100D8
:10AC0000E78080ED41011773FFFF6700034E1CC30F
:10AC100017B7FF1F232EF706D9B71773FFFFE702F9
:10AC2000834A97050000938565B7014597000000AA
:10AC3000E78000B001451773FFFF6700034B1773F0
:10AC4000FFFFE702434897000000E78080B01773DA
:10AC5000FFFF670083498347C500A5E31773FFFF24
:10AC6000E70263462A840355E50097000000E78069
:10AC700000C821C18347840093F7F7FB2304F40045
:10AC80001C4091C7DC4381C74C4001458297970027
:10AC90000000E78080B917B5FF1F1305A5FF9720B7
:10ACA0000100E780A0E50355E40097000000E7807D
:10ACB00020C61773FFFF6700434382801773FFFFAF
:10ACC000E702634097B7FF1F938747FC9705000093
:10ACD000938565C817B5FF1F1305C5FB23A00700A3
:10ACE00023A2070097200100E780E0CE1773FFFF43
:10ACF0006700A33F1C4D91CFDC4381CF1773FFFF4B
:10AD0000E702633C8345070082971773FFFF6700E4
:10AD1000C33D828097B7FF1F938707FA9C4303C503
:10AD20000700828097B7FF1F938707F99C4303C5ED
:10AD30001700828097B7FF1F938707F89C4303C5CE
:10AD40002700828097B7FF1F938707F79C4303C5AF
:10AD50004700828097B7FF1F938707F69C4303C580
:10AD60003700828097B7FF1F938707F59C4303C581
:10AD70005700828097B7FF1F938707F49C4303C552
:10AD80006700828097B7FF1F938707F39C4303C533
:10AD90007700828097B7FF1F938707F29C4303C514
:10ADA0008700828097B7FF1F938707F19C4303C5F5
:10ADB0009700828097B7FF1F938707F09C4303C5D6
:10ADC000A700828097B7FF1F938707EF9C4303C5B7
:10ADD000B70011E11D45828097B7FF1F9387C7ED2C
:10ADE0009C4303C5C700828097B7FF1F9387C7ECBA
:10ADF0009C4303C5D700828097B7FF1F9387C7EB9B
:10AE00009C4303C5E700828097B7FF1F9387C7EA7B
:10AE10009C4303D50701828097B7FF1F9387C7E93B
:10AE20009C4303C52701828097B7FF1F9387C7E81C
:10AE30009C4303D54701828097B7FF1F9387C7E7DD
:10AE40009C4303D56701828097B7FF1F9387C7E6AE
:10AE50009C4303D58701828097B7FF1F9387C7E57F
:10AE60009C4303C5A701828097B7FF1F9387C7E460
:10AE70009C4303C5B701828097B7FF1F9387C7E341
:10AE80009C4303C5C701828097B7FF1F9387C7E222
:10AE90009C4303C5D701828097B7FF1F9387C7E103
:10AEA0009C438857828097B7FF1F9387E7E09C43B6
:10AEB00003D5C702828097B7FF1F9387E7DF9C43C4
:10AEC00003D5E70219E11305800C828097B7FF1FB5
:10AED000938787DE9C4303C50703828097B7FF1FD4
:10AEE000938787DD9C43C85B828097B7FF1F93875A
:10AEF00027DC8843828097B7FF1F9387A7DB8843AF
:10AF0000828019E17D558280F5DE984265DFFDD9AA
:10AF100017B7FF1F130747FD1847AA877155058B01
:10AF2000631D072403C507001547E37DA7FC03C77E
:10AF300037001305F0057D171377F70FE364E5FC81
:10AF400003C35700E30003FC83C86700E38C08FADF
:10AF500003C77700494579171377F70FE364E5FADC
:10AF600003C7A70011481305F7FF1375F50FE36B2F
:10AF7000A8F803CE97000D481305FEFF1375F50FD3
:10AF8000E362A8F803C8B7006309080065181378DE
:10AF9000F80F1305600DE36705F703C5C70079488F
:10AFA00079151375F50FE36FA8F403C8D7000D45A5
:10AFB0007D181378F80FE36705F503D80701930EA2
:10AFC00040175118420813580801E3ED0EF303C867
:10AFD000E7007D181378F80FE36605F303C827012F
:10AFE0007D181378F80FE36F05F103C88700C54E8D
:10AFF00075181378F80FE3E70EF103D86701856E33
:10B00000938EBEE06D18420813580801E3EC0EEF72
:10B0100003D847016D18420813580801E3E40EEF06
:10B0200003D887017918420813580801E36C05ED2D
:10B0300003C8A7017D181378F80FE36505ED03C574
:10B04000B7011D487D151375F50FE36DA8EA03C51B
:10B05000D701714879151375F50FE365A8EA03D593
:10B06000E7011308E00F7D1542054181E36CA8E874
:10B0700003C50702494879151375F50FE364A8E87D
:10B08000C85301C937C834005915130858BFE36BBA
:10B09000A8E603A8870237C53400130555BF591821
:10B0A000E36205E717B5FF1F2326C5C003C60501E8
:10B0B00017B5FF1F2322F5C00545E375C5E403D886
:10B0C0002501D04933760603E31E06E203C61501C7
:10B0D000E30A06E217B6FF1F232CB6BC83C5270080
:10B0E00001466387A50003C61700F1453306B60283
:10B0F00083C707039305C00272971A071307C70592
:10B1000016031A9796084697B387B70241553E979C
:10B110003297420741836362E8061773FFFFE70235
:10B1200083FA368597800000E780A06897000100C9
:10B13000E78020482A8497A00000E780805A2A945C
:10B1400097F00000E78060262A9497900000E7803F
:10B15000A0812A9497F0FFFFE780E06F2A94974040
:10B160000000E78060932A9497700000E780A09C1D
:10B1700022951773FFFF670043F782801773FFFF65
:10B18000E70263F44111A307A10097A00000E78044
:10B19000A0C59305F100170500001305E5B597F06C
:10B1A000FFFFE780802F014541011773FFFF670014
:10B1B000C3F31773FFFFE70283EE17B4FF1F1304F7
:10B1C000A4D20328840079599368180097B4FF1F0C
:10B1D00023A014D31378180063100802BA84BE8920
:10B1E000368B328A2E89AA8A97F0FFFFE780E0A784
:10B1F0007D15269519E531594A851773FFFF6700BC
:10B2000083ED97F0FFFFE78040A67D152695A167A7
:10B21000E353F5FE97B7FF1F9387C70398433E8C10
:10B22000814B01CB014597F00000E7802044933B20
:10B2300015004A85DA865686D28597900000E78009
:10B24000C04D2A8911CD1C44F99B17B7FF1F23213C
:10B25000F7CA83270C00CDD3E3800BFA829769BF2E
:10B26000268597B7FF1F23A307C897F0FFFFE78046
:10B27000809C4146CE8517B5FF1F130565D09730DA
:10B280000100E780C05697D00000E7804099032571
:10B29000040B97D00000E780009D054597D0000083
:10B2A000E78000A4054597000000E78060EDA9B79E
:10B2B00097B7FF1F938747C39C47858BEDC71773CD
:10B2C000FFFFE70243E017B5FF1F1305A5C997B7B6
:10B2D000FF1F23AB07C097B7FF1F23A907C097B76E
:10B2E000FF1F23A707C097200100E7802081975008
:10B2F0000000E780E0F597100100E780A04C971070
:10B300000100E780A05297B7FF1F938767BC9C435B
:10B3100091C7054597800000E780402097B7FF1F41
:10B320009387C7A49C4399C741657D15977000001A
:10B33000E78040A297F00000E780E03D97D0000052
:10B34000E780808F97B7FF1F9387C7CE9C431397E3
:10B3500017016356070097F00000E78000AD97B72C
:10B36000FF1F23AF07C097B7FF1F23AD07C097B7D5
:10B37000FF1F23AB07C097B7FF1F23A907C0970084
:10B380000000E780008C97000000E780007297F0D3
:10B39000FFFFE780401897F00000E78040D6177362
:10B3A000FFFF670083D4828097B7FF1F9387C7B3DF
:10B3B000884382801773FFFFE702E3D09780000085
:10B3C000E780607597800000E780C0771773FFFF04
:10B3D0006700A3D11773FFFFE70243CD2A849304CC
:10B3E000140201112E85B289A685214636C63A89F6
:10B3F00097300100E780403D0DE9B24638082686C7
:10B40000CE851305940497500000E78060412146E3
:10B410002C084A8597300100E780003B1335150062
:10B4200005611773FFFF6700A3CB0145D5BF1773F5
:10B43000FFFFE70243C99305450617B5FF1F130534
:10B44000E58797100100E78020691773FFFF670009
:10B45000C3C91773FFFFE70203C741112EC697F058
:10B46000FFFFE780601BB24588C141011773FFFFF2
:10B470006700A3C71773FFFFE70243C3AA842E84A4
:10B4800097800000E780006CAA8985452285970097
:10B490000000E780E07D83C7E4011389940899E305
:10B4A00013890403CE85228597000000E780407C45
:10B4B000214693051902228597000000E7806078F5
:10B4C00097B7FF1F938747A28C43228597100000F0
:10B4D000E780C08221469385840222859700000080
:10B4E000E78020761773FFFF670083BF1773FFFFA6
:10B4F000E702E3BA397197F00000E780E0B4930502
:10B50000400661E997800000E7800060630205144F
:10B5100097A7FF1F83C7477C13B7170097A6FF1F86
:10B52000238CE67A014499CFC16417B9FF1F130930
:10B53000A99B9309400EFD1497000000E780C08688
:10B540006342A40A97F0FFFFE780000D4169B72925
:10B550000900096AFD7A2A8B81447D199389F97B58
:10B56000130A0A71938A8AC797000000E780C08394
:10B5700063D7A4041304400EB387840217B7FF1FD8
:10B58000130787960324070B3E948357C4016382F5
:10B59000270B18403307EB4063EAE9008347440078
:10B5A0008507B3874703D6976365F708014681454A
:10B5B000094597F0FFFFE780604EAA8B29E5974089
:10B5C0000000E780808385476317F50689659385CA
:10B5D000057117A5FF1F1305656E97100100E78021
:10B5E000A04F95A0B30734030327090BBA9703D7DD
:10B5F000C7016308970003C75700A382070023828F
:10B60000E700050415BF9305C500228597000000DB
:10B61000E78080E65E852286976501009385C526D2
:10B6200097F0FFFFE780E0525E8597100000E7800B
:10B63000608A850415BF97B7FF1F9387E78A9C47E9
:10B640008D83858BC1F721611773FFFF6700A3A866
:10B6500001468545094502D002D202D402D697F0B0
:10B66000FFFFE780A043AA8479DD97F00000E78020
:10B67000E09C1389C4002A8481454A859700000014
:10B68000E780005F0C4041464A8597000000E78054
:10B69000405B832944006385090C4E8502D802DA99
:10B6A00002DC02DE97300100E78060402ACE1410F1
:10B6B00005462C0808184ECC97500000E780E00A99
:10B6C0001375F50F51ED8355840093E525004A85E8
:10B6D00097000000E780E05E11460C104A85970055
:10B6E0000000E78000560146976501009385451AE2
:10B6F000268597F0FFFFE780C0452685970000006C
:10B70000E780407D5C40A1D3014685450D4597F01B
:10B71000FFFFE780A038AA841DD548401389C400E4
:10B7200097300100E780A0382AC64A8597000000BC
:10B73000E780404C3246636FC5004C404A85970015
:10B740000000E780005001468145268597F0FFFF05
:10B75000E7802040268597000000E780A077E5B5C8
:10B7600083558400ADB71773FFFFE702C39597A712
:10B77000FF1F938767779C471DC193E7870017A535
:10B78000FF1F1305A55317A7FF1F2323F776971055
:10B790000100E78040321773FFFF67000395DD9BD0
:10B7A00017A7FF1F2326F77497300000E780E06497
:10B7B0007DF117A5FF1F1305655097100100E78065
:10B7C000E033D1BF1773FFFFE702638D4169AA8998
:10B7D0002E8AB28A368BBA8B814417ACFF1F130CAA
:10B7E000AC70930C400E7D1997F0FFFFE780C05BB3
:10B7F00063C4A40001443DA03384940383270C0B4D
:10B800003E948357C401638627055A87D68652869D
:10B81000CE851305040397000000E780E0BB01C953
:10B8200023800B0022851773FFFF6700C38A8347BD
:10B83000F40185C35A87D6865286CE8513059408AF
:10B8400097000000E78040B909C585472380FB00C9
:10B85000D1BF850451BF835745006380071E17730E
:10B86000FFFFE702A38401112A8497000000E7800C
:10B87000C04D09C985476309F50605611773FFFFC8
:10B880006700038697E00000E780007C7DF5835722
:10B8900044004947ED9BE392E7FEC14522859700AE
:10B8A0000000E7804033AA84228597000000E780EB
:10B8B000204F0357440002CE91472A89631AF700AC
:10B8C000228597000000E780A0513C082ACC3ECE9C
:10B8D00097E00000E78080765C55C5D374084A86FF
:10B8E000A6850545829751BF03574400D147E3F62B
:10B8F000E7F8032A0400C169014997AAFF1F938A48
:10B90000AA5E130B400EFD1997F0FFFFE780C049B8
:10B91000634FA90E2285032A040097000000E780E8
:10B92000C042A1452A89228597000000E780A02A0D
:10B93000AA84228597000000E780804A14402A8666
:10B94000AA8978082685CA8597000000E780C0E7A5
:10B95000AA8405D503C7F40189476315F700834717
:10B96000C10181DF5546D2851385640097300100FF
:10B97000E780E0E7014597800000E780C01901C536
:10B9800083D7C401A5E797A7FF1F9387E7559C4777
:10B9900093551900858913D73700058B01CF89830B
:10B9A000858B6399B70001452EC697000000E7809C
:10B9B000C0DBB2454E8597800000E780601F0346DC
:10B9C000C1012A8493751900268597900000E780AD
:10B9D000E03935C1268597800000E780E01826858C
:10B9E00011C0014597800000E780004C97300000AF
:10B9F000E780A0408547E312F5E883C754001307AA
:10BA0000F00FE38CE7E68507A382F400BDB5B3042D
:10BA1000690383A70A0BBE9483D7C401638B3701E4
:10BA20005546D2851385640097300100E780C0D960
:10BA300055DD0509D1BD5DD86DB782801763FFFF65
:10BA4000E702C36697800000E780000C05C1C1646F
:10BA5000014417A9FF1F130929499309400EFD143A
:10BA600097F0FFFFE7804034634EA40017A5FF1F47
:10BA70001305C52497100100E780E0031763FFFF5B
:10BA800067000366330534038327090B3E9583570C
:10BA9000C501638897002312050097800000E780A6
:10BAA000A00C050475BF97A7FF1F9387E7439C472A
:10BAB0008D83858B8DE31763FFFFE702C36017A5B6
:10BAC000FF1F1305A51F97100100E78020031763D0
:10BAD000FFFF6700836182801763FFFFE702A35EB9
:10BAE000970500009385C5A017A5FF1F1305051D29
:10BAF00097100100E78020EE1763FFFF6700E35E09
:10BB00001763FFFFE702235C8841B7E70400BC5BD3
:10BB1000050542054181829709C585472300F50047
:10BB200005051763FFFF6700435C83C7F5FF2E859C
:10BB30008507A38FF5FE828083C7F5FFFD1793F776
:10BB4000F70FA38FF5FE99EF1763FFFFE702A357E7
:10BB5000B7E70400BC571385F5FF82971763FFFF13
:10BB60006700A35882801C41035745008D8FBA950A
:10BB70001CC12312B5003E85828093D78500A205A3
:10BB80001441DD8D835745001387E6FF18C18907EF
:10BB90002312F50013D685004111238FB6FEA38F23
:10BBA000C6FE4101828018419307F7FF1CC18357ED
:10BBB000450085072312F500A30FB7FE8280835747
:10BBC00045008D8F2312F5001C41BE950CC12E85BA
:10BBD0008280AA8703D7470008410D8FAA95239238
:10BBE000E7008CC38280184108453305A740828056
:10BBF00083574500035765001D8F1C410845338559
:10BC0000A7403305A74082801763FFFFE702A34BDD
:10BC100041112EC62A8497000000E780A0FDB2459E
:10BC20006373B50001A0835744000840BE952312FA
:10BC3000B4003E9541011763FFFF6700034B176394
:10BC4000FFFFE702434841112E84B28532C69700B8
:10BC50000000E780A0FB3246A28597300100E78014
:10BC600000B941011763FFFF670023481763FFFF17
:10BC7000E70263452E84854597000000E78000F9C0
:10BC8000230085001763FFFF670023461763FFFF4C
:10BC9000E702634341112317B10089459700000073
:10BCA000E780C0F68347E1002300F5008347F100F9
:10BCB000A300F50041011763FFFF6700034317630B
:10BCC000FFFFE702434093D78500A2054111DD8DB8
:10BCD0002317B100894597000000E78020F38347D0
:10BCE000E1002300F5008347F100A300F5004101C6
:10BCF0001763FFFF6700633F1763FFFFE702A33C83
:10BD00001397850193D78501C166938606F0D98F75
:10BD100013D78500758FD98FA2053707FF00F98DDE
:10BD20004111DD8D2EC6914597000000E78000EEA1
:10BD30006C00114697300100E78060AB410117634A
:10BD4000FFFF6700833A1763FFFFE702C3371C4119
:10BD5000854503C4070097000000E78080E6228540
:10BD60001763FFFF670063381763FFFFE702A33520
:10BD70001C414111894503C7070083C717002307EA
:10BD8000E100A307F10097000000E78080E303557E
:10BD9000E10041011763FFFF670023351763FFFFD1
:10BDA000E70263321C414111894503C7070083C77D
:10BDB00017002307E100A307F10097000000E780C8
:10BDC00040E08357E100410113D58700A2075D8D54
:10BDD000420541811763FFFF670023311763FFFFAF
:10BDE000E702632E0C4141112A8411466800973006
:10BDF0000100E780C09F9145228597000000E78001
:10BE000040DCB247C166938606F01397870113D5CD
:10BE10008701598D13D78700758F598DA207370772
:10BE2000FF00F98F5D8D41011763FFFF6700E32B72
:10BE30001C45BE950CC18280AE87944391E6584163
:10BE400001EF0CC15CC1828003C757001367170064
:10BE5000A382E700B687D5B70CC3EDB7AA87084120
:10BE600019CD1841D44398C36313D500D8C32A878A
:10BE7000034657009376160081E623200700828050
:10BE8000944381CA8C4203A847008CC36393060184
:10BE9000CCC3799A14C3A302C7003687D1BF1C450F
:10BEA000DC471D8DB777DBB6938777DB09853305D4
:10BEB000F502420541818280F147B385F50248458C
:10BEC0002E9582808347450085072302F5008280F6
:10BED0001763FFFFE702231F2A8409E41763FFFFAC
:10BEE0006700A32083474400F5DBFD1793F7F70FA6
:10BEF0002302F400E5F71C4403D72700050723912C
:10BF0000E700DC4399C3228582974C4889CD83475B
:10BF10005400898B99E71C4422859C479C439C478D
:10BF20008297232A04000040232004007DB7176372
:10BF3000FFFFE70243198357250041112EC681EB0D
:10BF40000144228541011763FFFF6700031A03576D
:10BF500005008147F146E305F7FEB385D70240456A
:10BF600085072E948345440008C4F5F5B247AA849A
:10BF700081E7232A040009A81C456C0022859C4304
:10BF80009C43829748C84DDD85472312F400B24791
:10BF900023200400231804002319F4005C485CC427
:10BFA00083D72400FD172391F40061BF1763FFFFBF
:10BFB000E702631197A7FF1F938747D28843232681
:10BFC000050023240500410597100100E78000B318
:10BFD0001763FFFF670063111763FFFFE702A30EFC
:10BFE00017A4FF1F130484CF1C40411199CF9C4715
:10BFF0002300B5002AC65CC197000000E78040FB23
:10C000001C40DC4399C33245829741011763FFFF0F
:10C010006700A30D0347450029E3584DAA877D55C6
:10C020001DCF1763FFFFE702030A1CC3DC4797A677
:10C03000FF1F23A5E6CAF156130507012390D70079
:10C04000970500009385050297100100E780A098EE
:10C0500001451763FFFF670043097D558280828099
:10C060001763FFFFE702230601116146814528009F
:10C070009760FFFFE780200897A7FF1F938707C6F9
:10C080009C4328009305F00FDC473EC69700000054
:10C09000E780C0F405611763FFFF6700030597A7FA
:10C0A000FF1F9387A7C39C43D847A1679387C70205
:10C0B000631EF70A397106DE22DC26DA80004AD8D0
:10C0C0004ED652D456D23285B28497000000E78013
:10C0D000C0C7AA89268597000000E78020C92318D9
:10C0E000A4FC268597000000E78040C82319A4FC23
:10C0F000268597000000E78060C783D744000A8A3E
:10C10000231AA4FC858393F7F70F230EF4FC86070C
:10C11000BD0793F7073F3301F1408A8A01498347FE
:10C12000C4FD6367F902CE85130584FC232C54FDFE
:10C1300097000000E78080EA5281130104FCF2506E
:10C140006254D2544259B259225A925A2161828081
:10C15000268597000000E78060C193171900D697E5
:10C1600005092390A7001379F90F55BF828097A77F
:10C17000FF1F9387A7B69C43D847A1679387A70261
:10C18000631AF70A397106DE22DC26DA80004AD803
:10C190004ED652D456D23285B28497000000E78042
:10C1A000C0BAAA89268597000000E78020BCFD5709
:10C1B0002318A4FC26852319F4FC97000000E780CF
:10C1C000E0BA83D744000A8A231AA4FC858393F734
:10C1D000F70F230EF4FC8607BD0793F7073F3301E3
:10C1E000F1408A8A01498347C4FD6367F902CE851D
:10C1F000130584FC232C54FD97000000E78000DE2B
:10C200005281130104FCF2506254D2544259B25983
:10C21000225A925A21618280268597000000E78089
:10C22000E0B493171900D69705092390A700137956
:10C23000F90F55BF828097A7FF1F938727AA9C43BA
:10C24000D847A16789076310F70A397106DE22DC37
:10C2500026DA80004AD84ED652D456D23285328958
:10C2600097000000E78060AEAA894A859700000029
:10C27000E780C0AF835749000A8A2318A4FC85834E
:10C2800093F7F70F230CF4FC8607BD0793F7073FDE
:10C290003301F1408A8A8144834784FD63E7F402D5
:10C2A000CE85130584FC232A54FD97000000E78007
:10C2B000E0D25281130104FCF2506254D25442592C
:10C2C000B259225A925A216182804A859700000011
:10C2D000E780C0A993971400D69785042390A70000
:10C2E00093F4F40F55BF828097A7FF1F9387079F92
:10C2F0009C43D847A1679387E704631EF70A397107
:10C3000006DE22DC26DA80004AD84ED652D456D237
:10C310003285B28497000000E78020A3AA89268591
:10C3200097000000E78080A42318A4FC26859700CE
:10C330000000E780A0A3231AA4FC26859700000034
:10C34000E780C0A283D744000A8A2319A4FC85830E
:10C3500093F7F70F230EF4FC8607BD0793F7073F0B
:10C360003301F1408A8A01498347C4FD6367F902BA
:10C37000CE85130584FC232C54FD97000000E78034
:10C38000E0C55281130104FCF2506254D254425968
:10C39000B259225A925A2161828026859700000064
:10C3A000E780C09C93171900D69705092390A70032
:10C3B0001379F90F55BF828097A7FF1F93870792C4
:10C3C0009C43D847A1679387C704631AF70A39715A
:10C3D00006DE22DC26DA80004AD84ED652D456D267
:10C3E0003285B28497000000E7802096AA892685CE
:10C3F00097000000E7808097FD572318A4FC26854E
:10C40000231AF4FC97000000E780409683D744008D
:10C410000A8A2319A4FC858393F7F70F230EF4FCF3
:10C420008607BD0793F7073F3301F1408A8A014928
:10C430008347C4FD6367F902CE85130584FC232C72
:10C4400054FD97000000E78060B95281130104FC9D
:10C45000F2506254D2544259B259225A925A21612E
:10C460008280268597000000E7804090931719008E
:10C47000D69705092390A7001379F90F55BF82803D
:10C4800097A7FF1F938787859C43D847A167DD0740
:10C490006317F7041763FFFFE702E3C27971328580
:10C4A000328497000000E780408A2AC622859700E0
:10C4B0000000E780A08B2311A102228597000000D5
:10C4C000E780A088B2452300A10228089700000059
:10C4D000E780C0B045611763FFFF670003C182803A
:10C4E0009797FF1F9387877F9C43D847A1679387C0
:10C4F00087046317F7041763FFFFE702C3BC797172
:10C500003285328497000000E78020842AC6228585
:10C5100097000000E78080852311A1022285970003
:10C520000000E7808082B2452300A102280897001E
:10C530000000E780A0AA45611763FFFF6700E3BA28
:10C5400082809797FF1F938767799C43D847A1679D
:10C550009387A7046312F7021763FFFFE702A3B6EE
:10C5600001112800814597000000E78020A70561A0
:10C570001763FFFF670063B782809797FF1F93875A
:10C58000E7759C43D847A167938757026319F70261
:10C590001763FFFFE70223B30111328597F0FFFF16
:10C5A000E780A07A2308A1008145280097000000B9
:10C5B000E780C0A205611763FFFF670003B38280B5
:10C5C0009797FF1F938787719C43D847A1679387ED
:10C5D000E702631BF7041763FFFFE702C3AE011115
:10C5E0003285328497F0FFFFE7804078AA84228565
:10C5F00097F0FFFFE7808077854709E9228597F06C
:10C60000FFFFE78080744205B337A0002800814512
:10C61000231891003ECA97000000E780209C056126
:10C620001763FFFF670063AC82809797FF1F9387B4
:10C63000E76A9C43D84799476313F7081763FFFFDE
:10C64000E70263A879713285328497F0FFFFE780B3
:10C65000C06F2AC6228597F0FFFFE7802071231064
:10C66000A102228597F0FFFFE780206E2301A1023F
:10C67000228597F0FFFFE780406DA301A10222858C
:10C6800097F0FFFFE780606C2302A102228597F0FC
:10C69000FFFFE780806B2313A102228597F0FFFF45
:10C6A000E780A06AB2452314A10228089700000081
:10C6B000E780C09245611763FFFF670003A3828094
:10C6C0009797FF1F938787619C43D847A1679387FC
:10C6D000C7036313F7081763FFFFE702C39E79716F
:10C6E0003285328497F0FFFFE78020662AC62285D4
:10C6F00097F0FFFFE78080672310A102228597F063
:10C70000FFFFE780A0662311A102228597F0FFFFBB
:10C71000E780A0632302A102228597F0FFFFE78054
:10C72000C062A302A102228597F0FFFFE780E061CB
:10C730002303A102228597F0FFFFE7800061B24545
:10C74000A303A102280897000000E7802089456123
:10C750001763FFFF6700639982801763FFFFE7029B
:10C76000839601112A8497F0FFFFE780005EAA8478
:10C77000228597F0FFFFE780605F228597F0FFFF3B
:10C78000E780C05E035744008D4763F7E7002285CA
:10C7900097F0FFFFE780805D228597F0FFFFE7803D
:10C7A000E05C2800A68597000000E78020830561F3
:10C7B0001763FFFF670063939797FF1F93870752E5
:10C7C0009C43D847A167FD07631FF7001763FFFF6E
:10C7D000E702638F328597000000E78040F8176317
:10C7E000FFFF6700839082809797FF1F9387074F13
:10C7F0009C43D847A167E5076315F7081763FFFF58
:10C80000E702638C79713285328497F0FFFFE7800D
:10C81000C0532AC6228597F0FFFFE7802055228566
:10C8200097F0FFFFE78080542310A102228597F044
:10C83000FFFFE780A053520551812311A1022285F9
:10C840002302010297F0FFFFE7802050A302A1021C
:10C85000228597F0FFFFE780404F2303A102228546
:10C8600097F0FFFFE780604EB245A303A1022808BE
:10C8700097F0FFFFE780807645611763FFFF670051
:10C88000C38682809797FF1F938747459C43D8476D
:10C89000A1679387E703631FF7001763FFFFE702B2
:10C8A0008382328597000000E78060EB1763FFFF0B
:10C8B0006700A38382809797FF1F938727429C433B
:10C8C000D847A16793874704631EF7021753FFFFFA
:10C8D000E702637F79713285328497F0FFFFE7804A
:10C8E000C0462AC6228597F0FFFFE7802048B24560
:10C8F000280897F0FFFFE780606E45611753FFFF40
:10C900006700A37E82809797FF1F9387273D9C43F4
:10C91000D847A167938787026310F7041753FFFF77
:10C92000E702637A79713285328497F0FFFFE780FE
:10C93000C0412AC6228597F0FFFFE7800041B2453B
:10C940002300A102280897F0FFFFE78020694561D6
:10C950001753FFFF6700637982801753FFFFE702D9
:10C960008376011197F0FFFFE780203EAA8528001B
:10C9700097F0FFFFE780806605611753FFFF6700B0
:10C98000C3769797FF1F938767359C43D847A16766
:10C99000D107631FF7001753FFFFE702C372328509
:10C9A00097000000E780A0FB1753FFFF6700E373C9
:10C9B00082809797FF1F938767329C43D847A16770
:10C9C000C507631FF7001753FFFFE702C36F3285E8
:10C9D00097000000E780A0F81753FFFF6700E3709F
:10C9E00082809797FF1F9387672F9C43D847A16743
:10C9F000B907631FF7001753FFFFE702C36C3285C7
:10CA000097000000E780A0F51753FFFF6700E36D74
:10CA100082809797FF1F9387672C9C43D847A16715
:10CA2000AD07631FF7001753FFFFE702C3693285A5
:10CA300097000000E780A0F21753FFFF6700E36A4A
:10CA400082809797FF1F938767299C43D847894720
:10CA50006318F7021753FFFFE702E36601113285FF
:10CA600032C897F0FFFFE780402EAA85280097F094
:10CA7000FFFFE780A05605611753FFFF6700E366DD
:10CA800082809797FF1F938767259C43D847A167AC
:10CA90008D076311F7041753FFFFE702C36201110B
:10CAA0003285328497F0FFFFE780202A1306610069
:10CAB000AA844C00228597300000E780C02328001C
:10CAC000A68597F0FFFFE780605105611753FFFFD0
:10CAD0006700A36182809797FF1F938767209C431D
:10CAE00081CFDC4391CB1753FFFFE702C35D8297F1
:10CAF0001753FFFF6700635F82801753FFFFE70252
:10CB0000835C79713C08AE843ED2A165B7070A0008
:10CB10002A843ED448103C08DD053ED636C432C6D1
:10CB20003AC297D0FFFFE780E02F12474810BA853E
:10CB300097F0FFFFE780C01332464810B28597F0A8
:10CB4000FFFFE780E014A2464810B68597F0FFFF8C
:10CB5000E7800012501001478146A685228597D0B4
:10CB6000FFFFE780805145611753FFFF6700E357E0
:10CB70001753FFFFE702235501117C000329C5016C
:10CB8000AE843ECAA165B70707002A843ECC480898
:10CB90007C00C5053ECE97D0FFFFE780A0288345E7
:10CBA000D900480897F0FFFFE780800C5008014744
:10CBB0008146A685228597D0FFFFE780004C05615E
:10CBC0001753FFFF670063521753FFFFE702A34F9E
:10CBD00083C7950093F7F707A384F500970000003B
:10CBE000E78040F91753FFFF670023501753FFFFFB
:10CBF000E702634D79713C08AE843ED2A165B70768
:10CC000009002A843ED448103C08938545043ED64A
:10CC100032C636C497D0FFFFE780C020A246481036
:10CC2000B68597F0FFFFE780A00432464810B28532
:10CC300097F0FFFFE780C005501001478146A685A9
:10CC4000228597D0FFFFE780404345611753FFFFE0
:10CC50006700A3491753FFFFE702E34683C7950028
:10CC600041112A8493F7F707A384F50032852EC675
:10CC700097F0FFFFE780800F85672AC46370F50295
:10CC800097700000E78020E92246B24509ED114780
:10CC90008146228597000000E78060E64101175336
:10CCA000FFFF6700834401478346F501DDB7175353
:10CCB000FFFFE702A33F01113C003ECAB7070A008D
:10CCC0003ECC3C003ECE83C79500AA89328593F7BF
:10CCD000F707A384F5002E8497F0FFFFE780000993
:10CCE0008567637DF504A165AA849385850448085A
:10CCF00097D0FFFFE7800013268597700000E7803C
:10CD000080E12A8929E19145480897F0FFFFE780F3
:10CD100020F6A685480897F0FFFFE78060F7CA85F0
:10CD2000480897F0FFFFE780A0F4014781465008CC
:10CD3000A2854E8597D0FFFFE78020340561175309
:10CD4000FFFF6700E3398145480897F0FFFFE78060
:10CD500020F20349090275BF1753FFFFE7020335AD
:10CD600079711C103ECAB7070F003ECC404D1C1015
:10CD7000AA84AE894808994532C636893ECE97D0F6
:10CD8000FFFFE780200A32464808B28597F0FFFF90
:10CD9000E78000EE630C0902A545480897F0FFFF05
:10CDA000E780C0E62546CA8597200100E78020A4D9
:10CDB000500801478146CE85268597D0FFFFE78042
:10CDC000C02B45611753FFFF670083318355C402B1
:10CDD000480897F0FFFFE780A0EB0355E402814588
:10CDE00005C5854785456301F502C167FD179305B4
:10CDF000F00F630BF5007D1597700000E780208E23
:10CE00009305150093F5F50F480897F0FFFFE780AD
:10CE100020E683450403480897F0FFFFE78040E5DC
:10CE200083451403480897F0FFFFE78060E48355CB
:10CE30002403480897F0FFFFE78080E5835544030B
:10CE4000480897F0FFFFE780A0E49DB71753FFFF66
:10CE5000E702632783C795008146014693F7F707EA
:10CE6000A384F50097000000E78040EF1753FFFF11
:10CE70006700A3271753FFFFE702E32479713E847D
:10CE80001C103ECA2E89B7070F00A1653ECCFD05D8
:10CE90001C10AA84480842C03AC23ECE36C432C6EC
:10CEA00097D0FFFFE78000F832464808B28597F038
:10CEB000FFFFE780E0DBA2464808B68597F0FFFF5A
:10CEC000E78000DD12474808BA8597F0FFFFE7804A
:10CED00020DC0248630C08029145480897F0FFFFE8
:10CEE000E780C0D21146A28597200100E7802090FC
:10CEF000500801478146CA85268597D0FFFFE78005
:10CF0000C01745611753FFFF6700231E8945480876
:10CF100097F0FFFFE78080CF834704002300F500F0
:10CF200083471400A300F500E1B71753FFFFE702A2
:10CF3000E31783C7950001112A8A93F7F707A384A3
:10CF4000F5003285AE8432C697F0FFFFE78000E23D
:10CF500032462A89328597F0FFFFE78000DF856738
:10CF60006373F902AA894A8597700000E780A0BA26
:10CF70002A8419ED114781464A86A6855285970075
:10CF80000000E780C0B705611753FFFF6700431536
:10CF90009387E9FF93F7F70F0547E366F7FE8347AB
:10CFA000F50195EB8947E380F9FE8346F40152854C
:10CFB00001474A86A68597000000E78040B4A16734
:10CFC000D90748083ECC230A010002CE9700000092
:10CFD000E780A0B04DBF639EE7008947639EF900DC
:10CFE00093071020231FF50097700000E780C0B75B
:10CFF0006DBF0947E39BE7FA8D47E398F9FA22856D
:10D0000097700000E78080DF9797FF1F938747ECBA
:10D010009C4399E79797FF1F938747D59C4399C7F0
:10D0200003D5040097800000E780A0CE231F0400F2
:10D0300022855DBF1753FFFFE702E30801113C00A3
:10D040003ECAB7070B003ECC3C003ECE83C79500DE
:10D050002A89328593F7F707A384F500AE8497F009
:10D06000FFFFE780A0D093170501C187635AF00640
:10D07000A1652A849385E502480897D0FFFFE780E1
:10D0800060DAA285480897F0FFFFE78060C09797B5
:10D09000FF1F9387A7CD9C43A9EB01449375F40F21
:10D0A000480897F0FFFFE780A0BC9355844093F5B4
:10D0B000F50F480897F0FFFFE78080BB93550441C8
:10D0C00093F5F50F480897F0FFFFE78060BA014736
:10D0D00081465008A6854A8597D0FFFFE780E0F992
:10D0E00005611753FFFF670043004165854605460C
:10D0F000A2857D1597500000E78060BD59DD510580
:10D1000097000100E780808F1304400633448502B6
:10D1100071B71753FFFFE70203FB0111B7070600C2
:10D120003EC683C7950021642A8993F7F707A38435
:10D13000F500AE8428009305A4040AC40AC897D059
:10D14000FFFFE78020CE300001478146A6854A8553
:10D1500097D0FFFFE78060F297E0FFFFE780801540
:10D1600013049404480822CC230A010002CE97003D
:10D170000000E780809605611753FFFF6700E3F624
:10D180001753FFFFE70283F2C1642A89014497998C
:10D19000FF1F938969D5130A8002FD1497E0FFFFF2
:10D1A000E78080C16347A40001451753FFFF670074
:10D1B00023F3B307440303A7C90ABA9703D70700A9
:10D1C0006306970083D72700638427010504F9B716
:10D1D0000545E1BF1753FFFFE70243ED2A8A2E8979
:10D1E00099C123A0050081498144979AFF1F938A22
:10D1F0006AAF614B97E0FFFFE78040C263C7A400BE
:10D200004E851753FFFF6700A3ED3384640383A7A4
:10D210000A003E948357040099E763040900232021
:10D2200089008504C1BF4146D2851305440097108B
:10D230000100E780605975F5A289E5B71753FFFF34
:10D24000E702C3E639717C083ED4B7070A003ED630
:10D250007C083ED883C795002A8A328593F7F70762
:10D26000A384F5002E8932C697F0FFFFE78000B057
:10D2700085676373F5083246AA84328597F0FFFF0D
:10D28000E780A0AC8547AA8963E8A706A1659385D6
:10D290008504281097D0FFFFE780C0B826859770D7
:10D2A0000000E78040872A8429ED9145281097F0F7
:10D2B000FFFFE780E09BA685281097F0FFFFE7803F
:10D2C000209DCE85281097F0FFFFE780609A0147E8
:10D2D00081463010CA85528597D0FFFFE780E0D99C
:10D2E000A1679387770448183EDC230A010202DE17
:10D2F00097F0FFFFE780607E21611753FFFF670013
:10D3000023DE8145281097F0FFFFE7806096A68511
:10D31000281097F0FFFFE780A0979797FF1F93874C
:10D3200027F39C4381CB22856389090097D00000B5
:10D33000E78040248345040271B797D00000E7805E
:10D34000C022CDBF1753FFFFE70243D683C7950026
:10D350004111AA8993F7F707A384F5003285AE84BB
:10D36000328A97F0FFFFE78060A08567637FF50250
:10D370002A8997600000E780007A2A84914631C5A7
:10D380008347F50105476387E70291C70D47636649
:10D39000F704AD461DA89305050303250A00414681
:10D3A00097100100E78040420DE941011753FFFF4C
:10D3B000670003D39305950803250A00414697109B
:10D3C0000100E7806040814669F54A86A6854E8562
:10D3D00097000000E780C081C9BF83250A001305BC
:10D3E000940897700000E780A02919C1C146F1BFD9
:10D3F0009797FF1F9387C7AD9C4399E79797FF1FA8
:10D400009387C7969C4399C7228597800000E78041
:10D41000208A69FD8547A30FF400228597B000009C
:10D42000E7806084228597600000E780E0734E8586
:10D4300081464A86A68597F0FFFFE780607BA1675B
:10D440009387570448003EC42302010002C697F0A8
:10D45000FFFFE780806891BF1753FFFFE70223C4F7
:10D4600083C795004111AA8993F7F707A384F500B4
:10D4700032852E89B28A97F0FFFFE780208F85677B
:10D480006374F50EAA8497600000E780C0682A8460
:10D490000DED416B014A979BFF1F938BEBA4130C7F
:10D4A000400E7D1B19A833048A0383A70B0B3E94FF
:10D4B0008357C40163836705050A97E0FFFFE78090
:10D4C000A08EE342AAFE95460DA08357C501639640
:10D4D00097029305050303A50A0041469710010032
:10D4E000E780802E994611E181462686CA854E85C1
:10D4F00097F0FFFFE780C06F85A883A50A0013059A
:10D50000040397700000E780A017C14679FD2285CB
:10D51000231E940097A00000E780E07422859760A6
:10D520000000E78060649797FF1F938767D29C4352
:10D53000A9C323000402228597D00000E78040F0B1
:10D540004E8581462686CA8597F0FFFFE780406AB0
:10D55000A1679387070448003EC42302010002C666
:10D5600097F0FFFFE780605741011753FFFF670007
:10D5700083B689472300F402E1B7397106DE22DC65
:10D580004AD8800052D456D25AD026DA4ED65ECE31
:10D590002E8A32892A8B97D0FFFFE780E07D06052F
:10D5A000710541998A8A3301A140232224FC231466
:10D5B00004FC97D0FFFFE780207C83479A00060594
:10D5C000350593F7F7072315A4FCA304FA004A8551
:10D5D000232624FC97E0FFFFE7804079931705019D
:10D5E000C1876340F0025681130104FCF25062547B
:10D5F000D2544259B259225A925A025BF24B2161DB
:10D600008280AA844A8597E0FFFFE7802076AA8976
:10D610004A8597E0FFFFE7806075A1659385C502A5
:10D620002A89130544FC97C0FFFFE780A07F268569
:10D6300097C0FFFFE780E073854511C94A86CE8514
:10D6400097C0FFFFE780606DAA8B21E9894513052C
:10D6500044FC97E0FFFFE780A061A685130544FC2A
:10D6600097E0FFFFE780C062CE85130544FC97E09A
:10D67000FFFFE780E061CA85130544FC97E0FFFFE8
:10D68000E780006101478146130644FCD2855A8534
:10D6900097D0FFFFE780609EB9B78145130544FC32
:10D6A00097E0FFFFE780C05CA685130544FC97E088
:10D6B000FFFFE780E05DCE85130544FC97E0FFFFA8
:10D6C000E780005DCA85130544FC97E0FFFFE78013
:10D6D000205C814497D0FFFFE780006AE3D4A4FA7E
:10D6E00083A70B0113971400BA9783D5070099C538
:10D6F000130544FC97E0FFFFE78080598504D9BFFC
:10D70000797106D622D44AD000184ECE52CC56CAD1
:10D7100026D25AC8AE893289AA8A97D0FFFFE780FD
:10D72000A0650605690541990A8A3301A140232AAB
:10D7300024FC231C04FC97D0FFFFE780E06383C731
:10D74000990006052D0593F7F707231DA4FCA38474
:10D75000F9004A85232E24FC97E0FFFFE780006153
:10D7600093170501C187634FF0005281130104FD37
:10D77000B250225492540259F249624AD24A424B60
:10D7800045618280AA844A8597E0FFFFE780005EBA
:10D79000A1659385A5022A89130544FD97C0FFFF63
:10D7A000E7804068268597C0FFFFE780805C85455D
:10D7B00009C9CA8597C0FFFFE78020592A8B29E154
:10D7C0008945130544FD97E0FFFFE780604AA68581
:10D7D000130544FD97E0FFFFE780804BCA851305E2
:10D7E00044FD97E0FFFFE780A04A0147814613060A
:10D7F00044FDCE85568597D0FFFFE7800088B5B7FA
:10D800008145130544FD97E0FFFFE7806046A6854C
:10D81000130544FD97E0FFFFE7808047CA851305A5
:10D8200044FD97E0FFFFE780A046814497D0FFFFCB
:10D83000E7808054E3DBA4FA83270B0113971400DD
:10D84000BA9783D5070099C5130544FD97E0FFFFFC
:10D85000E78000448504D9BF1753FFFFE702A38682
:10D8600083474500404DD5EFFD575DC48346940086
:10D8700009476363D70A0346B400854663EEC608CA
:10D880008306E40063CA06085C45F9562390D70076
:10D890009787FF1F83C7474599E3A304E400978751
:10D8A000FF1F9387A74C9C4381E78947A306F40099
:10D8B0009797FF1F9387C7999C4381E78947230662
:10D8C000F4009705000093854506AA84130504011A
:10D8D00097F00000E7802010FD57231AF4028147DB
:10D8E0001CDC01489787FF1F23AC873E9787FF1FEB
:10D8F0009387473F232E040304C0804397D0FFFF44
:10D90000E780C05161463306C502814522859740B4
:10D91000FFFFE780407E81473E851743FFFF67009A
:10D92000C37CFD57D5BF1743FFFFE702C3792A84A5
:10D930000355450297600000E780E01D19E5231EAE
:10D9400004001743FFFF6700437A8357E401F5DBC8
:10D95000930504FF174501001305452D97E00000CE
:10D96000E780E014F9BF1743FFFFE702C3752E8974
:10D97000A16541119385E5032A8436C432C6BE846D
:10D980003AC297C0FFFFE780E04912472285BA8577
:10D9900097E0FFFFE780C02D32462285B28597E0F1
:10D9A000FFFFE780E02EA2462285B68597E0FFFFC5
:10D9B000E780002E630309029145228597E0FFFF6F
:10D9C000E780C0241146A68597100100E78020E279
:10D9D00041011743FFFF670043718945228597E0A6
:10D9E000FFFFE780A02283C704002300F50083C760
:10D9F0001400A300F500E9BF1743FFFFE702A36C83
:10DA000083C79500444D054793F7F707A384F500B6
:10DA10001C42411183C707006367F7062E842A89D9
:10DA2000B1C003C7D400630FF7021787FF1F1307A6
:10DA3000E733184305C3A386F40097A00000E780EE
:10DA4000404A83C7D40099E741657D15974000009F
:10DA5000E780403083D72403918B89C797E000008B
:10DA6000E780C0134A85A28597F0FFFFE78080100A
:10DA7000A167C10748003EC42302010002C697F017
:10DA8000FFFFE780800541011743FFFF6700E36563
:10DA90001743FFFFE702236303D745008D47AA849E
:10DAA00041112E8432892E8563E3E70297E0FFFF60
:10DAB000E780C02BAA8523000900268597C0FFFFB9
:10DAC000E780A02841011743FFFF6700036297E04A
:10DAD000FFFFE780A0292AC6228597E0FFFFE780A5
:10DAE000E028B24585472A862300F900268597C09D
:10DAF000FFFFE7808022F9B7397106DE22DC26DAE3
:10DB000080004ED652D456D24AD85AD05ECEAE8974
:10DB1000B284AA8A97D0FFFFE78000250605130587
:10DB2000250241990A8A3301A140232224FC2314AF
:10DB300004FC97D0FFFFE780202383C799000605E8
:10DB40004D0593F7F7072315A4FCA384F900268558
:10DB5000232624FC97E0FFFFE7804021931705016F
:10DB6000C1876340F0025281130104FCF2506254F9
:10DB7000D2544259B259225A925A025BF24B216155
:10DB80008280AA8B03AB040097C0FFFFE780601E72
:10DB900051E583D7440001498544F11793B7170035
:10DBA000A301F4FC834734FCA165C9C79385E50450
:10DBB000130544FC97C0FFFFE780C026A685130528
:10DBC00044FC97E0FFFFE780A00ADE85130544FCD4
:10DBD00097E0FFFFE780C00B834734FC114691E3D9
:10DBE0000946DA85130544FC97E0FFFFE7806005EE
:10DBF0008144630A0900416B7D1B97D0FFFFE780DA
:10DC0000A01663CCA40201478146130644FCCE85CE
:10DC1000568597C0FFFFE7804046B1B7A68513063B
:10DC200034FC97000000E780E0E6933415002A8971
:10DC300086048DBF9385C504A5BF8327C9001397AC
:10DC40001400BA9783D5070063886501130544FC67
:10DC500097E0FFFFE780C003850445B71743FFFF48
:10DC6000E702E34379711C103EC4B7070F003EC6BC
:10DC70001C103EC883C79500AA8A328593F7F70720
:10DC8000A384F500AE89328497E0FFFFE780000EA1
:10DC900093170501C187635AF0062A8A228597E007
:10DCA000FFFFE780A00C2A895285032B040097C050
:10DCB000FFFFE780000C39ED8357440081440544A1
:10DCC000F11793B71700A303F10083457100DA87BA
:10DCD0002287CA865286280097000000E780E0C8A5
:10DCE000014781463000CE85568597C0FFFFE7800B
:10DCF000C038A1679387D70348083ECC230A810028
:10DD000026CE97F0FFFFE78040DD45611743FFFF18
:10DD10006700633CA2851306710097000000E7804E
:10DD200060D7AA84094455D13544E30055FB4A85A0
:10DD300097F0FFFFE78000450D4441D9014497D09B
:10DD4000FFFFE7806002634DA400C16B0144FD1B2F
:10DD500097D0FFFFE7804001634EA4001544B5B79C
:10DD6000DC4413171400BA9783D707006383270393
:10DD70000504F1B7D84493171400BA9703D70700E6
:10DD8000631B770123902701268597A00000E78079
:10DD900080DB01441DBF050465BF1743FFFFE70299
:10DDA000E33083C7950041112A8A93F7F707A384CC
:10DDB000F50032852E89328497E0FFFFE78000FB73
:10DDC00093170501C1876353F006AA89228597E05E
:10DDD000FFFFE780A0F92311A1004E85832A0400EC
:10DDE00097C0FFFFE780E0F839E58357440085449A
:10DDF0000144F11793B71700A300F1000348110085
:10DE000003572100D6875285CE862686CA8597F08D
:10DE1000FFFFE7806006A167F10748003EC42302C8
:10DE2000910022C697F0FFFFE78020CB4101174306
:10DE3000FFFF6700E32AA285130611009700000088
:10DE4000E78040C52A84894455D98357210011674A
:10DE50008544BA97C2071167C1831307F7EFE36FD1
:10DE6000F7F89787FF1F9387A7069C4381CB8545CB
:10DE70001305210097500000E7802075835521008D
:10DE80002285814497C0FFFFE78040E525D9231014
:10DE90000500228597A00000E78040CD85B7174395
:10DEA000FFFFE702C31F83C7950041112A8B93F739
:10DEB000F707A384F50032852E8A328497E0FFFFAE
:10DEC000E780C0EA93170501C1876351F006AA8A6B
:10DED000228597E0FFFFE78060E92A895685832B3A
:10DEE000040097C0FFFFE780C0E831E58357440096
:10DEF00081440544F11793B71700A301F1000348CB
:10DF00003100DE875A854A87D6862286D28597F0E9
:10DF1000FFFFE78060F6A167ED0748003EC42302DB
:10DF2000810026C697F0FFFFE78020BB4101174321
:10DF3000FFFF6700431AA285130631009700000017
:10DF4000E78040B5AA8409445DD99167CA97C207A2
:10DF50001167C1831307F7EF0544E362F7FACA8537
:10DF600097C0FFFFE78080D7014451F9814997D0DE
:10DF7000FFFFE78060E063DBA900984893971900F2
:10DF8000BA9703D7070005EF2390270197D0FFFF2B
:10DF9000E78080DE1544E384A9F6268597A000007B
:10DFA000E780C0BC9787FF1F938787F29C4301449B
:10DFB000B9D74A8597500000E780C05889B78509CE
:10DFC0007DB71743FFFFE702630E79713E847C083B
:10DFD0003EC82E8AB7071400A1653ECAE5057C0835
:10DFE000AA89080836C4428932C6BA8AC6843ECC99
:10DFF00097C0FFFFE78000E3CA85080897E0FFFFAE
:10E00000E78000C732460808B28597E0FFFFE78047
:10E0100020C8A246630A09049D45080897E0FFFF4F
:10E02000E780C0BE1D4681459740FFFFE780A00CFA
:10E0300063890A089145080897E0FFFFE78000BD63
:10E040001146A68597000100E780607A1008014715
:10E050008146D2854E8597C0FFFFE780000245616B
:10E060001743FFFF6700C307B685080897E0FFFF67
:10E07000E78000C21C400808D8439355C701858932
:10E0800012075183B205D98D97E0FFFFE78040C0AA
:10E090001C40080883C5870097E0FFFFE78040BD6C
:10E0A0001C40080883C5A70097E0FFFFE78040BC3D
:10E0B0001C40080883C5970097E0FFFFE78040BB3E
:10E0C00085BF8945080897E0FFFFE78020B483C734
:10E0D00004002300F50083C71400A300F500BDB7BA
:10E0E0001743FFFFE70283FC83C795004111AA890C
:10E0F00093F7F707A384F5003285AE84328497E066
:10E10000FFFFE780A0C693170501C187635DF00498
:10E110002A89032A040097C0FFFFE78080C519E918
:10E12000835744000548F11793B71700A307F10080
:10E13000814631A81306F100A28597000000E78010
:10E1400060951DC51C459DC783D647000148034700
:10E15000F10093078500D2884A86A6854E859700F0
:10E160000000E78040E641011743FFFF670043F7E7
:10E1700009487DBF1D486DBF1743FFFFE70203F34A
:10E1800065715C083EC4B7077B013EC65C083EC8AB
:10E1900083C795002A8A328593F7F707A384F50091
:10E1A000AE8997E0FFFFE78040BA8357E100E1C7FF
:10E1B0008945280097C0FFFFE780C0C68145280039
:10E1C00097E0FFFFE780C0AA97C0FFFFE780A0CCE1
:10E1D0009787FF1F9387C7079C431784FF1F03443C
:10E1E000A4B0AA843334800099C3136424009787B1
:10E1F000FF1F9387A7B79C4399C313644400978775
:10E20000FF1F9387E7CC9C4399C31364840083D595
:10E2100004002800014997E0FFFFE78060A783D54D
:10E220002400280097E0FFFFE78080A683D5440004
:10E23000280097E0FFFFE780A0A597D0FFFFE780C9
:10E24000A0AE93150501C181280097E0FFFFE7808C
:10E2500020A4A285280097E0FFFFE78060A39C44EC
:10E260006360F902014781463000CE85528597C030
:10E27000FFFFE78080E059611743FFFF670043E637
:10E28000DC441314490028003E9497E0FFFFE78028
:10E290006096834744000347540089070607BA97EE
:10E2A0008607E36AF5FC835524002800814A97E03D
:10E2B000FFFFE780E09D83454400280097E0FFFFD3
:10E2C000E780009B83455400280097E0FFFFE7802C
:10E2D000209A8347440063C9FA00814A8347540067
:10E2E00063C1FA020509A5BF1C4413975A00280010
:10E2F000BA9783D50700850A97E0FFFFE78040992A
:10E30000C9BF032BC40093975A0028003E9B835536
:10E310002B00850A97E0FFFFE780809783550B006D
:10E32000280097E0FFFFE780A0964DBF1743FFFF4F
:10E33000E70263D95C4993E717005CC997A0000026
:10E34000E78020B61743FFFF670023DA1743FFFF7C
:10E35000E70263D72E84814597F0FFFFE780C0E78F
:10E3600005C583570500FD172310F50009C4835721
:10E3700025002310F40097000000E78060FB0145B2
:10E380001743FFFF670063D631457DD82310040093
:10E39000C5BF1743FFFFE70263D183C79500411153
:10E3A0002A8A93F7F707A384F50032852E893284F1
:10E3B00097E0FFFFE780809B93170501C1876356B5
:10E3C000F006AA89C145228597E0FFFFE780A0807B
:10E3D0002A8B4E85832A040097C0FFFFE78060994F
:10E3E00031E983574400231101000544F11793B725
:10E3F0001700A300F10081440348110003572100D6
:10E40000D6875285CE862286CA8597F0FFFFE780A1
:10E41000A0A6A1679387170248003EC4230281008B
:10E4200026C697E0FFFFE780406B41011743FFFFDF
:10E43000670003CB13061100A28597F0FFFFE7806A
:10E440006065AA8409E523110100094475B79305A5
:10E4500021005A8597000000E78080EF8357210054
:10E460002A84D9DB9787FF1F938787A69C4381CB9C
:10E4700085451305210097500000E780001583555E
:10E4800021002685314497C0FFFFE78020852DD5E8
:10E4900023100500268597900000E780206D014439
:10E4A000A1BF1743FFFFE70203C241112E896C0091
:10E4B000AA8402C697F0FFFFE78000D20DC1035780
:10E4C000050005072310E50097000000E78040E6FF
:10E4D00081473E8541011743FFFF670003C1324773
:10E4E000954765DBCA85268597300000E780400D9B
:10E4F000C147E34005FE3244854741462310F400FE
:10E5000083570900A685130544002311F4009700E2
:10E510000100E780C02D228545BF1743FFFFE702BA
:10E52000E3B883C795004111AA8A93F7F707A3843C
:10E53000F5003285AE89328497E0FFFFE7800083E3
:10E5400093170501C1876356F0062A8AC1452285C3
:10E5500097D0FFFFE7802068AA845285032B040030
:10E5600097C0FFFFE780E08031E983574400231123
:10E5700001008544F11793B71700A300F10001448F
:10E580000348110003572100DA875685D286268674
:10E59000CE8597F0FFFFE780208EA1679387070263
:10E5A00048003EC42302910022C697E0FFFFE780A7
:10E5B000C05241011743FFFF670083B2A2851306D3
:10E5C000110097F0FFFFE780E04C2A8409E5231152
:10E5D0000100894475B72685930521009700000046
:10E5E000E78060ECAA8449FD83552100228597B01D
:10E5F000FFFFE780A06E49F5014997C0FFFFE78064
:10E60000A077635DA900184893171900BA9703D73C
:10E6100007000DEF035721002390E70097C0FFFF8D
:10E62000E7808075630625039787FF1F9387478AD6
:10E630009C4399C70355210097500000E78080F064
:10E64000228597900000E78060521DBF050975B7CD
:10E6500095443DB705C19307F00F630FF500C5471B
:10E66000630CF5009307F5FF05453315F5004205EA
:10E67000418182800145828041657D158280B9E9B2
:10E680001743FFFFE70223A40345060332849700E4
:10E690000000E78060FC9305803EB305B502C2052B
:10E6A000C18181CD0357E402854763F8E700130574
:10E6B000040197E00000E78020428357E4024167AD
:10E6C0007D176385E700FD172317F4021743FFFF4B
:10E6D0006700A3A182801743FFFFE702439C00422B
:10E6E00083C79500444D0349140093F7F707A384AB
:10E6F000F50083470400220911673369F900A16717
:10E70000B347F90041112A8BAE8A63ECE70E8347C9
:10E7100024001307C00EB91793F7F70F6373F710B0
:10E7200003473400C14763EEE70E834744001307F5
:10E73000E00793C707086371F70C83498400834798
:10E740007400A209B3E9F900856763F7F90A034A7F
:10E750006400834754004E85220A336AFA009750BA
:10E760000000E780403B61C123962403834B3400C3
:10E77000137AFA00239A34032388740323994403F9
:10E7800093890401631C090023A604022398040250
:10E790004E8597E00000E78060363DA003492400E5
:10E7A0004A8597000000E78020EB2397A402834767
:10E7B00044004E85A388F402E38D0BFCE30B09FCB7
:10E7C00097E00000E780202F97900000E78000731B
:10E7D00081460146D6855A8597E0FFFFE7800058BD
:10E7E000A167938797033EC423020100480002C635
:10E7F00097E0FFFFE780602E41011743FFFF6700AE
:10E80000838D8544A2862686D6855A8597E0FFFFAC
:10E81000E780C054A167938797033EC42302910009
:10E82000F1B7BD44C5B79144F1BF1743FFFFE702FD
:10E83000E38701111C08404D3EC2B7070F003EC4DC
:10E840001C083EC62A89AE8997C0FFFFE780A0DA80
:10E85000585C1C5C6346B70E6394E50063E2A70E48
:10E860003385A740B3B7A700B305B7401306803E72
:10E8700081469D8D97000100E78080B793140501C4
:10E88000C180A1659385C503480097B0FFFFE7806D
:10E8900060598145480097D0FFFFE780603D835570
:10E8A0000404480097D0FFFFE780803E835524048E
:10E8B000480097D0FFFFE780A03D814589CCC16724
:10E8C000FD179305F00F6388F4002685975000002C
:10E8D000E780E0E0AA85480097D0FFFFE780403955
:10E8E00003554404814501CDC167FD179305F00F21
:10E8F0006307F50097500000E78060DEAA854800B6
:10E9000097D0FFFFE780C03683456404480097D066
:10E91000FFFFE780E03583457404480097D0FFFF90
:10E92000E7800035500001478146CE854A8597B083
:10E93000FFFFE780807405611733FFFF6700437AAC
:10E94000814481B71733FFFFE702E37783C7950060
:10E9500093F7F707A384F50097000000E78020ED08
:10E960001733FFFF670063781733FFFFE702037475
:10E9700083C795004111404D93F7F707A384F50035
:10E980002A8A3285B284AE8997D0FFFFE780003EA5
:10E990002A8B268597D0FFFFE780403D2A89268570
:10E9A00097D0FFFFE780603A93170B0163CA070215
:10E9B000E177CA97C207C183116763E3E702930750
:10E9C0000910C207C1831307B00F637BF7009317C9
:10E9D0000901C187AA8A634AF000C54763FE57014F
:10E9E00041011733FFFF6700A36F97B0FFFFE78078
:10E9F000C028E31725FFD5B763080B026306090299
:10EA0000814463890A02B7077F002310640523113C
:10EA100024057CC0568597000000E780E0C393047E
:10EA2000803EB304950239A0B7077F002320040479
:10EA30007CC081440355240497E00000E780A0A334
:10EA4000A1C497C0FFFFE78000BB269593D7F44190
:10EA500033379500AE97BA9708DC5CDCCE855285DB
:10EA600097000000E780A0DC99E023220404A1675E
:10EA70009387B70348003EC42302010002C697E013
:10EA8000FFFFE7808005A9BF814701481CDC232EDA
:10EA90000403E9B71733FFFFE702E36297C0FFFF04
:10EAA000E780C037E1473305F502914597500000F4
:10EAB000E78000C5E55711C59777FF1F23A4A7225C
:10EAC00081473E851733FFFF67002362854717772D
:10EAD000FF1F230BF72082801733FFFFE702A35E9F
:10EAE0009777FF1F9387C71F80433DC08357040458
:10EAF0006390A70683572404639CB7043689B284C5
:10EB000097C0FFFFE78020AF5C5C63C3B7046395E9
:10EB1000B7001C5C63EEA7028347640463F3F40050
:10EB2000A6872303F4048347740463F39700A6873E
:10EB3000A303F4048357440441677D176385E7000A
:10EB400085072312F4043C4481C7CA852685829731
:10EB50001733FFFF670063599777FF1F93874718A5
:10EB60009C43014599C303C5870082801733FFFF8B
:10EB7000E70263550111B70707003EC683C795003A
:10EB8000584D0AC493F7F7070AC8A384F5002A89E9
:10EB9000AE8411CB1C4283C707002304F700979073
:10EBA0000000E7800034216493055402280097B0E8
:10EBB000FFFFE780202797000000E78020FAAA8562
:10EBC000280097D0FFFFE780A00A30000147814668
:10EBD000A6854A8597B0FFFFE780204A13044402C8
:10EBE000480822CC230A010002CE97E0FFFFE7800D
:10EBF000C0EE05611733FFFF6700234F1733FFFF98
:10EC0000E702634C01117C003ECAB70707003ECC07
:10EC10007C003ECE83C795002E84AA8493F7F70725
:10EC2000A384F500A16593855502480897B0FFFFBE
:10EC3000E780401F97000000E78040F2AA8548085F
:10EC400097D0FFFFE780C002500801478146A285A8
:10EC5000268597B0FFFFE780404205611733FFFF2D
:10EC60006700A3489777FF1F938787079C43094551
:10EC700099C303C5970082809777FF1F9387470644
:10EC80009C43094599C303C5D70082809777FF1F2E
:10EC9000938707059C43014599C303C5A70082805C
:10ECA0001733FFFFE70283400111B70708003EC694
:10ECB00083C79500404D0AC493F7F7070AC8A38499
:10ECC000F5002A89AE8429C41442854703C706008B
:10ECD00063E0E70A83479400094681496380C702DD
:10ECE000B307F740A304E400B339F00083C716006C
:10ECF0002305F40097900000E780A01E035724032B
:10ED0000058B19C76386090097D00000E78000E9EA
:10ED1000216493058402280097B0FFFFE7808010EC
:10ED200097000000E78040F4AA85280097D0FFFFF5
:10ED3000E78000F497000000E78080F5AA852800AE
:10ED400097D0FFFFE780C0F2014781463000A685DB
:10ED50004A8597B0FFFFE7804032130474024808E9
:10ED600022CC230A010002CE97E0FFFFE780E0D625
:10ED700005611733FFFF6700A3361733FFFFE70274
:10ED8000833401117C003ECAB70708003ECC7C00EA
:10ED90003ECE83C795002E84AA8493F7F707A384F9
:10EDA000F500A16593858502480897B0FFFFE780CD
:10EDB000600797000000E78020EBAA85480897D0FD
:10EDC000FFFFE780E0EA97000000E78060ECAA859B
:10EDD000480897D0FFFFE780A0E950080147814627
:10EDE000A285268597B0FFFFE780202905611733AC
:10EDF000FFFF6700832F9777FF1F938767EE9C4382
:10EE0000014599C303C5B70082801733FFFFE702AE
:10EE1000832B0111B70707003EC683C79500404DFD
:10EE20000AC493F7F7070AC8A384F5002A89AE84B9
:10EE300005C81C42054783C707006368F7060347F8
:10EE4000B400630FF700A305F40097900000E7807B
:10EE500040098347B400B9CF97D0FFFFE78040BE99
:10EE600021649305B400280097B0FFFFE78080FB82
:10EE700097000000E78060F8AA85280097D0FFFF80
:10EE8000E78000DF014781463000A6854A8597B0BC
:10EE9000FFFFE780801E2904480822CC230A0100D6
:10EEA00002CE97E0FFFFE78040C305611733FFFF05
:10EEB0006700A32397D0FFFFE78020BF55B7173324
:10EEC000FFFFE702432001117C003ECAB70707009D
:10EED0003ECC7C003ECE83C795002E84AA8493F757
:10EEE000F707A384F500A165AD05480897B0FFFFBB
:10EEF000E78040F397000000E78020F0AA854808EB
:10EF000097D0FFFFE780C0D6500801478146A28511
:10EF1000268597B0FFFFE780401605611733FFFF96
:10EF20006700A31C9777FF1F938787DB9C430945E6
:10EF300099C303C5C70082801733FFFFE702A318F8
:10EF400001117C00AE843ECAA165B70707002A8480
:10EF50003ECCD1057C0048083ECE97B0FFFFE7804D
:10EF600060EC97000000E78020FCAA85480897D055
:10EF7000FFFFE780E0CF500801478146A685228544
:10EF800097B0FFFFE780600F05611733FFFF670051
:10EF9000C3151733FFFFE702031383C7950093F7E9
:10EFA000F707A384F50097000000E78020F91733E6
:10EFB000FFFF670083131733FFFFE702230F83C7A9
:10EFC00095000329C501411193F7F707A384F500C4
:10EFD0001C4283C90700854763E637079777FF1F01
:10EFE000938707279C432E84AA8485CF970000002F
:10EFF000E78080F389476306F502630409028347CB
:10F00000C900638037032306390197900000E78029
:10F0100040ED83572903898B89C797D00000E7808B
:10F02000E0B72685A28597000000E78020F1A16760
:10F03000CD0748003EC42302010002C697E0FFFF4F
:10F04000E780A0A941011733FFFF670063099777A5
:10F05000FF1F9387E7C89C431D4599C303C5E7007D
:10F0600082801733FFFFE70203060111B70707008D
:10F070003EC683C79500584D0AC493F7F7070AC8E0
:10F08000A384F5002A89AE8415C71C4283C70700F4
:10F0900093968701E18663C4060685466381D70699
:10F0A0008346E7006388F6002307F7009790000087
:10F0B000E78020E321649305E400280097B0FFFF78
:10F0C000E78040D697000000E780A0F8AA852800D6
:10F0D00097D0FFFFE780C0B9014781463000A68581
:10F0E0004A8597B0FFFFE78040F93504480822CCF5
:10F0F000230A010002CE97E0FFFFE780009E056132
:10F100001733FFFF670063FE1733FFFFE702A3FB20
:10F1100001117C003ECAB70707003ECC7C003ECE02
:10F1200083C795002E84AA8493F7F707A384F5007C
:10F13000A165B905480897B0FFFFE780A0CE97000A
:10F140000000E78000F1AA85480897D0FFFFE7801C
:10F1500020B2500801478146A285268597B0FFFF5F
:10F16000E780A0F105611733FFFF670003F817334D
:10F17000FFFFE702A3F3AA8401441779FF1F1309D5
:10F1800069B6E14997C0FFFFE78040C96344A40026
:10F19000014519A833053403832709003E95835799
:10F1A00025006397970011051733FFFF670043F3AE
:10F1B0000504C9BF032E8500630A0E121773FF1FD3
:10F1C000130303D103230300631503002943639052
:10F1D000061203234E01631503001D4363990710B4
:10F1E0001733FFFFE702A3EBC689428A3E89BA8A3A
:10F1F000B684328BAE8B2A84B5E103554E0019E5F7
:10F2000001431A851733FFFF6700E3ECA167A98F5D
:10F21000116763FBE70097000000E78080F58145F8
:10F2200097F0FFFFE780C0120844B70700E058419D
:10F23000F98F18455CC1B707001FF98F1CC55C49E1
:10F2400091C7610597E00000E780408BE38A09FAE7
:10F25000228597900000E78060C65DB7328597C031
:10F260000000E78040430D4349DD1C44116703D58E
:10F270004700A167A98F63FBE70097000000E780C4
:10F2800040EF814597F0FFFFE780800C0323840067
:10F2900093164B01D1828347B300035663008588E0
:10F2A000FD8BA305F300FD777D8E558EFD76FD1653
:10F2B000B204F18E83274301C58E231273012313F9
:10F2C000D3002304530123052301A3044301BDDF1D
:10F2D000228597B0FFFFE78020CDAA850844B5D1ED
:10F2E000610597D00000E780207F8DB71D431A8508
:10F2F00082801733FFFFE70263DB0569AA84AE89CA
:10F30000328A0144FD5A7D1997C0FFFFE780C0A5EE
:10F310006347A40001451733FFFF670063DCD8444F
:10F3200093171400BA9703D70700631F370323907E
:10F33000570163070A00268597900000E780A080A8
:10F340009C449DC383D76700B3F72701639E3701B1
:10F35000D28801488147014781460146814526857B
:10F3600097000000E78040E5050479BF1733FFFFF1
:10F37000E702C3D379711C103EC4B7070F003EC625
:10F380001C103EC883C79500AA8A328593F7F707F9
:10F39000A384F5002E89328497D0FFFFE780009D7B
:10F3A00093170501C187635AF006AA89228597D071
:10F3B000FFFFE780A09B2A8A4E85032B040097B0AD
:10F3C000FFFFE780009B39ED8357440081440544EB
:10F3D000F11793B71700A303F10083457100DA8793
:10F3E0002287D2864E86280097E0FFFFE780E0570D
:10F3F000014781463000CA85568597B0FFFFE780F8
:10F40000C0C7A1679387F70348083ECC230A810051
:10F4100026CE97D0FFFFE780406C45611733FFFF92
:10F42000670003CCA2851306710097E0FFFFE78019
:10F430006066AA84094455D1528597E0FFFFE780B2
:10F4400060D40D4459D90546D28526859700000021
:10F45000E78060EA2A8451B71733FFFFE702A3C6AB
:10F46000835507000346270041112A842E8532C6A2
:10F470002EC497E0FFFFE780E0D001C93246A245E5
:10F48000228597000000E78000E741011733FFFF66
:10F490006700A3C51733FFFFE70263C083C795006A
:10F4A0004111AA8A93F7F707A384F5003285AE8944
:10F4B000328497D0FFFFE780608B93170501C187E7
:10F4C0006357F00AC1452A8A228597C0FFFFE7806B
:10F4D00080702A8D228597D0FFFFE78020892A89B6
:10F4E000228597D0FFFFE7804086930705F893F7C2
:10F4F000F70F1307E007AA8B637BF706228597D0E7
:10F50000FFFFE78080842A8C228597D0FFFFE78069
:10F51000C083AA8C5285032B040097B0FFFFE780BD
:10F52000408539E983574400231101008144F117D4
:10F5300093B71700A300F100054403471100835659
:10F540002100938784005685DA8822885286CE85EA
:10F5500097F0FFFFE78020A7A167E90748003EC4B6
:10F560002302810026C697D0FFFFE78000574101A4
:10F570001733FFFF670023B613061100A28597E03B
:10F58000FFFFE7802051AA8409E523110100094407
:10F590006DB7930521006A8597F0FFFFE780A0F023
:10F5A0002A8441FD835521009356C9001316490151
:10F5B00085486688E2875E87858A5182268597001E
:10F5C0000000E78060BF2A848DBF1733FFFFE7028A
:10F5D00003AD83C7950041112A8B93F7F707A384E6
:10F5E000F5003285AE89328497C0FFFFE78000784E
:10F5F00093170501C1876352F00A2A8A228597C0B2
:10F60000FFFFE780A076AA8A228597C0FFFFE780E8
:10F61000E0752A89228597C0FFFFE7800073930772
:10F6200005F893F7F70F1307E0072A8C6377F706BF
:10F63000228597C0FFFFE7804071AA8C228597C082
:10F64000FFFFE78080702A8D5285832B040097A0EE
:10F65000FFFFE780007239E5835744008544014489
:10F66000F11793B71700A301F10003473100930787
:10F6700084005A85DE882688D6865286CE8597F005
:10F68000FFFFE78040948D4748003EC4230291006D
:10F6900022C697D0FFFFE780404441011733FFFFA8
:10F6A000670063A3A2851306310097E0FFFFE780A0
:10F6B000603E2A84894455D99356C90013164901DE
:10F6C00085486A88E6876287858A5182D685970051
:10F6D0000000E78060AEAA8449BF1733FFFFE7024E
:10F6E000E39C2A8981440144617A916A176BFF1F68
:10F6F000130B0B7E97B0FFFFE780006863C7A40081
:10F7000022851733FFFF6700A39D83270900939984
:10F710001400CE9703D50700330745014207418304
:10F720006364570305C103270B0019C785453E8550
:10F7300097400000E78060E9832709000504CE9721
:10F740002390070085047DB797000000E78060A242
:10F75000832709000504CE972390070065D58145CE
:10F7600097F0FFFFE780C0BEF1BF1733FFFFE7024E
:10F77000E39383C7950041112A8A93F7F707A3847F
:10F78000F50032852E89328497C0FFFFE780005E46
:10F7900093170501C187635AF004AA89832A0400DC
:10F7A00097A0FFFFE780E05C31E583574400854484
:10F7B0000144F11793B71700A301F100034831008A
:10F7C000D68752850147CE862686CA8597D0FFFF09
:10F7D000E780806AA167F50748003EC423029100D4
:10F7E00022C697D0FFFFE780402F41011733FFFF6C
:10F7F0006700038FA2851306310097E0FFFFE780C3
:10F8000060292A8489445DD99767FF1F9387476CD5
:10F810009C4381CF044997B0FFFFE780E055AA855C
:10F82000268597400000E78040DA13050401970021
:10F830000000E780C0EA228597800000E78000335F
:10F840008144ADBF1733FFFFE702638583C795008F
:10F850004111AA8A93F7F707A384F5003285AE8990
:10F8600032842311010097C0FFFFE78020509317D7
:10F870000501C1876354F0062A8AC145228597C0D5
:10F88000FFFFE7804035AA8B5285032B040097A029
:10F89000FFFFE780004E21E983574400854401447F
:10F8A000F11793B71700A300F100034811000357A5
:10F8B0002100DA875685D2862686CE8597D0FFFF2F
:10F8C000E780805BA1679387270248003EC423023C
:10F8D000910022C697D0FFFFE78020204101172327
:10F8E000FFFF6700437FA2851306110097E0FFFF2B
:10F8F000E780401A2A8489444DD99767FF1F938770
:10F90000275D98433E8901CF044997B0FFFFE78008
:10F91000A046AA85268597400000E78000CB130506
:10F92000040197000000E78080DB97B0FFFFE780CD
:10F93000A04495443DD9930521005E8597F0FFFFD3
:10F94000E78060B6AA8435F11C4803572100228560
:10F950002390E70097800000E7804021832709007B
:10F96000A9D70355210097400000E780A0BD35BF0F
:10F970001723FFFFE702A37283C795004111AA8AEC
:10F9800093F7F707A384F5003285AE89328497C0D8
:10F99000FFFFE780A03D93170501C1876351F00683
:10F9A0002A8A228597C0FFFFE780403C2A8952853A
:10F9B000032B040097A0FFFFE780A03B31E58357AE
:10F9C000440085440144F11793B71700A301F100E7
:10F9D00003483100DA8756854A87D2862686CE8547
:10F9E00097D0FFFFE7804049A167F90748003EC470
:10F9F0002302910022C697D0FFFFE780000E41014D
:10FA00001723FFFF6700236DA2851306310097E0DF
:10FA1000FFFFE78020082A8489445DD99167CA974F
:10FA2000C2071167C1831307F7EF8544E362F7FA52
:10FA30009767FF1F9387C7499843BE8B01CF04493F
:10FA400097B0FFFFE7804033AA85268597400000E6
:10FA5000E780A0B71305040197000000E78020C8E5
:10FA600097B0FFFFE780403195443DD11C48228587
:10FA700081442390270197800000E780200F83A70F
:10FA80000B00B9D74A8597400000E780A0AB89B743
:10FA90001723FFFFE70223632A844105B2849700FE
:10FAA0000000E780C0C311C5228597800000E78071
:10FAB000E00B81460146A685228597800000E780FD
:10FAC000C04E1C4C89C7DC4799C3228582971723F7
:10FAD000FFFF670083619767FF1F938767209C4341
:10FAE000014599C31385070182809767FF1F93879C
:10FAF000271F884382801723FFFFE702C35C931709
:10FB0000C600DD8DC2054111C1812A8432C697C06D
:10FB1000FFFFE780E0173246228511829375F60FCA
:10FB200097C0FFFFE780C01441011723FFFF670064
:10FB3000C35B1723FFFFE702635779713C083ED28E
:10FB4000B7070C003ED43C083ED683C79500AE8470
:10FB50002A8993F7F707A384F500A16593853504F7
:10FB6000481097A0FFFFE780E02BC165FD15014419
:10FB7000176AFF1F130A4A37930A400EAE892E8B6D
:10FB80002EC697B0FFFFE78020224205931704019D
:10FB90004181C183B24563E9A702C167FD1763874D
:10FBA000F500481097C0FFFFE780800E5010014716
:10FBB0008146A6854A8597A0FFFFE780004C4561F6
:10FBC0001723FFFF6700C3513307540383270A0B32
:10FBD000BA9703D6C701630A3601638A3501481014
:10FBE00097000000E78060F1DA85050451BFB28517
:10FBF000EDBF1723FFFFE702834A79717C083EC8F7
:10FC0000B70711003ECA7C083ECC83C79500AA897D
:10FC1000328593F7F707A384F5002E8997C0FFFF7D
:10FC2000E780C01485676378F504A165AA84890517
:10FC3000080897A0FFFFE780E01E26859740000098
:10FC4000E78060ED133415000A04A285080897C008
:10FC5000FFFFE780E001A685080897C0FFFFE78067
:10FC6000200325CC014781461008CA854E8597A000
:10FC7000FFFFE780804045611723FFFF6700A34532
:10FC8000B30754030327CA0ABA9703D70700631CB4
:10FC9000970003D6270063806505080897000000D9
:10FCA000E780A0E5DE8505042EC697B0FFFFE7805C
:10FCB000A0104205931704014181C183B245E3E1DD
:10FCC000A7FCC167FD17E38FF5F8080897C0FFFF91
:10FCD000E78000FC41BFB285F9B7C165FD1501445D
:10FCE000176AFF1F130A4A20930A80022E8BAE8BDD
:10FCF00065BF1723FFFFE702033D18418347170045
:10FD000083460700A207D58FD207D1832390F50041
:10FD100083472700034717008D45A207D98F91839A
:10FD20002310F60097C0FFFFE780A0E91723FFFF2D
:10FD30006700A33B1723FFFFE7024337C164014479
:10FD40001769FF1F1309491A93098002FD1497B020
:10FD5000FFFFE78060066347A40001451723FFFF0C
:10FD600067000338330534038327C90A3E95835758
:10FD70000500E38597FE0504D9BF1723FFFFE702BF
:10FD8000E3322A8AAE89B284B68A97400000E780BF
:10FD900080D819E591473E851723FFFF670043345C
:10FDA0002A894E8597C00000E780E08E2A84638E02
:10FDB0000A048D476DD103570500C547E31D47FD74
:10FDC0000347F9018546AD47E317D7FC8347450054
:10FDD00081CF4146A6855D0597F00000E780C09E73
:10FDE000814755D9AD4745BF130965012302E50099
:10FDF000CA85268597100000E780606231C1A5475B
:10FE0000E38B0AF82302040079B705C18357050084
:10FE1000E39247F94146A685190597F00000E7806F
:10FE2000A09A81472DD99947BDB74E85970000000C
:10FE3000E78080F02A84954739DD130955004DBFCE
:10FE40004146A685231044012311340113051900EE
:10FE500097F00000E780A099228597800000E78056
:10FE6000A0EA81470DBF1723FFFFE702C325797181
:10FE70007C003ECCB7070A003ECE7C003ED083C754
:10FE80009500B2842E8493F7F707A384F500130638
:10FE9000A1002A892C00268597000000E780A0E5B4
:10FEA000A16528088D0597A0FFFFE780A0F7904087
:10FEB0008355A10003558100854697000000E78027
:10FEC00000ECAA84AA85280897C0FFFFE78040DAE3
:10FED0000356A10083558100280897000000E780A1
:10FEE000C0C1300801478146A2854A8597A0FFFF1F
:10FEF000E780A018854748103ED42302910202D61D
:10FF000097D0FFFFE78060BD45611723FFFF6700C3
:10FF1000C31D1723FFFFE702031B79717C003ECC52
:10FF2000B7070A003ECE7C003ED083C79500B2845E
:10FF30002E8493F7F707A384F5001306A1002A89FE
:10FF40002C00268597000000E780E0DAA1652808EC
:10FF50008D0597A0FFFFE780E0EC90408355A1005E
:10FF600003558100814697000000E78040E1AA84A4
:10FF7000AA85280897C0FFFFE78080CF0356A1001D
:10FF800083558100280897000000E78000B73008FB
:10FF900001478146A2854A8597A0FFFFE780E00DD3
:10FFA00048102302910202D402D697D0FFFFE780C7
:10FFB000C0B245611723FFFF670023131723FFFF1C
:10FFC000E702631097000000E78060DB1723FFFF64
:10FFD0006700A3119767FF1F9387C7D0884382806C
:10FFE0001723FFFFE702230E835725004111AE843C
:10FFF0002A842307B10017F5FFFF130525466C007F
:020000040001F9
:100000002316F10097A0FFFFE780204991C42285C5
:1000100097800000E780E0D6FD572310F400130618
:1000200020028145130554009720FFFFE780A00CB4
:1000300041011723FFFF6700430B1723FFFFE70270
:10004000E30679717C003ECCB7070A003ECE7C0007
:100050003ED083C79500AA89AE8493F7F70732850F
:10006000A384F5001306A1002C0097000000E78090
:1000700080C803558100114497400000E780A0A983
:1000800015C50355A100014497B00000E780A060AA
:1000900011CD035705008357810045446318F700CD
:1000A000854597000000E780E0F30144216993054E
:1000B0003900280897A0FFFFE780C0D6A28528084E
:1000C00097C0FFFFE780C0BA0356A10083558100A7
:1000D000280897000000E78040A2300801478146C9
:1000E000A6854E8597A0FFFFE78020F948104AD4E7
:1000F0002302810202D697D0FFFFE780009E456170
:100100001723FFFF6700C3FD1723FFFFE70203FA72
:100110009767FF1F9387C7BC2A8488432E8915C51C
:10012000035745038357C4016311F70223260502D1
:1001300023180502410597D00000E780209C630644
:10014000090097800000E78060DB81449769FF1F0A
:10015000938989D9130A800297B0FFFFE780C0C551
:1001600063C4A4049767FF1F938747C09C4399C744
:100170000355C40197200000E780C0BD6307090054
:10018000228597800000E780C0A01306400E8145BD
:1001900022859720FFFFE78000F6FD57231EF4001D
:1001A0001723FFFF6700C3F33385440383A7C90AFE
:1001B0003E95035705008357C4016317F700CA85AE
:1001C00097000000E78000E2850479B71723FFFF5E
:1001D000E702C3ED83C795004111AA8993F7F7079A
:1001E000A384F5003285AE8497C0FFFFE78000B896
:1001F00085676378F5042A8997400000E780A0911D
:10020000014401CD83D7040031446388270185452B
:1002100097000000E78080EF01444E85A2864A8661
:10022000A68597D0FFFFE780A09CA167938717045E
:1002300048003EC42302810002C697D0FFFFE7803A
:10024000C08941011723FFFF670083E91723FFFFE0
:10025000E702C3E59767FF1F938787A8804329C4F8
:10026000014597C00000E780002181470148C16433
:100270001CDC232E0403232004041769FF1F130929
:10028000A9C601449309400EFD1497B0FFFFE78013
:10029000A0B1634FA400814517F5FFFF1305857FCB
:1002A00097A0FFFFE780601F1723FFFF670043E36E
:1002B000330534038327090B3E958357C5016387B4
:1002C0009700854597000000E78040E4050475BF6E
:1002D0009357050113D78700A380F50093170501F5
:1002E000C183A1832380E5002381F500A381A500BC
:1002F00082801723FFFFE70203DD2300050083C789
:100300001500A300F50083C725002301F50083C76E
:100310003500A301F50083C745002302F50083C71C
:100320005500A302F50083C7650093059500A3035C
:1003300005002303F5002304050032859700000023
:10034000E78040F91723FFFF670023DA1723FFFF39
:10035000E702C3D54111E9540DCD85CD93F9C5FF11
:100360002E842A89AA84338AA900B7EA0400631874
:100370009A020D88854411CCB7E704009C5F8297F0
:100380002AC622866C003305390197E00000E78019
:100390000046268541011723FFFF670063D483A72A
:1003A0008A039104829793170501C183A183A38EC9
:1003B000F4FE93570501238FF4FEA183238EA4FE40
:1003C000A38FF4FE6DB763E6D5021723FFFFE702A4
:1003D00083CFB28741113686BE8536C697E00000CE
:1003E000E780E040B246410136851723FFFF6700F2
:1003F000C3CF814636858280838705001387F50049
:100400003D05FD8793F77708834607007D1586062F
:10041000B58FA300F5006307B7007D17834717006A
:100420009D83DDB782801723FFFFE702C3C9B7E7CB
:10043000040083A7070932872A863A8582971335F5
:1004400015001723FFFF670043CA15C181478DC1FF
:100450001723FFFFE70223C7414697E00000E7802C
:10046000003985473E851723FFFF670003C8814792
:100470003E8582801DCD1723FFFFE702C3C441469E
:1004800081452A849720FFFFE780E0C641468145E9
:10049000130504039720FFFFE780E0C50147C1670C
:1004A0002322040438C87CC805451723FFFF6700D2
:1004B000C3C30145828081473DCDB5CD1723FFFFE2
:1004C000E70263C0B2842E891306800581452A8421
:1004D0009720FFFFE78020C2CA8524C426859700A5
:1004E0000000E780C0F64146814522859720FFFF46
:1004F000E78060C03044A285228597000000E78035
:10050000C0F293040401A285268597000000E780CD
:10051000E0EEA6851305040297000000E78000EED8
:10052000228597000000E78020F585473E85172348
:10053000FFFF670083BB3E8582801723FFFFE70232
:10054000E3B64111E9540DCD85CD93F9C5FF2E8455
:100550002A89AA84338AA900B7EA0400639844036D
:100560000D88814411CCB7E704009C5F82972AC6AE
:1005700022866C003305390197E00000E7802027D0
:10058000268541011723FFFF670083B583A78A03F0
:100590009104829793170501C183A183A38EF4FE72
:1005A00093570501238FF4FEA183238EA4FEA38F0E
:1005B000F4FE6DB765CD1723FFFFE70223AFB284CA
:1005C00011E605451723FFFF670083B12A842E89B2
:1005D0000145EDD93C487848B3E6E700E5D6938677
:1005E000F7FFB3B7F6007D17032A4404BA9734C85F
:1005F0007CC863050A06C14913050A03B38949414A
:100600002295637D3601B2862E86A685970000006E
:10061000E780A0DB7C40BE9464C065B7CE862E86A2
:10062000CE8597000000E78040DAC114D2944E993D
:1006300023220404A2879306040103C7070003C60C
:1006400007038507318FA38FE7FEE398F6FE30445A
:10065000A285228597000000E78020DD2699C14908
:100660003306994063EC9900A9DCA686A68513059C
:10067000040397000000E78040D579BF8147B306A7
:10068000F4003307F6000347070083C5060085071B
:100690002D8F2380E600E39437FF3044A285228526
:1006A00097000000E78060D8C1145DBF01458280DB
:1006B0000DC11723FFFFE70203A113068005814543
:1006C0009720FFFFE78020A305451723FFFF670062
:1006D000C3A101458280814749C5C1C51723FFFFDA
:1006E000E702639EFC4141462E84AA846399C704B5
:1006F00013860501A2878146C14503C7070003C5CC
:1007000007038507298F3305D600034505008506B5
:10071000298FA38FE7FEE392B6FE3044A28526859B
:1007200097000000E78060D0228597000000E780F6
:1007300060F885473E851723FFFF6700039B1385FD
:1007400007031D8E814522959720FFFFE780A09A21
:100750007C40130700F813060402A2972388E702DF
:1007600051BF3E8582801723FFFFE702C3956D715D
:100770002E84B284AA859010280036899700000044
:10078000E780A0D309EDD55725A050400C402800A4
:1007900097000000E78040E27DD5FD142104F5F4C8
:1007A0002C004A8597000000E78020F3814761DD37
:1007B0003E8551611723FFFF670023931723FFFF37
:1007C000E702639041112EC432C62C000546970003
:1007D0000000E78080F941011723FFFF6700E390E5
:1007E0001723FFFFE702238E01112A842EC602C8B9
:1007F00002CA02CC02CE97E00000E780402BB2464E
:100800002A86A285080897000000E78060FB137520
:10081000F50F05611723FFFF6700238D1723FFFFE7
:10082000E702638A7971B2872A8421462308B100DE
:1008300013051101BE853AC436C697E00000E78073
:1008400000FBB24693059101368597000000E780D2
:1008500060A82285141035460C0897000000E78038
:1008600020F62A84224701E921460C103A8597E0B8
:100870000000E780C0F7228545611723FFFF67006E
:10088000C3861723FFFFE70203847171AE84AA8534
:100890000A85328497000000E78060BB11C90A8690
:1008A000A685228597000000E78020B8814711E1E6
:1008B000C5473E854D611723FFFF6700038317136C
:1008C000FFFFE702437D1D712A8AB289BE84354647
:1008D0008547130511012E8CB68A3A8BC28C468D42
:1008E0002308F10097E00000E78060F010100C088A
:1008F0005285231F010097000000E780C0F82A847A
:100900003DEDA1476313FD089307900591E0E5478E
:100910003546E2851305110113990A012308F100F8
:100920001359090197E00000E78060EC1357890034
:1009300093978A00D98F90080C085285231FF100E5
:1009400097000000E78020F42A8415E9A1E493874A
:10095000FA0091831379F9003EC6631309004149F7
:10096000668B8144C14B854DB247639F970C6A8665
:100970008C0033855C0197E00000E78040E722852A
:1009800025611713FFFF6700C37493079004C9F034
:10099000A547BDBF834701050947C14B2308F100A7
:1009A00083471105A58FA308F10093872400814494
:1009B00063E1FB04014714083386E6008C08B38624
:1009C000E400BA95DA9683C6060083C505000507DC
:1009D000AD8E2300D600E390E7FE4147639CE70419
:1009E00090080C08528597000000E780C0E925D1E7
:1009F00081A0B3069B00BA871008B305F6009008E3
:100A00003E9603C506000346060085078506298E27
:100A10002380C500E39277FF998F90080C085285D8
:100A2000BE9497000000E78000E68947014749D15E
:100A30002A84B1B790083E96034606001408BE9675
:100A40002380C600850759BFB24785046387971482
:100A500081471808B306F70098083E973386F900D7
:100A600003470700034606008507318F2380E60011
:100A7000E39177FF90080C08528597000000E7800B
:100A800080E05DF53546E285130511012308B101CB
:100A900097E00000E780A0D5139704014183939766
:100AA00084002183D98F10180C085285231FF10070
:100AB00097000000E78020DD25FD8147101833876F
:100AC000F9003E960347070003460600B306FB0005
:100AD0008507318F2380E600E39277FF65A8180829
:100AE000B306F70098083E973386F90003470700DE
:100AF000034606008507318F2380E600E3E127FFE8
:100B0000CA87639E770990080C08528597000000F9
:100B1000E78060D711FD81479800B306F700900881
:100B200018103E973E9603470700034606008507C8
:100B3000318F2380E600E39177FF3546E285130588
:100B400011012308B10197E00000E78040CA139724
:100B500004014183939784002183D98F10180C08D6
:100B60005285231FF10097000000E780C0D1E311F8
:100B700005EC814710183387F9003E9603470700BC
:100B800003460600B306FB008507318F2380E6008D
:100B9000E3E227FFC109410BC1BB814785B7940838
:100BA000BE9683C6060018083E972300D700850727
:100BB00089BF638006321713FFFFE702C34D5971E7
:100BC0002A84BE89B28B85473546130511022E8BC8
:100BD000468C4289BA8A368A2300F10297E00000E7
:100BE000E780E0C010180C1022852317010297003F
:100BF0000000E78040C963180512A147631FFC0687
:100C00009307900563930900E5473546DA85130598
:100C1000110293140A012300F102C18097E0000041
:100C2000E780E0BC93178A0013D78400D98F90081F
:100C30000C1022852317F10297000000E780A0C462
:100C40007DE1639209049307FA00BD88918391E0E6
:100C5000C144C207C183DE8C814A3EC6414DB247C2
:100C600063E2FA0E6286B3854B01881097E00000BC
:100C7000E78080B54DC93D557DA093079004E3966C
:100C800009F8A54759B7834701050947C14C230017
:100C9000F10283471105B3C7F900A300F10293875E
:100CA0002900814963E1FC04814618103306D7000E
:100CB0008C083387D900B69556970347070083C53C
:100CC000050085062D8F2300E600E390D7FE4147FF
:100CD0006390E70690080C10228597000000E780DB
:100CE00080BA35D189A0B3863A01BA871010B3050E
:100CF000F60090083E9603C50600034606008507E9
:100D00008506298E2380C500E39297FF3387EC4048
:100D100090080C102285BA9997000000E780A0B6D1
:100D20008947014741D165611713FFFF6700633AA7
:100D300090083E96034606001410BE962380C60017
:100D4000850779B7B247850A93990A01939D8A006E
:100D500093D909016391570F85473546DA85130505
:100D600011022300F10293D9890097E00000E78087
:100D700000A8B3ED3D0190000C1022852317B103AC
:100D800097000000E78020B059FD8147A68963EAFB
:100D9000970626860C084A8597E00000E78020A584
:100DA00081471810B306F700100898083E973E9642
:100DB00003470700034606008507318F2380E600BE
:100DC000E3E197FE639FA90590080C102285970028
:100DD0000000E78040AB21F981479810B306F70087
:100DE000900818183E973E960347070003460600F2
:100DF0008507318F2380E600E391A7FF4109C10CED
:100E0000B9BD18089000B306F7003E963387FC0082
:100E100003470700034606008507318F2380E6005D
:100E2000B5B798084E97034707001C10CE9723804C
:100E3000E700850941BF85473546DA85130511026C
:100E40002300F10293D9890097E00000E780209AFF
:100E5000B3ED3D0190000C1022852317B1039700DC
:100E60000000E78040A2E31005EC814718089000DD
:100E7000B306F7003E963387FC000347070003469E
:100E800006008507318F2380E600E391A7FF4146E6
:100E90000C084A8597E00000E780609581471810AC
:100EA000B306F700100898083E973E9603470700E0
:100EB000034606008507318F2380E600E391A7FFF4
:100EC00090080C10228597000000E780C09B1DD57C
:100ED00099BD7D5582801713FFFFE702C31E0111E4
:100EE0002A842E8593055100328902C002C202C4B1
:100EF00002C69304740097F0FFFFE780A03D1D46F3
:100F0000A6851305910097E00000E780408E100849
:100F10008A854A8597000000E780E09619ED9307DF
:100F20001400180883C60700034607008507050755
:100F3000B18EA38FD7FEE397F4FE05611713FFFF71
:100F40006700A31A1713FFFFE70243162E848C4194
:100F50004111AA89838715003289914463D3070020
:100F6000A1449757FF1F9387A72E9C43A1C7C1CACF
:100F70008D472310F10083C725004A852301F10026
:100F800083C73500A301F10083C745002302F100A8
:100F900083C75500A302F10083C765009305910044
:100FA000A30301002303F1002304010097F0FFFFD6
:100FB000E78040320C404A860A8597F0FFFFE780C1
:100FC00080330328040083564400A6881D08814707
:100FD0000147E51642868A854E8597000000E78026
:100FE000408E2A8919E5A685228597B0FFFFE78004
:100FF000E0C14A8541011713FFFF6700630E4A866F
:101000000A8597F0FFFFE780002F6DB71713FFFFEA
:10101000E702C3092E848C414111AA8983871500F8
:101020003289914463D30700A1449757FF1F9387E8
:1010300027229C43A1C7C1C68D472310F10083C757
:1010400025004A852301F10083C73500A301F10083
:1010500083C745002302F10083C75500A302F100B6
:1010600083C7650093059100A30301002303F100EA
:101070002304010097F0FFFFE780C0250C404A865B
:101080000A8597F0FFFFE780002783564400032876
:1010900004008A85858EC2061D08C1822312D400F1
:1010A000A68881470147E51642864E8597000000D5
:1010B000E78060B041011713FFFF670063024A86B3
:1010C0000A8597F0FFFFE78000234DBF1713FFFF4E
:1010D000E70263FFB335B000011185052A891315B6
:1010E000F601336515012308B1009305110136841B
:1010F0003AC632C03EC442C297F0FFFFE780801D6F
:10110000A2471248425593D68700230BF10093055E
:10111000910193578800A30AD100A30BF100230C7F
:10112000010197F0FFFFE780E01A324702460328EB
:101130000400B337E000835644009207914411C283
:10114000A1444A85A68842860C0897F0FFFFE780F5
:1011500040772A8919E5A685228597B0FFFFE780A9
:10116000E0AA4A8505611713FFFF670003F817130C
:10117000FFFFE702A3F301113EC68647B335B00077
:101180008505AA891315F6015D8D2308B100930525
:10119000110136843A89B28442C446C297F0FFFFF7
:1011A000E780401322489248164593578800A30AC7
:1011B000F1009305910193D78800230B0101A30B44
:1011C000F100230C110197F0FFFFE780A0103247D8
:1011D000104083564400B337E0009207032809000B
:1011E000914891C0A1480C084E8597000000E78007
:1011F000809CAA8401E9835544004A8597B0FFFF8B
:10120000E780C0A0268505611713FFFF670043ED47
:10121000AA959307F00F171701001307A7A46317E8
:10122000B50013C5F7FF1375F50F828005058346DA
:10123000F5FFB58FBA9783C70700D5B703574500A9
:1012400014419307F00F171601001306A6A1369755
:1012500042074183139506014181631BE500AD8F71
:10126000B29703C50700130515F3133515008280E7
:10127000850603C5F6FFA98FB29783C70700D9BFBC
:101280001713FFFFE70223E4B28736842E86BA865F
:10129000AA853E85BA8497F0FFFFE7806052634FCE
:1012A0000500228597E00000E78060802A86A686F8
:1012B000A285268597F0FFFFE78080501713FFFF78
:1012C0006700A3E21713FFFFE70243DE5D712A8B7D
:1012D000AE8A17150100130565962C00B284368A74
:1012E000BA893E8997F0FFFFE780C04F2A845DE10D
:1012F00034104146DA85280097F0FFFFE780404C24
:101300002A8449E98547A303F100A6C29307710027
:101310002408BEC4A68685470D462C18281002DC7A
:1013200002DED6C0BEC697F0FFFFE78000442A84E5
:1013300035E183477102A6860D4693F7F707230030
:10134000FA00C1473EDE2C188947281026DCA3038B
:10135000F10097F0FFFFE78040412A8405ED414608
:10136000A6854E8597D00000E78060488D47A68609
:101370000D462C182810A303F10097F0FFFFE7801B
:10138000C03E2A8401E94146A6854A8597D00000DF
:10139000E780E045228561611713FFFF670043D4B2
:1013A0001713FFFFE70223D297F70000938707EF99
:1013B000984383C7470079712A89AE8417150100C5
:1013C000130545880C083AC42306F10097F0FFFF87
:1013D000E78040412A8405ED14104146CA8508087B
:1013E00097F0FFFFE780C03D2A8415E114081546F9
:1013F0002C00081097F0FFFFE780803C2A8401E969
:1014000021462C08268597D00000E780403E2285A3
:1014100045611713FFFF670043CD1713FFFFE70276
:1014200083CA97F70000938767E79C477971AA847E
:101430002E8417150100130565810C083EC697F030
:10144000FFFFE780203A0DE914104146A685080801
:1014500097F0FFFFE780C03605E1140811466C00E5
:10146000081097F0FFFFE780A03519E58347F101E9
:1014700093F7F7032300F40045611713FFFF67009C
:10148000C3C61713FFFFE70203C43688A14881478C
:101490000147E54697F0FFFFE780A0421713FFFFE3
:1014A0006700A3C41713FFFFE702E3C13688A14812
:1014B00081470147E54697F0FFFFE780C06F1713AC
:1014C000FFFF670083C21713FFFFE702C3BF0111CD
:1014D0002A842E850C0832C697F0FFFFE780803003
:1014E00009ED3247970601009386C6741008C1457E
:1014F000228597000000E780E0D805611713FFFF01
:101500006700A3BE1713FFFFE702E3BB4111C1470A
:101510002EC032C48A8509463EC23EC697F0FFFF00
:10152000E780A02441011713FFFF670003BC1713D6
:10153000FFFFE70243B94111AE8613061009AA85E1
:101540000A8502C002C202C402C697F0FFFFE7800C
:10155000202741011713FFFF670023B91713FFFF6F
:10156000E70263B63287970601009386A66E2E8641
:101570009305000297000000E780C0D01713FFFF1B
:101580006700A3B61713FFFFE702E3B37971C14702
:101590002ACC2ED032D42C080D4628003ECE3ED286
:1015A0003ED602C402C602C802CA97F0FFFFE78017
:1015B000C01B45611713FFFF670023B31713FFFF1D
:1015C000E70263B00111AA842E84170501001305F8
:1015D000E5688A8597F0FFFFE780C02015E51408CD
:1015E0004146A6850A8597F0FFFFE780601D09ED5B
:1015F0008347E1010347F101A207D98FCA07C983D5
:101600006177D98F2310F40005611713FFFF67007E
:10161000C3AD15CD1713FFFFE702E3AA9747FF1FDE
:101620009387C77090439745FF1F93856570174553
:10163000FF1F1305A56B97D00000E78000C5174575
:10164000FF1F1305A56A1713FFFF670003AA1745BD
:10165000FF1F1305A56982808DCD1713FFFFE702D9
:1016600083A69747FF1F9387676C944301112E84CD
:101670000A869745FF1F9385A56B97D00000E780EA
:1016800040C60A850294014505611713FFFF6700F4
:10169000C3A57D5582801713FFFFE702C3A297D031
:1016A0000000E78080D19747FF1F23A1A76817F5A7
:1016B000FFFF1305E5C997B00000E780C07417135A
:1016C000FFFF670083A21747FF1F13076768931781
:1016D000150008433E95FD572310F500828017132F
:1016E000FFFFE702439E2A84084009E51713FFFF26
:1016F0006700A39F1C4158401CC06313E5005CC0F9
:101700008347550023200500F99BA302F50097A00D
:10171000FFFFE780207CC9BF1713FFFFE702039993
:101720009747FF1F9387C76498432A8411CB834749
:10173000350093F7070289C70355050089450297CD
:101740001305440197B00000E780403B8355040037
:101750000355E40097300000E780A00C485819C5F5
:1017600097A0FFFFE7800077232A04021305840374
:1017700097000000E780E0F68144B1499790FFFFB1
:10178000E780C06D63CBA4028347340023200404A8
:1017900093F727FCA301F40000489790FFFFE78030
:1017A000E06C13161500814522859710FFFFE78036
:1017B00080941713FFFF6700A392B38734030329B4
:1017C000040385043E994A8597000000E78060F194
:1017D0002304090065B78347350093F7070299E3AF
:1017E000014582808357E500E39CB7FEC167FD1782
:1017F0006316F60005458280054599A81713FFFF7B
:10180000E702638C93170601C187B2842A840149D9
:101810006359F002835705009DCB01456367F600CD
:10182000034584003E953325A6001375F50F0DA0E2
:101830001C4813171900BA9783D70700E38E97FA4D
:1018400005099790FFFFE7806062E343A9FE014529
:101850001713FFFF670063891713FFFFE702038574
:10186000AE89AA849790FFFFE78000562A8497D01C
:10187000FFFFE780A02EAA86014713068401970583
:101880000000938585E41745FF1F1305A54C97902D
:10189000FFFFE780801C2A8925C98C441304C500FA
:1018A00022859E0593F5050897A0FFFFE780403C41
:1018B000CC4083877400E18163DD070493E505086C
:1018C000228597A0FFFFE780A03A0D46938544004C
:1018D000228597A0FFFFE780C03683D504002285CC
:1018E00097A0FFFFE780E03D83D52400228597A0E5
:1018F000FFFFE780003D03D6490083A5090022854C
:1019000097A0FFFFE780E0334A851703FFFF6700DA
:10191000237D93F5F5076DB71703FFFFE702A37A61
:1019200001112A84328532C697A0FFFFE780E027A5
:101930009780FFFFE7806034835704001747FF1F3D
:101940001307875A3246231BF100930700F8A30DB3
:10195000F1001C471843231AA1008983858BB30724
:10196000F740B28548083ECE231C0100230D01003C
:1019700097000000E78080EE05611703FFFF670016
:10198000C3761703FFFFE7026372004101453DC4C0
:101990009304C40026853289AE8997A0FFFFE780B3
:1019A000C02495452A8A2685035B040197A0FFFF82
:1019B000E7802021268597A0FFFFE780603E8D45C8
:1019C000AA8A268597A0FFFFE780A01F268597A0FB
:1019D000FFFFE780E03C5C48420A135A0A01D297B5
:1019E0005CC423186401814763983A0146054D8120
:1019F000330625419337160013F5F70F1703FFFF42
:101A00006700036E1703FFFFE702636989692A8B8A
:101A1000AE8B328AB68A81440144314CFD199790CD
:101A2000FFFFE780A04363CDA4009790FFFFE7800E
:101A3000E045018D33B5AA001703FFFF6700A369D6
:101A40003389840383270B003E9963170A00834779
:101A5000890085043E94E1B703560A00DE854A8575
:101A600033F6C90097000000E780E0F16DD105452D
:101A7000E1B71703FFFFE702036501112A847C0029
:101A80000355E5003ECAB70707003ECC7C003ECEBA
:101A900097200000E78020082A898545480897A0FC
:101AA000FFFFE78020399945480897A0FFFFE780AE
:101AB000E015AA844A8597200000E780A0082380CB
:101AC000A4009747FF1F938727429C434166130654
:101AD00006F09396870113D78701558F93D6870019
:101AE000F18E558FA207B706FF00F58FD98F1146EB
:101AF0002C00138514003EC497D00000E78020CF4F
:101B00005008A38204008945228597000000E780E1
:101B1000E0E019C9AA851305840397A0FFFFE780B9
:101B2000E0313C4085073CC005611703FFFF6700BB
:101B3000C35B1703FFFFE70203599790FFFFE7809E
:101B4000E0342A8405049790FFFFE78020333305B3
:101B5000A402F14791453305F50297200000E78084
:101B600020BA11E565551703FFFF67000358974733
:101B7000FF1F23A7A71E9790FFFFE78020312A842D
:101B800005049790FFFFE780602F3305A402894585
:101B9000060597200000E780A0B669D59747FF1F8C
:101BA00023A8A71A9790FFFFE780402E2A840504F8
:101BB0009790FFFFE780802C3304A4029747FF1F14
:101BC000239A87189790FFFFE780402C2A849790EC
:101BD000FFFFE780A02A930714003385A7029747E9
:101BE000FF1F239AA716970701009387E7CA174795
:101BF000FF1F2325F7160145BDB71703FFFFE702B7
:101C0000E34AAA842E8901449749FF1F9389C92D6D
:101C1000130A80069790FFFFE78040266347A400E1
:101C200001451703FFFF6700A34B3305440383A758
:101C300009024A86A6853E9597000000E780E0B934
:101C400019E10504C1BF0545E9BF1703FFFFE7021E
:101C50000345AA8A2E8BB28B368C3A8A8144014482
:101C60008149974CFF1F938C2C28130D8006979069
:101C7000FFFFE780A02063C9A40011E085494E85DD
:101C80001703FFFF670023453389A40383A70C02D2
:101C90005E86D6853E994A8597000000E780E0B3CE
:101CA0001DC19790FFFFE780601E0544636D4501ED
:101CB000D2866286DA851305090397000000E78063
:101CC000A0D411C1854985045DB71703FFFFE70262
:101CD000E33DC16441112A8901449749FF1F93895B
:101CE000A920130A8006FD1436C632C42EC297906E
:101CF000FFFFE780A01892452246B2466348A40041
:101D0000014541011703FFFF6700833D330544038D
:101D100083A709023E9509C683473500C18B9DC73D
:101D200091C68347350093F707028DC36306990078
:101D30008357E500639C27010357050001CB63E748
:101D4000E50083478500BA97E3CDF5FA050469BF3E
:101D50001703FFFFE7028335C1642A8901449749CD
:101D6000FF1F93896918130A8006FD149790FFFFDF
:101D7000E780C0106346A4001703FFFF67004336E7
:101D80003305440383A709023E958357E500638A20
:101D90009700630499006396270197000000E7808D
:101DA000E0970504E1B71703FFFFE702C32E896937
:101DB0002A8AAE8A328BB68B8144174CFF1F130CD4
:101DC000AC12930C8006314DFD199790FFFFE78010
:101DD000E00A63C6A4001703FFFF6700832F33895F
:101DE000940383270C028355CA015A863E994A857B
:101DF00097000000E780609E31C1814D15A03384BB
:101E0000AD038327090303D60B00D68533F6C9003B
:101E10003E94228597000000E780E0B609E9850D31
:101E20009790FFFFE7808003E3CBADFC01A82285FC
:101E300097000000E780E08A23040400850471B75E
:101E40001703FFFFE702A3254169AA8A014A174B3E
:101E5000FF1F130B6B097D19C14B054C9790FFFFBA
:101E6000E780C0016346AA001703FFFF6700A326AF
:101E700093098006B3073A0383290B02BE9983D7DF
:101E8000E900638E270163842A01639A570103A442
:101E9000890301E84E8597000000E780C0BD050A70
:101EA00075BF83570401639977099304C40026859D
:101EB00097A0FFFFE78060D385452A8D2685835C48
:101EC000040197A0FFFFE780C0CF268597A0FFFF02
:101ED000E780A0E762056185635905048D45268585
:101EE00097A0FFFFE780E0CD8945268597A0FFFFFB
:101EF000E78020CD8945268597A0FFFFE78060CC4D
:101F00008545268597A0FFFFE780E0CC8347050045
:101F1000094793F7F707639AE7009945268597A045
:101F2000FFFFE78040CBA30285014848337D2D01A8
:101F3000231894016A9548C40040A1BF1703FFFF0E
:101F4000E702631837E404008327041D829797474C
:101F5000FF1F83C767E61715FF1F1305655BA30007
:101F6000F5008327441C82978327841C814613062F
:101F7000F00F8145014582971703FFFF6700E316C5
:101F80001747FF1F130747D318439745FF1F83C504
:101F9000A5E29747FF1F9387A7E083468703034681
:101FA00097036397D5009747FF1F2387C7E0828079
:101FB00083C587010347A7036317B6009747FF1F31
:101FC000238CE7DE828003C687016317C70097472B
:101FD000FF1F2383D7DE828083C687011307500249
:101FE0006319D700930760021747FF1F2306F7DC2A
:101FF000828083C68701130660026315D6009307AB
:102000007002DDB783C7870155BF9747FF1F9387CE
:1020100027D9D44B0947638DE6081703FFFFE70272
:10202000830A1749FF1F1309E9D43E848347090037
:10203000918B9DCFB7E4040083A7041D829783A7EB
:10204000441C1745FF1F130565D3829783A7841C83
:1020500081461746FF1F034666D481450145829796
:1020600021C583470900ED9B1747FF1F2304F7D0C5
:102070008347040093F7F70F85CB91471747FF1F5E
:10208000232AF7D297000000E78080EB970000003A
:10209000E78040EFB7E70400BC4F41469145174544
:1020A000FF1F034565D082971703FFFF6700E30317
:1020B00082801703FFFFE70203018D47411163068A
:1020C000F504C5476308F50285476310F502974795
:1020D000FF1F2385A7CEB7E70400BC4B9305001074
:1020E0001745FF1F034545CC829741011703FFFFAA
:1020F0006700A3FF85471747FF1F2301F7CCB7E70A
:102100000400BC4B93050020E1BF9747FF1F938756
:1021100027C9D44B1147638DE600B7E7040083A7B6
:10212000071D8297B7E70400BC4B930500044DBF21
:1021300005491747FF1F232F27C783C7070032C64C
:102140002E8493F7F70FD5D3B7E4040083A7041DBB
:102150007D141374F40F8297E37689FCB245994796
:1021600003C61500E3F0C7FCFC4409061745FF1F32
:10217000130505C58297BC48930500081745FF1F46
:10218000034585C2829779BF1703FFFFE702A3F3D8
:102190001747FF1F1307C7C04047184B1C409746FF
:1021A000FF1F23A5F6C06316E4001747FF1F232176
:1021B000F7C0130584FE9790FFFFE78000AA035540
:1021C00064FF9780FFFFE780807297A0FFFFE780A2
:1021D00060D01703FFFF670043F11703FFFFE7021B
:1021E00083EE9747FF1F9387A7BBD84BDC4789C770
:1021F00097000000E78080F985471747FF1F232BD2
:10220000F7BA9747FF1F938727AB9C4393050002BC
:102210001745FF1F034545B983C787031747FF1FAE
:10222000230CF7B8B7E70400BC4B82971703FFFFF6
:102230006700A3EB9747FF1F23A6A7B6828017036B
:10224000FFFFE702A3E637E404007C4CA1451745F5
:10225000FF1F034565B582977C48A1451745FF1FC1
:10226000034585B49744FF1F938484B38297DC446D
:1022700089EB97000000E78080D91703FFFF670014
:1022800023E603D567FF9780FFFFE7804066AA89B2
:102290006DD1D84891476310F7027C4C91451745A2
:1022A000FF1F034565B082977C4891451745FF1F86
:1022B000034585AF829703A9490103D409018947E2
:1022C000B7E904001747FF1F2326F7AE83A7091DB0
:1022D00021044204829783C784011715FF1F130549
:1022E000252361191717FF1FA304F72283A7491C91
:1022F000418082979747FF1F238207AC83A7C91CA1
:10230000814609469375F40F4A85829711E99747EC
:10231000FF1F83C7E7BA89C79710FF1FE780E08BCD
:10232000B7E70400BC4F2146A1451745FF1F0345F1
:10233000A5A7829799B71703FFFFE702C3D893F7C2
:10234000052001112E8481CF97000000E78020E94D
:102350001345042005611703FFFF670003D993F7B6
:102360000510A9CF9744FF1F938484A3DC489700EE
:102370000000E78020C11747FF1F1307E7931843AA
:1023800083C78401034787036318F700DC4489C7C8
:1023900097000000E78080DF85471747FF1F232B4A
:1023A000F7A0B7E70400BC4B930500021745FF1FD9
:1023B0000345859F82971345041069BF93F705086D
:1023C000BDC79747FF1F83C7B79FE91719469745B2
:1023D000FF1F9385059F1305D10093F4F70F17494D
:1023E000FF1F0349E99D97C00000E7804040939795
:1023F0000401C1831747FF1F1307079D231DF10029
:10240000231CF1009747FF1F938787993ACE3ACA5A
:10241000D8432306010009CBDC43931589015408F6
:102420000D46E185680082971345040825B793F7A8
:102430002500A5C39747FF1F93878796D84B8947E9
:102440006306F7029747FF1F83C7C79213F727005A
:1024500011EF918B99CFB7E70400BC4F1306000A28
:1024600089451745FF1F034525948297134524008E
:10247000D5B59747FF1F938727849C4383C787035E
:102480001747FF1F230AF79297000000E78060DBE1
:10249000F1BF93F7050281CB97000000E78060DA77
:1024A0001345040245BD93F7850081CB97000000DA
:1024B000E780E0D21345840071BD93F7150081CB0E
:1024C00097000000E780A0B41345140061B593F7AE
:1024D000450081CB97000000E78060B313454400BE
:1024E00095BD93F7050495C39747FF1F83C7478B97
:1024F00091CB97000000E780A0A491471747FF1FEA
:10250000232AF78A13450404B1B593F70501014561
:10251000E38207E49747FF1F93878788D84B91474B
:102520006310F7049747FF1F9387C7849C4313D713
:1025300027008583D98F858B91E7B7E7040083A7B0
:10254000071D8297B7E70400FC4F91451745FF1F11
:1025500003458585829785471747FF1F232CF784FE
:1025600013450401C5BB9747FF1F238BA7948280A7
:102570001703FFFFE70223B59747FF1F23A8078232
:102580009747FF1F23A6078285471734FF1F1304B1
:10259000A4721747FF1F232FF7801C4083C78703B0
:1025A0001747FF1F230AF7809790FFFFE7804093AC
:1025B00029C59717FF1F23A1A7F61C401705000088
:1025C0001305A5D783C787031737FF1F2306F77E99
:1025D0001717FF1FA30EF7F29737FF1FA382077C81
:1025E000B7E7040083A7070882979737FF1F238D5B
:1025F000A77A1703FFFF670043AFB7C7898E93879A
:1026000067ED1717FF1F2329F7F045BF1737FF1F87
:1026100003470779795555E79737FF1F9387477821
:1026200003C7170005079736FF1FA38BE67603C77E
:1026300017008D463377D7029736FF1FA382E676C1
:1026400083C617001737FF1F13070767184393F652
:10265000F60FA9EE834787031737FF1F230EF77482
:1026600085471737FF1F230DF7729737FF1F938793
:1026700067709C430145998BA9E71703FFFFE702A9
:1026800083A437E404007C48C1451735FF1F034588
:10269000A57182973C4885451735FF1F0345C570D6
:1026A000829701451703FFFF670023A483C7170024
:1026B00085466395F6008347970379BF8347A70351
:1026C00061BF82809737FF1F83C7876DA1CF170334
:1026D000FFFFE702439F37E404009737FF1F238182
:1026E000076C7C4885451735FF1F0345E56B8297CE
:1026F0007C4C91451735FF1F0345056B82977C483D
:1027000091451735FF1F0345256A82973C48C1450F
:102710001735FF1F03454569829701451703FFFFE2
:102720006700A39C795582801703FFFFE702A399F6
:102730002A84035565FF9780FFFFE780401B97378A
:10274000FF1F9387E765D847BE841DEF9790FFFF73
:10275000E78080779C48232004009DEB9737FF1F7C
:1027600023A887649737FF1F23A28764B7E7040075
:10277000BC4B89451735FF1F03450563829701450B
:102780001703FFFF67006396630A8700184375BF4E
:1027900080C39737FF1F23AD8760C9BF7955CDB779
:1027A0001703FFFFE70223929737FF1F9387877175
:1027B00088432326050023240500510597A0000027
:1027C000E780C0331703FFFF670023921703FFFF63
:1027D000E702638F1734FF1F1304C46E1C404111BE
:1027E00099CF9C472302B5002AC61CC19700000060
:1027F000E78040FB1C409C4B99C3324582974101C6
:102800001703FFFF6700638E1703FFFFE702A38B29
:102810004111444D328532842EC69790FFFFE780E8
:10282000C0522AC422859790FFFFE780205403A856
:102830004400630C0800B245835744001840224608
:1028400083D54500AA862685029841011703FFFF1C
:102850006700A3891703FFFFE702E386404D1DC809
:1028600008C097050000938565031305440197A0F0
:102870000000E78040169737FF1F9387A7649C43AB
:10288000014589E79737FF1F23AE87621703FFFFD4
:102890006700A3857D55DDBF1703FFFFE702A38215
:1028A000011168009305F00F02C602C802CA02CCEB
:1028B00002CE97000000E780A0F105611703FFFF3B
:1028C0006700A3829737FF1F9387C75F9C43D84752
:1028D000A1679D076319F70217F3FEFFE702A37EC6
:1028E000011132859790FFFFE7802046230AA1005F
:1028F0008145680097000000E78080ED056117F3CF
:10290000FEFF6700837E82809737FF1F9387875B78
:102910009C43D847A167938777036319F70217F39E
:10292000FEFFE702437A011132859790FFFFE780AF
:10293000C041230AA1008145680097000000E7809C
:1029400020E9056117F3FEFF6700237A828097373D
:10295000FF1F938727579C43D84795476316F70473
:1029600017F3FEFFE7022376011132853284979038
:10297000FFFFE780803D230AA10022859790FFFF9B
:10298000E780C03E83574400231BA10081453ECC15
:102990001C4068003ECE97000000E78060E30561C0
:1029A00017F3FEFF670063748280930785FF8DC372
:1029B0008327C5FF91CFDC4B81CF17F3FEFFE702E2
:1029C0008370032585FF829717F3FEFF6700E3718D
:1029D000828017F3FEFFE702036F2A843285979007
:1029E000FFFFE7808036BD4763EBA700184493776D
:1029F000F5000345B70041995D8DA305A70017F3C6
:102A0000FEFF6700836E17F3FEFFE702C36B011141
:102A10007C003ECAB70707003ECC7C003ECE5C4D32
:102A2000A9C72A8413858700AE8497A00000E78099
:102A3000E0FCA1652A899D0548089770FFFFE780A3
:102A4000603E9305803EB345B902480893F5F50F03
:102A50009790FFFFE780C021014781465008A68577
:102A600022859770FFFFE7804061056117F3FEFF45
:102A70006700A36717F3FEFFE702E3649700000017
:102A8000E780A0F817F3FEFF6700236617F3FEFF49
:102A9000E702636301117C00AE843ECAA165B707FB
:102AA00007002A843ECC48087C00938575033ECEFF
:102AB0009770FFFFE78000371C44480883C5B700C4
:102AC000BD899790FFFFE780A01A50080147814613
:102AD000A68522859770FFFFE780205A056117F3CE
:102AE000FEFF6700836017F3FEFFE702C35D2A84E1
:102AF000AE8497000000E78000EEA685228597004F
:102B00000000E780E0F817F3FEFF6700035E17F3AD
:102B1000FEFFE702435B97000000E78060F717F3D2
:102B2000FEFF6700835C17F3FEFFE702C35903292A
:102B3000C5014111630809022A843285B284979045
:102B4000FFFFE78080202AC626859790FFFFE78059
:102B5000E021832749002A8691C7DC4781C7B24517
:102B600022858297410117F3FEFF6700035817F390
:102B7000FEFFE7024355444D91CC2A84328597905D
:102B8000FFFFE780A01EDC40AA8589C79C4799C348
:102B90002285829717F3FEFF6700235517F3FEFF88
:102BA000E702C350032AC5014111630D0A062E89AD
:102BB000AA849545328532849770FFFFE78080268E
:102BC000854522859790FFFFE7804004AA89CA8542
:102BD00022859790FFFFE780A00B83274A008DCBCB
:102BE000DC439DC722859790FFFFE780A0008327E5
:102BF0004A00104083564400DC437115A307A1002E
